:0200000460009A
:100000004643464200000156000000000103030081
:1000100000000000000000000000000000000000E0
:1000200000000000000000000000000000000000D0
:1000300000000000000000000000000000000000C0
:1000400000000000010408000000000000000000A3
:100050000000800000000000000000000000000020
:100060000000000000000000000000000000000090
:100070000000000000000000000000000000000080
:10008000EB04180A063204260000000000000000FD
:10009000050404240000000000000000000000002F
:1000A0000000000000000000000000000000000050
:1000B0000604000000000000000000000000000036
:1000C0000000000000000000000000000000000030
:1000D00020041808000000000000000000000000DC
:1000E0000000000000000000000000000000000010
:1000F0000000000000000000000000000000000000
:10010000D8041808000000000000000000000000F3
:100110000204180804200000000000000000000095
:1001200000000000000000000000000000000000CF
:10013000600400000000000000000000000000005B
:1001400000000000000000000000000000000000AF
:10015000000000000000000000000000000000009F
:10016000000000000000000000000000000000008F
:10017000000000000000000000000000000000007F
:10018000000000000000000000000000000000006F
:10019000000000000000000000000000000000005F
:1001A000000000000000000000000000000000004F
:1001B000000000000000000000000000000000003F
:1001C000000100000010000001000000000000001D
:1001D000000001000000000000000000000000001E
:1001E000000000000000000000000000000000000F
:1001F00000000000000000000000000000000000FF
:10020000FFFFFFFFFFFFFFFFFFFFFFFFFFFFFFFFFE
:10021000FFFFFFFFFFFFFFFFFFFFFFFFFFFFFFFFEE
:10100000D100204327140060000000000000000011
:10101000201000600010006000E00160000000008F
:101020000000006000EC010000000000FFFFFFFF77
:10103000FFFFFFFFFFFFFFFFFFFFFFFFFFFFFFFFC0
:10104000FFFFFFFFFFFFFFFFFFFFFFFFFFFFFFFFB0
:10105000FFFFFFFFFFFFFFFFFFFFFFFFFFFFFFFFA0
:10106000FFFFFFFFFFFFFFFFFFFFFFFFFFFFFFFF90
:10140000884207D0904205D251F8043B40F8043B93
:101410008242F9D87047884204D2002340F8043B46
:101420008142FBD870472DE9F843644A644B5A6403
:10143000644A1A644FF42A029A63634B9D46BFF3D1
:101440004F8FBFF36F8F00F01DFA604B0822604989
:101450006048C3F85421604AFFF7D2FF5F4A6049F1
:101460006048FFF7CDFF60496048FFF7D4FF4FF4B5
:1014700070025F4B5F491A6000235F4A42F82310F5
:1014800001335D4DB02BF9D15C4B80215C4A03F8F0
:10149000011B9342FBD14D4C4FF08037594A5A4BB8
:1014A000DFF89C91DFF89C811D60C4F80471C4F8DA
:1014B0000091C4F8F470C4F8F0801368534E43F4FC
:1014C000E02313604FF0FF32F36923F07F0343F012
:1014D0004003F361736A23F07F0343F040037362B8
:1014E000374B9A66DA661A675A6700F0CEF9484BAE
:1014F0006322AB63474BEB630025474B1A60032223
:101500005D6043F8042C454AC3F80C2D444A136827
:1015100043F080731360434A136843F00103136080
:10152000414B1A68414B1A6000F068FBC4F8047123
:101530003F48C4F80091C4F8F470C4F8F08000F09B
:1015400007FDF36E43F44053F3663A4B1D60C3F856
:101550000851C3F81851C3F82851C3F8385103F59E
:10156000A0239A6BD20708D4334A5A6542F6156213
:101570001A659A6B42F001029A639A6842F001126E
:101580009A6000F0F1F900F091FC00F0C1FC00F06D
:1015900063FB00F078F9294A1368284C132BFBD918
:1015A00000F0E8FB2368B3F5967FFBD300F06CF9FD
:1015B00000F0D2FC00F0A8FC30BFFDE7BFAAAAAA49
:1015C00000C00A40070020000080062000800D4077
:1015D0000C27006000000000F07E0100C0360020F3
:1015E00000A601600000002000740020C03600202A
:1015F00088ED00E0D55401000034002000E400E054
:10160000A0E400E024ED00E008ED00E000C00F40A1
:10161000BD660100C166010014E000E0000020206A
:10162000FCED00E0001000E0041000E098670020EE
:10163000002CA330004008400000C0569C670020EA
:101640001B1018200C0D1113F8B58F005C4B0C46C5
:1016500038461A6000F074FC5A4B054618601E4666
:1016600020B92021584800F06FFCA3E03A46002141
:1016700000F05EFC25F01F033D44BFF34F8F534A3B
:10168000136020339D42FBD8BFF34F8FBFF36F8FA2
:101690004F4B32681A604F4A4F4B1C80D36F43F454
:1016A0004023D3674D4B4E4A1A674FF43162C3F85B
:1016B000802042F21072C3F890201A6F22F48052F8
:1016C0001A67196F454A0029FBDAD2F870310126F2
:1016D00044494FF4803523F40003434823F4004386
:1016E000C2F87031136F23F48033136702F51032A0
:1016F000D36923F4406343F40063D361936A23F412
:10170000FF7323F0010343F079039362A2F5A02253
:10171000536823F4002323F0070343F400235360AA
:101720000022324B1A66DE60196131495D619861B1
:10173000D961C3F8E020C3F88C6006F1E066C3F815
:101740009060C3F89450C3F898000320C3F89C102D
:101750002849C1F82801C1F82401C1F88001D3F853
:101760008810254841F01041C3F88810234999603A
:101770002349C1F8200123484FF08075056080F8A7
:1017800083237F20204A1070204AC1F85821D0219D
:101790001F4A204811704021A2F23E3211601621EA
:1017A0009A6842F480729A6000F0CEFB21461A4893
:1017B00000F0B6FB1848BDE8F84000F0B5BB00BF2C
:1017C000CC65002000420020AA29002070EF00E034
:1017D0000866002000C00F40AC67002000800D406C
:1017E0001B201100010000471B1F01000040384072
:1017F000001F1F1F00801F402100000001000090FB
:101800000034002004E100E038E400E0750000004E
:1018100046E400E0CB29002000300020024B18688D
:1018200008B100F079BB7047004200200004084B6B
:10183000012200F47020C3F8A010C3F8A400C3F87C
:10184000B0205A69D207FCD50122014B5A6170477A
:1018500000402A40094B0A4AC3F8A000C3F8A4205C
:101860000122C3F8B0205969044AC907FBD5D2F850
:101870000001212380B25361704700BF00402A401D
:101880000400030070477047704710B5214A0020DC
:10189000214C1023214920601360214B1960112134
:1018A000116020491960122111601F4919601F49F8
:1018B00011601F4919601F4911601F4919601F49B4
:1018C00041F0150111601E49196001F181510D317E
:1018D00011601C4919601C4911601C4919601C49A0
:1018E00011601C4919601C4911601C4A1A600123CF
:1018F0002360BFF34F8FBFF36F8F194B1860BFF397
:101900004F8FBFF36F8F174A136843F44033136050
:1019100010BD00BF9CED00E094ED00E03F00001022
:10192000A0ED00E0250008030900100013002000CE
:101930002100020714000020250008130074002075
:101940000900001027000B1317000040330010138C
:10195000180000602F000B07190000702F000B13F8
:1019600050EF00E014ED00E073B58F4B4FF40054DE
:101970008E4A8F49C3F85C22C3F8601248F20C719A
:10198000C3F86422A2F53042C3F8682202F5E042AF
:10199000C3F86C22C3F87022C3F87422C3F878220B
:1019A0001822DA661A675A679A67DA67C3F88020DE
:1019B000C3F88420C3F888200122C3F82C27C3F879
:1019C0003027C3F83427C3F83827C3F83C27C3F8B7
:1019D0005027784A936923F0604323F4407343F01F
:1019E000204343F440739361D2F8843043F00C03F6
:1019F000C2F88430704B1A6842F002021A601A680A
:101A000011406E4A0A436E491A604FF0FF325A6025
:101A100002F57702886802F56052024042F00052F7
:101A20009A60DA6822F07802DA60664A186A024040
:101A300042F0004242F040021A62624A186A0240D2
:101A4000614842F0004242F040025A625F4A9A62A4
:101A5000DA62D1F8B82022F03F0242F00102C3F866
:101A6000B820D1F8BC2040F2056122F03F0242F0DC
:101A70000102C3F8BC2000221A611C661867C3F873
:101A800080105C665867C3F884101968504821F0CC
:101A9000020119604F4999610221D9614E4941F80B
:101AA000042B8142FBD11A6842F001021A60424ABB
:101AB0001468414B14F00104FAD1464A022621462B
:101AC00020469A6140F2F562DE61C3F8002240F2DE
:101AD0006642C3F8102240F29942C3F820223F4ADE
:101AE000C3F8302242F20142C3F8342240F23542B8
:101AF000C3F840223A4AC3F850223A4AC3F8542263
:101B0000394AC3F8602242F20122C3F86422FFF787
:101B10008DFE21460120FFF789FE21463046FFF762
:101B200085FE2046FFF796FE45F60D530546984282
:101B300031D121460420FFF779FE20464FF4000101
:101B40002A4CFFF773FE4FF400010120FFF76EFEF1
:101B50004FF400013046FFF769FE4FF40000FFF735
:101B600079FEA84207D14FF400010420FFF75EFE82
:101B70001023237001E0082323701D4900231D4A10
:101B80002078521A0093012302EB00521A4800F009
:101B9000E7F902B070BD10222146174802B0BDE837
:101BA000704000F0C5B900BF00801F40F9B00100CF
:101BB000F910010000C00F4000402A401200FFFF52
:101BC00000802A4000FFF07C63000200FF000F83CA
:101BD00000432A40F05AF05A00422A409F0418302D
:101BE000EB06180A063201263806180AAB720020E6
:101BF0000000007000000070C0730020F0B5154BAD
:101C000040204FF480314FF480544FF400554FF48E
:101C1000404643F242071A6912F0020F03D09E6158
:101C200059619F61F7E712F4005F01D15D61F2E74E
:101C300012F4805F01D15C61EDE7002AEBDA12F467
:101C4000803F01D09961E6E7520601D45861E2E78E
:101C5000F0BD00BF00800D40394AB3EE096A394833
:101C600013689FED395A23F0010310B51360032365
:101C7000364C1361364BD3F8E030D9B2016007EE31
:101C8000901AC3F30B201B0DB8EEE77A314907EE2B
:101C9000900A2060F8EEE76A07EE903A37EE455A70
:101CA0002D4BF8EEE77A37EE466A77EEE67A81ED6D
:101CB000006A25EE275AC3ED007A1368C5EE065A6E
:101CC00075EEA65AFCEEE55A15EE901ADFED235A92
:101CD00037EE657A43EA0153136027EE277A204BEB
:101CE00066EE277AD2F81011C7EE065A35EEA67ABC
:101CF000BCEEC77A17EE100A87EE867A03EA004335
:101D00000B43C2F81031D2F8101177EE267AFCEEB0
:101D1000E77A17EE903AC3F30B030B43C2F8103186
:101D2000136843F00203136000220E4B1A700E4A30
:101D30000E4BC3F8402101220D4B1A6010BD00BFAD
:101D400080810D40886700200000AA42846700203F
:101D500000441F408C670020906700200000B442C0
:101D60000000FF0F40E400E079560100003400203D
:101D700008E100E038B540F661722D4BC3F8202130
:101D800000F0F2F82B4A2C49D2F8803043F00303DC
:101D9000C2F8803040F20442284BC3F86021284A40
:101DA0001068014019B9D3F8A811890718D04FF06D
:101DB00000415163D3F8402142F00202C3F84021B0
:101DC0001E4AD2F840319B07FBD44FF400321D4B22
:101DD00019201A604FF00042194B9A6300F0ACF8DA
:101DE000174B00214FF08042174D144C9A63284640
:101DF00019600A234FF42072C4F8A83100F098F853
:101E00004FF48103114A2B604FF480032B6440F29E
:101E10004313C4F85851C4F848310D4BC3F8042299
:101E20000C4B4FF400321A600123C4F8403138BD26
:101E300000800D4000C00F40001C1E0000002E401E
:101E400000900D408CE200E00000002035590100B8
:101E5000003400200CE100E008B50E4B1B6E9B0720
:101E600001D4FBBE16E072B600220B4BC3F8402132
:101E7000A3F50D13094A1A64A3F1FF53A3F52B230D
:101E80009D46BFF34F8F064B06480360064B1B6809
:101E90009B68984700441F4000002E40030020002C
:101EA000000012EB008020201C0020000F4BDA6E97
:101EB00042F44032DA66DA6E42F44072DA66A3F532
:101EC000603340F237625A64A0229A649A6C120618
:101ED000FCD4074B40F237625A64A0229A649A6C91
:101EE00012F08002FBD1034B1A70704700C00F4004
:101EF00000800C40A2720020F8B500BFF8BC08BCFE
:101F00009E467047000000005FF800F0756A01000F
:101F10005FF800F0C96E01005FF800F095700100F5
:101F20005FF800F03B6901005FF800F07D68010098
:101F30005FF800F0155301005FF800F0B5530100A1
:101F40005FF800F0857001005FF800F02163010088
:101F50005FF800F08D6B01005FF800F03970010050
:101F60005FF800F0876F01005FF800F0915E0100FC
:101F7000A902000039AF000021B20000A9BD000095
:041F800025F7000041
:101F8400FF7FFF7FFF7FFF7FFF7FFF7FFF7FFF7F5D
:101F9400FF7FFF7FFF7FFF7FFF7FFF7FFF7FFF7F4D
:101FA400FF7FFF7FFF7FFF7FFF7FFF7FFF7FFF7F3D
:101FB400FF7FFF7FFF7FFF7FFF7FFF7FFF7FFF7F2D
:101FC4000180018001800180018001800180018005
:101FD40001800180018001800180018001800180F5
:101FE40001800180018001800180018001800180E5
:101FF40001800180018001800180018001800180D5
:1020040001800180018001800180018001800180C4
:1020140001800180018001800180018001800180B4
:1020240001800180018001800180018001800180A4
:10203400018001800180018001800180FF7F018097
:1020440001800180FF7F018001800180FF7F01808A
:1020540001800180FF7F018001800180FF7F01807A
:1020640001800180FF7F018001800180FF7F01806A
:1020740001800180FF7F01800180FF7FFF7F01805D
:1020840001800180FF7F01800180FF7FFF7F01804D
:1020940001800180FF7F01800180FF7FFF7F01803D
:1020A40001800180FF7F01800180FF7FFF7F01802D
:1020B40001800180FF7F0180FF7FFF7FFF7F018020
:1020C400FF7F0180FF7F01800180FF7FFF7F018010
:1020D40001800180FF7F0180FF7FFF7FFF7F018000
:1020E400FF7F0180FF7F01800180FF7FFF7F0180F0
:1020F40001800180FF7FFF7FFF7FFF7FFF7F0180E3
:10210400FF7F0180FF7F01800180FF7FFF7F0180CF
:1021140001800180FF7FFF7FFF7FFF7FFF7F0180C2
:10212400FF7F0180FF7F01800180FF7FFF7F0180AF
:10213400018001800180FF7FFF7FFF7F018001809C
:10214400FF7F0180018001800180FF7F0180018089
:1021540001800180FF7FFF7FFF7FFF7FFF7F018082
:10216400FF7F0180FF7F01800180FF7FFF7F01806F
:102174000180FF7F0180FF7FFF7FFF7F018001805F
:10218400FF7FFF7F018001800180FF7F018001804C
:1021940001800180FF7FFF7FFF7FFF7FFF7F018042
:1021A400FF7F0180FF7F01800180FF7FFF7F01802F
:1021B400FF7FFF7F0180FF7F0180FF7F018001801F
:1021C400FF7FFF7F018001800180FF7F018001800C
:1021D40001800180FF7FFF7FFF7FFF7FFF7F018002
:1021E400FF7F0180FF7F01800180FF7FFF7FFF7FF2
:1021F400FF7FFF7F0180FF7F0180FF7F01800180DF
:10220400090180961180FF3A81550A3601082A0493
:10221400000000F02B040000014021800A13800A12
:102224002980FF0000000000000000000000000002
:10223400000000000000000000000000000000009A
:10224400000000000000000000000000000000008A
:10225400000000000000000000000000000000007A
:10226400000000000000000000000000000000006A
:10227400000000000000000000000000000000005A
:10228400000000000000000000000000000000004A
:10229400000000000000000000000000000000003A
:1022A4000000007F41414141417F00002731272147
:1022B4007100000077417711710000007741774188
:1022C40071000000175177414100000077117741F8
:1022D4007100000077117751710000007741474188
:1022E4004100000077517751710000000020243E26
:1022F40004000000594B5B4BD900000000000000B3
:1023040000000000000000000000000000000000C9
:1023140000000000000000000000000000000000B9
:102324000000000000000000000000183C3C1818E9
:10233400001800363600000000000036367F367F75
:102344003636000C3E031E301F0C00006333180C9D
:102354006663001C361C6E3B336E000606030000E9
:10236400000000180C0606060C1800060C181818B5
:102374000C060000663CFF3C660000000C0C3F0CA1
:102384000C000000000000000C0C060000003F00E0
:1023940000000000000000000C0C006030180C0667
:1023A4000301003E63737B6F673E000C0E0C0C0C44
:1023B4000C3F001E33301C06333F001E33301C30EC
:1023C400331E00383C36337F3078003F031F3030F3
:1023D400331E001C06031F33331E003F3330180C1A
:1023E4000C0C001E33331E33331E001E33333E30B9
:1023F400180E00000C0C00000C0C00000C0C00006B
:102404000C0C06180C0603060C180000003F000014
:102414003F0000060C1830180C06001E3330180C50
:10242400000C003E637B7B7B031E000C1E33333F9A
:102434003333003F66663E66663F003C6603030333
:10244400663C001F36666666361F007F46161E16FB
:10245400467F007F46161E16060F003C6603037374
:10246400667C003333333F333333001E0C0C0C0CC7
:102474000C1E007830303033331E006766361E364B
:102484006667000F06060646667F0063777F7F6BEC
:1024940063630063676F7B736363001C366363630A
:1024A400361C003F66663E06060F001E3333333B80
:1024B4001E38003F66663E366667001E33070E38D8
:1024C400331E003F2D0C0C0C0C1E003333333333FE
:1024D400333F0033333333331E0C006363636B7F4A
:1024E4007763006363361C1C3663003333331E0C7E
:1024F4000C1E007F6331184C667F001E060606061C
:10250400061E0003060C18306040001E1818181828
:10251400181E00081C3663000000000000000000C4
:102524000000FF0C0C18000000000000001E303EEC
:10253400336E000706063E66663B0000001E33034A
:10254400331E003830303E33336E0000001E333FFC
:10255400031E001C36060F06060F0000006E333300
:102564003E301F0706366E666667000C000E0C0CC4
:102574000C1E00300030303033331E070666361E22
:102584003667000E0C0C0C0C0C1E000000337F7F11
:102594006B630000001F333333330000001E3333FA
:1025A400331E0000003B66663E060F00006E3333A8
:1025B4003E307800003B6E66060F0000003E031EAE
:1025C400301F00080C3E0C0C2C1800000033333371
:1025D400336E0000003333331E0C000000636B7F46
:1025E4007F3600000063361C36630000003333334B
:1025F4003E301F00003F190C263F00380C0C070C1E
:102604000C38001818180018181800070C0C380C8F
:102614000C07006E3B0000000000000000000000FA
:10262400000000A2A0D0EBE5B9334487C068B6B778
:102634002699C7001603550053004200200053009A
:1026440065007200690061006C00180354006500A5
:1026540065006E00730079006400750069006E0007
:102664006F000403090409024B00020100C0320890
:102674000B00020202010009040000010202010031
:102684000524001001052401010104240206052487
:102694000600010705820310001009040100020A64
:1026A4000000000705030240000007058402400003
:1026B4000009024B00020100C032080B00020202B2
:1026C40001000904000001020201000524001001B8
:1026D400052401010104240206052406000107055E
:1026E400820310000509040100020A000000070526
:1026F4000302000200070584020002000A06000229
:08270400EF0201400100010099
:10270C0000000000000000000000000000000000BD
:10271C0000000000000000000000000000000000AD
:10272C000E480F4B02881B6833F8121001320D4B08
:10273C0019800D4B19884B00013B13409BB2038051
:10274C0013B90A4A137004E0994205D10122074BD0
:10275C001A704022064B1A60704700BFAE6700200B
:10276C000866002022403840AC6700204A31002027
:10277C0008E200E0194B1A78194B70B5194E1A4D36
:10278C001A4C8AB131881B682868984731882A68A6
:10279C00490822F01F0302EB8102BFF34F8F236025
:1027AC0020339A42FBD814E031882A6848081B6809
:1027BC0002EB8000984733882A685B08990053180D
:1027CC0023F01F020B44BFF34F8F22602032934241
:1027DC00FBD8BFF34F8FBFF36F8F70BD4A31002012
:1027EC00CC650020AC6700200042002070EF00E0B8
:1027FC00614B1B782DE9F04F03F0FF0299B00B925F
:10280C00002B00F0B6805D4B05AD4FF0000E4FEA8B
:10281C006109B3F90820D3F804A0F4460C92B3F97B
:10282C001420D3F810B00D92B3F92020544C0E9212
:10283C00B3F92C200F92B3F938201092B3F944203D
:10284C0011921A680592DA6806929A6907925A6A86
:10285C0008921A6B0992DA6B0A92DA6902929A6AF6
:10286C0003925A6B0492D3F840800A99099A089BF8
:10287C000190E0CD0198CC4500F1040001900AEBE9
:10288C00050016900BEB0600159002983844149036
:10289C0003981844139004981044129008EB01000C
:1028AC00179021DB29EAE971069A079C01FB0B20A2
:1028BC00029A059B01FB0245039A089C01FB0A3313
:1028CC0001FB0246049A099C01FB02440A9A01FB93
:1028DC000821BEF1000F4CD0284A1360D0609561DE
:1028EC0056621463D16344E0C5F305250C98C6F316
:1028FC000526C7F3052734F91550C3F3072334F91C
:10290C001660C2F3072245430D9834F9177004EB97
:10291C00430346430E98B3F9803004EB4202F6129F
:10292C0047430F98C1F3072106EBE525B2F9802048
:10293C00434304EB410105EBE7250CF1010CB1F924
:10294C00801005EBE325109B159E5A43119BDDF877
:10295C002CE0594305EBE225019B12AA05EBE1257E
:10296C0017992DB223F8045C23F8025C169D8CCACF
:10297C0080E719B0BDE8F08FAD7200202C66002006
:10298C00841F006010B5054C237833B9044B13B188
:10299C000448AFF300800123237010BDD0600020E9
:1029AC0000000000F47E0100084B10B51BB1084973
:1029BC000848AFF300800848036803B910BD074B03
:1029CC00002BFBD0BDE81040184700BF00000000F2
:1029DC00D4600020F47E0100C0360020000000000E
:1029EC00624B2DE9F74F5B78002613F0020F604B1A
:1029FC0032461B6814BF102708271C1F03F17C01EB
:102A0C00C7F5807514F8043F7600D02B10D0AB427C
:102A1C00C8BFA3F58073834208DA3B44984205DCB7
:102A2C00013246F00106D2B2042A01D0A142E9D10A
:102A3C00504B4FF40072043CC7F100091B68C7F5FA
:102A4C00807E4FF4803A0093A7F1080342FA03F812
:102A5C00431E0193002E00F08580F5077FD5E179A8
:102A6C00637911F0800F18BF203B4B4577DD11F0D7
:102A7C000F02104673D025793F49754594F806B07E
:102A8C00D1F800C04FEACB0BC8BFA5F580750199F2
:102A9C00082F009A18BF0BF4FC6B4D1B002B374909
:102AAC005D441A44095C0CEB050B04DA5B424AFAF0
:102ABC0003F3013B10E07345C9BF6FF480704FF610
:102ACC00FF731B18DB19C1BF08FA03F303F1FF33C3
:102ADC0083F47F4383F0FF031CF80550082F4FEA63
:102AEC00052514BF9BF810C04FF0000C4CEA0505EF
:102AFC001D4015F47F4F17D0280448BF11706B048C
:102B0C0048BF5170A80448BF9170EB0448BFD17006
:102B1C00280548BF11716B0548BF5171A80548BF06
:102B2C009171EB0548BFD17115F0FF0F17D0280636
:102B3C0048BF11726B0648BF5172A80648BF91720C
:102B4C00EB0648BFD172280748BF11736B0748BF0B
:102B5C005173A80748BF9173EB0748BFD173760830
:102B6C00043C77E703B0BDE8F08F00BFA4730020EE
:102B7C0058730020C4650020AC730020FF67002050
:102B8C00244BF0B51C68244B244E1B780BB1F25C23
:102B9C0000E01A463270224A5278520608D41F4975
:102BAC0020464FF48072C95CBDE8F04014F032BF8F
:102BBC001C4BC208C0F3820704F58475196804F134
:102BCC000803DFF864E001EB4212013ADEF8001072
:102BDC00083312F8014F394411F834100C0901F084
:102BEC000F01345D715C03F80D4C03F80E4C03F8C7
:102BFC000F4C03F8104C03F8091C03F80A1C03F8DB
:102C0C000B1C03F80C1C9D42E0D1BDE8F040FFF713
:102C1C00E7BE00BFC465002071730020FF67002071
:102C2C00A47300206C730020B87300203D4B2DE979
:102C3C00F0471E683C4B3D4F1B780BB1FA5C00E033
:102C4C001A463A703A4A5278520608D437493046F6
:102C5C004FF48072C95CBDE8F04714F0DBBE354B15
:102C6C00C5084FEA401E00F00709D3F80080324B2C
:102C7C000EF4C05ED3F800C0304B1A6806F108039E
:102C8C0006F5847602EB4515013D15F8012F083346
:102C9C0009EBC20272441CF8021018F802400A092F
:102CAC0001F00F0114F0800FBA5C795C14BF9246EE
:102CBC008A4614F0400F03F810AC14BF92468A46B3
:102CCC0014F0200F03F80FAC14BF92468A4614F090
:102CDC00100F03F80EAC14BF92468A4614F0080F7E
:102CEC0003F80DAC14BF92468A4614F0040F03F897
:102CFC000CAC14BF92468A4614F0020F03F80BACCE
:102D0C0014BF92468A4614F0010F08BF0A4603F816
:102D1C000AAC03F8092C9E42B7D1BDE8F047FFF787
:102D2C005FBE00BFC465002071730020FF670020E8
:102D3C00A4730020B87300205C7300206C73002017
:102D4C003B4B2DE9F0431E683A4B3B4F1B780BB1C4
:102D5C00FA5C00E01A463A70384A5278520608D4A7
:102D6C00354930464FF48072C95CBDE8F04314F02D
:102D7C0051BE334BC50800F0070CDFF8C8801A6849
:102D8C0006F10803DFF8C0E006F5847602EB451582
:102D9C00013D15F8014F0833D8F80020E1080CEB81
:102DAC00C404515CDEF80020145D0A0901F00F0127
:102DBC00BA5C14F0800F795C14BF9146894614F00C
:102DCC00400F03F8109C14BF9146894614F0200F55
:102DDC0003F80F9C14BF9146894614F0100F03F8AA
:102DEC000E9C14BF9146894614F0080F03F80D9CF5
:102DFC0014BF9146894614F0040F03F80C9C14BFC1
:102E0C009146894614F0020F03F80B9C14BF9146AF
:102E1C00894614F0010F08BF0A4603F80A9C03F810
:102E2C00092C9E42B5D1BDE8F043FFF7D9BD00BFD8
:102E3C00C465002071730020FF670020A47300207C
:102E4C006C7300205C730020B87300202F4B304A49
:102E5C00F0B51C682F4B1B780BB1D15C00E0194608
:102E6C0011702D49497811F0400FD15C06D12046E4
:102E7C004FF48072BDE8F04014F0CCBD274BC6086F
:102E8C00234A28271B7800F00700DFF898E0D25C73
:102E9C00234B1D68A31D07FB065504F1F606013DE7
:102EAC00DEF80040063315F8017F044414F837406F
:102EBC0014F0800F14BF17460F4614F0400F03F8A0
:102ECC000C7C14BF17460F4614F0200F03F80B7C34
:102EDC0014BF17460F4614F0100F03F80A7C14BFEA
:102EEC0017460F4614F0080F03F8097C14BF174659
:102EFC000F4614F0040F03F8087C14BF14460C465C
:102F0C0003F8074C9E42CBD1F0BD00BFC465002036
:102F1C00FF67002071730020A47300202073002031
:102F2C006C730020B873002013460A4619460AF049
:102F3C00EDBC0000A1F1C0031F2B044B96BF01F0A8
:102F4C001F0101F07F017F31196070472867002055
:102F5C000022014B1A6070472867002008B509F061
:102F6C00BFFD034B186009F09BFF024B186008BDB6
:102F7C00246700202067002070B5144D0024144EE7
:102F8C00A4552346013415F8010C2978033515F89E
:102F9C00022C0AF019FC102CF2D10E4C236823B928
:102FAC004FF4804009F060FD20600B4C236823B97E
:102FBC004FF4404009F058FD2060084C236823B9B9
:102FCC004FF4807009F050FD206070BD1731002067
:102FDC00FF670020C0650020EC600020C465002065
:102FEC00F8B5454B07461A780AB901221A704349BD
:102FFC00434B444C1A680B68434D444E286893FB72
:10300C00F2F3FF2BDCBF13020B60FF21404BDA61A4
:10301C00227802F0040283F82B20002283F82A2065
:10302C004FF4404214F0F6FC4FF48042FF2130681C
:10303C0014F0F0FC237813B1364809F005FD4FF479
:10304C000052296834480AF0B3F9237813B1334895
:10305C0009F0FAFC237813B1384609F0F5FC29681D
:10306C004FF40042384601F580410AF0A1F923786B
:10307C0013B12B4809F0E8FC237813B1294809F067
:10308C00E3FC0AF027FC2849284A01250B6828484C
:10309C0013604B68274953609F22274B1D70274BA9
:1030AC001A700023264A1370264A1370264A13708E
:1030BC00264A137032680A6025490A6025490A605D
:1030CC0025490A6025490A60254A264913704FF69E
:1030DC00FF72254B5A801A8000F0BCFB294614481D
:1030EC0000F0CAFB0A4806F037FE237813B11F48DC
:1030FC0009F0AAFC0120F8BD463100201030002058
:10310C003C2F002047310020EC600020C0650020DF
:10311C0024730020182900203F2900205129002069
:10312C00602900206E29002004280020A4730020B0
:10313C0074730020B8730020B473002060730020F7
:10314C0071730020207300207073002066730020C0
:10315C005C7300206C730020AC730020587300204B
:10316C00B07300202908000062730020952900200C
:10317C0010B5044C204606F051FE2046BDE8104028
:10318C0006F04CBE24730020234B24491A682448B3
:10319C000968C2F30E030068002818BF014623B16A
:1031AC00013B63F00F039BB201E04FF6FF73303924
:1031BC00492906D81B48415619B14B1E63F00F0321
:1031CC009BB2D00644BF23F480439BB2910644BF0C
:1031DC0023F040039BB2500642BF4FF6F0711940EA
:1031EC0041F00203110744BF23F480639BB25007E4
:1031FC0044BF23F480739BB2D10744BF23F4006314
:10320C009BB29207084A44BF23F400739BB213800D
:10321C004FF6FF735380704724670020206700200F
:10322C0028670020AA21002062730020A0F5C0436B
:10323C00B3F5005F1CD20F4BC0F309001B68184498
:10324C0000F57053197000F56053197000F5505368
:10325C00197000F54053197000F53053197000F5D2
:10326C002053197000F5105300F5005019700170BF
:10327C00704700BFEC600020054BB0F5C04F1B68D9
:10328C0023BFC018A0F580400078185C704700BFC1
:10329C00EC6000207047000000F0E003A02B19D078
:1032AC00E02B2ED1184BC0F340001A78174B1AB1F3
:1032BC0033F81000000A08E033F81030144903F01A
:1032CC000F0203F0F003885C184300F04F0040F04D
:1032DC0030007047C30709D50E4A137898B203F033
:1032EC005F03137001220C4B1A7008E00B4A0C4957
:1032FC0013880968C85C0133C3F30D031380C0B293
:10330C007047FF20704700BFB0730020627300202D
:10331C00F426002060730020B4730020B2730020E8
:10332C00C065002000F0E0020B46A02AF0B412D0D9
:10333C0004D8802A40F0E280002209E0C02A06D09E
:10334C00E02A40F0DB806E48F0BC00F0BDBA0122F0
:10335C006C4B1A70D2E010F0010F6B4A00F0C28077
:10336C00117821B16948013903701170C6E001214F
:10337C00117003F0C002402A00F0AC80802A07D004
:10338C00002A40F0BB806149614A09781170A7E0BE
:10339C0003F007015D4B481E1A785E4B062805D8D2
:1033AC00DFE800F00A4E5C6A78868F005C78C2F326
:1033BC00420004F0180404E01878C0F3420402F050
:1033CC0018002043544C012808D002DC50B90120CD
:1033DC000BE0082804D0102806D003E0022004E0FB
:1033EC00032002E0207800E00020247884426FD093
:1033FC004A4D9F7805EBC005494C2E7924683E4018
:10340C00484F04EB86263E601F79AE793E40464F0E
:10341C0004EBC6263E60DF786E793E40434F04EBEA
:10342C0086163E605E79ED793540414E04EBC5154C
:10343C0035609D7904EBC5243E4D2C60364C46E03E
:10344C0035480478354800EBC400007902EA0004E2
:10345C003348006800EB8420324C30E02E4804786E
:10346C002E4800EBC400407902EA00042C480068A6
:10347C0000EB84102D4C22E027480478274800EB01
:10348C00C400807902EA00042548006800EBC420DF
:10349C00254C14E020480478204800EBC400C07987
:1034AC0002EA00041E48006800EBC410204C06E041
:1034BC001B4802F03F021F4C006800EBC22020604A
:1034CC0006E010091C4C207002F00F001B4C207001
:1034DC005A5413E00D4903F03F03194A097811704F
:1034EC0053700BE012784AB1154A0D4811880068E8
:1034FC00435413880133C3F30D031380F0BC70479E
:10350C0074730020B0730020B4730020FE67002099
:10351C00B2730020A473002070730020402F002091
:10352C00C06500206C730020B87300205C73002011
:10353C0058730020AC73002020730020717300209E
:10354C00687300202DE9F84FB04F0C46C121064698
:10355C003B78AF4D0133DFF8F88293FBF1F201FBBE
:10356C001233D8B2C02B387013D02B786BB9A94B4F
:10357C001A78A94B53F832309847A8483B78C022A8
:10358C004FF4807100680AF049F9D8F80030F36103
:10359C0038E1A34B6FF0BF01D8F800201B6801FB8A
:1035AC000233F361FFF7F0FD9E4A1378013303F009
:1035BC000703032B137017D99B4B1B7843B19B4B01
:1035CC001A8842F040021A805A8842F040025A800F
:1035DC00974B1B7843B1954B1A8842F480421A8062
:1035EC005A8842F480425A800221924800F044F9F1
:1035FC002B78874A13B1013B137005E08E4B1B7877
:10360C00013B13700AF0F0F88C4A137803F05F0357
:10361C0063F07F0313707F4B1B78002B00F0E3806B
:10362C009F2313700022864B1B6813F822105FFA3D
:10363C0082FED02903D00132202AF6D19646814A47
:10364C0008338149527802F0020202F0FF0C12B9E1
:10365C00D1F800907AE0D1F800804FF0000C5FFABE
:10366C008CF6B64540F2BF8013F8052C15075DD0DB
:10367C0001361F46F6B2B64558D017F8012C100784
:10368C0050D017F8041C13F8082C521AD2B2A2F11D
:10369C001001C9B2E02945D913F8071C17F8035CCF
:1036AC004D1BEDB2A5F11001C9B2E0293AD913F8BE
:1036BC00061C0F2A17F8020C4FEAC10188BF5242B0
:1036CC004FEAC00001F4FC6188BFD2B200F4FC6088
:1036DC00414440448CBF89188018F02D04D9894688
:1036EC006D420146EDB24846C2F10F02D2B2013230
:1036FC000A4491F800A091F8109090F800B009EBF2
:10370C000A2990F810A01FFA89F90AEB0B2A49FA3A
:10371C0005F91FFA8AFA19EA0A0F61D10131013051
:10372C009142E6D101360437F6B2A4E70CF1010C54
:10373C00043394E713F8052C110704D001301F460D
:10374C00C0B2864507D10CF1010C04335FFA8CF042
:10375C008645EFD847E017F8012C12073CD017F834
:10376C00041C13F8082C521AD2B2A2F10801C9B2E7
:10377C00F02931D917F8035C13F8071C491BC9B29F
:10378C00A1F10805EDB2F02D26D9072A13F8066C25
:10379C0017F8025C88BF524209EBC60609EBC50557
:1037AC008ABFD2B2AD18B618F82904D9B04649422E
:1037BC002E46C9B24546C2F1070205F1FF38013E5B
:1037CC0055FA82F216F8015F18F801AF0D4115EAAF
:1037DC000A0F05D14245F5D101300437C0B2B0E72C
:1037EC00BF22164B1A7001232360184B1B784BB168
:1037FC00144B4FF6FF705B7813F0200F18BF662048
:10380C00BDE8F88F4FF6FF70BDE8F88F66730020A7
:10381C00FD67002070730020402F0020C46500203D
:10382C0010300020FA670020FB6700206273002034
:10383C00FC67002074730020463100206073002068
:10384C0058730020A4730020AC730020B4730020C4
:10385C003C2F00200023C16243604361836083617D
:10386C00C360C3610361036280F82A3080F8293099
:10387C0080F8283043627047436A2DE9F0410446D2
:10388C0088463BB90023B8F1020F84F82A3017D1CF
:10389C00BDE8F08190F82A30002BF3D0061D0127EB
:1038AC00002594F82A303B4204D0E36A284632695A
:1038BC003168984701357F000436042DF1D1E1E7DA
:1038CC00C4F82480BDE8F08101F0F003B02B2DE9A1
:1038DC00F04104462DD005D8902B2AD0A02B24D013
:1038EC00802B03E0D02B24D002D8C02B30D11CE08D
:1038FC00E02B02D0F02B1CD02AE001F0030190F851
:10390C0028308B426FD0032956D8DFE801F002052E
:10391C00080B44F6206306E042F2107303E041F218
:10392C00883300E0C368236146E084F82910BDE8C1
:10393C00F081A1F19003C9435B1101F00F01DDB2DD
:10394C0004EB830309015A6991424CD0596134E06C
:10395C0094F8296016F0C00F45D0A6F1800501F04F
:10396C003F0106F00F0643F69823C5F3471506EB07
:10397C0001114FF4003604EB8507013196FBF1F68B
:10398C009E42C8BF00267B689E422CD0022D11D1CE
:10399C0094F8280003280DD1636A266133B194F89A
:1039AC002A3043F0080384F82A3003E0E36A3146F6
:1039BC00226A98477E6000E00325636A4BB10123BD
:1039CC0003FA05F594F82A301D4384F82A50BDE813
:1039DC00F08104EB8503E46A28465A69596823464A
:1039EC00BDE8F0411847BDE8F081000010B5044671
:1039FC008089431CA381FFF73FFC034B1A5C236AAD
:103A0C009B1A236202E000BFF4220020FF2801F27F
:103A1C000083DFE810F000010B01160121012C01DD
:103A2C003701420153015E016A01760182018E0168
:103A3C009A01A601B801C401DC01F4010C022402B4
:103A4C003C0254026F0287029802A902BA02CB020E
:103A5C00DC02ED02030314031E03280332033C03B0
:103A6C00460350035F0369037603830390039D03AE
:103A7C00AA03B703CA03D703E503F103FD03090443
:103A8C001504210432043E04480452045C04660408
:103A9C0070047A048A049404A204B004BE04CC0416
:103AAC00DA04E804F80406051405220530053E0581
:103ABC004F055D056D057B0589059705A505B305C6
:103ACC00C105CF05DF05ED05FB0509061706250623
:103ADC003306410651065F066D067B06890697067E
:103AEC00A506B306C306D106DF06ED06FB060907DD
:103AFC00170725073507430751075F076D077B0736
:103B0C0089079707A707B507C307D107DF07ED0795
:103B1C00FB070908190827082C08310836083B0848
:103B2C00400845084F08540859085E08630868089F
:103B3C006D0872087C08810886088B089008950827
:103B4C009A089F08A908AE08B308B808BD08C208AF
:103B5C00C708CC08D608DB08E008E508EA08EF0837
:103B6C00F408F908030908090D09120917091C09B9
:103B7C0021092609300935093A093F09440949093F
:103B8C004E0953095D09620967096C0971097609C7
:103B9C007B0980098A098F09940999099E09A3094F
:103BAC00A809AD09B809BD09C209C709CC09D109D1
:103BBC00D609DB09E609EB09F009F509FA09FF0951
:103BCC00040A090A140A190A1E0A230A280A2D0AC9
:103BDC00320A370A420A470A4C0A510A560A5B0A49
:103BEC00600A650A700A750A7A0A7F0A840A890AC9
:103BFC008E0A930A9E0AA30AA80AAD0AB20AB70A49
:103C0C00BC0AC10ACC0AD10AD60ADB0AE00AE50AC8
:103C1C00EA0AEF0AFA0AE378B549DA0942EA4303F9
:103C2C00DBB2E370CB5C1343237010BDA378B049B7
:103C3C00DA0942EA4303DBB2A370CB5C1343237073
:103C4C0010BD6379AA49DA0942EA4303DBB2637116
:103C5C00CB5C1343237010BD2379A549DA0942EAE2
:103C6C004303DBB22371CB5C1343237010BDE379A8
:103C7C009F49DA0942EA4303DBB2E371CB5C13439D
:103C8C00237010BDA3799A49DA0942EA4303DBB2E7
:103C9C00A371CB5C1343237010BDE088FFF7ECFAE3
:103CAC00C0F3C712924B42EA4001E088C9B25B5C98
:103CBC0013432370BDE81040FFF7B8BA63788C4902
:103CCC00DA0942EA4303DBB26370CB5C1343237023
:103CDC0010BDE17801F00102D30143EA510384499C
:103CEC00E370CB5C1343237010BDA17801F001028B
:103CFC00D30143EA51037E49A370CB5C1343237079
:103D0C0010BD617901F00102D30143EA51037849F6
:103D1C006371CB5C1343237010BD217901F0010258
:103D2C00D30143EA510372492371CB5C13432370D3
:103D3C0010BDE17901F00102D30143EA51036C4952
:103D4C00E371CB5C1343237010BDA17901F0010228
:103D5C00D30143EA51036649A371CB5C134323702F
:103D6C0010BDE088FFF788FA00F00102C0F34701AC
:103D7C005F4BE08841EAC2115B5C13432370BDE8E2
:103D8C001040FFF753BA617801F00102D30143EA06
:103D9C00510357496370CB5C1343237010BDE27819
:103DAC00237812F0800F52494FEA420203F00103CC
:103DBC0007D01A43D2B28B5CE27043F0010323703C
:103DCC0010BD1343DBB2E370CB5C237010BDA27843
:103DDC00237812F0800F46494FEA420203F00103A8
:103DEC0007D01A43D2B28B5CA27043F0010323704C
:103DFC0010BD1343DBB2A370CB5C237010BD627992
:103E0C00237812F0800F3A494FEA420203F0010383
:103E1C0007D01A43D2B28B5C627143F0010323705A
:103E2C0010BD1343DBB26371CB5C237010BD2279E0
:103E3C00237812F0800F2E494FEA420203F001035F
:103E4C0007D01A43D2B28B5C227143F0010323706A
:103E5C0010BD1343DBB22371CB5C237010BDE27930
:103E6C00237812F0800F22494FEA420203F001033B
:103E7C0007D01A43D2B28B5CE27143F0010323707A
:103E8C0010BD1343DBB2E371CB5C237010BDA27980
:103E9C00237812F0800F16494FEA420203F0010317
:103EAC0007D01A43D2B28B5CA27143F0010323708A
:103EBC0010BD1343DBB2A371CB5C237010BDE08843
:103ECC00FFF7DAF9217810F0800F4FEA400001F08B
:103EDC000101074B41EA0001E088C9B25B5C18BFE5
:103EEC0043F001032370BDE81040FFF79FB900BFFA
:103EFC00042700206278237812F0800FB7494FEA2C
:103F0C00420203F0010307D01A43D2B28B5C6270F9
:103F1C0043F00103237010BD1343DBB26370CB5C21
:103F2C00237010BDE378217813F0010F4FEA53038F
:103F3C00AA4A43EAC113DBB2E370D35C18BF43F067
:103F4C000103237010BDA378217813F0010F4FEA01
:103F5C005303A24A43EAC113DBB2A370D35C18BF6C
:103F6C0043F00103237010BD6379217813F0010F26
:103F7C004FEA5303994A43EAC113DBB26371D35C32
:103F8C0018BF43F00103237010BD2379217813F07F
:103F9C00010F4FEA5303914A43EAC113DBB2237179
:103FAC00D35C18BF43F00103237010BDE379217873
:103FBC0013F0010F4FEA5303884A43EAC113DBB2F3
:103FCC00E371D35C18BF43F00103237010BDA379D8
:103FDC00217813F0010F4FEA5303804A43EAC113CF
:103FEC00DBB2A371D35C18BF43F00103237010BD87
:103FFC00E088FFF741F9217810F0010F4FEA5000EB
:10400C00764B40EAC111E088C9B25B5C18BF43F043
:10401C0001032370BDE81040FFF708B963782178DD
:10402C0013F0010F4FEA53036C4A43EAC113DBB29E
:10403C006370D35C18BF43F00103237010BDE278AA
:10404C0066495300DBB2E370CB5C43EAD2132370B6
:10405C0010BDA27861495300DBB2A370CB5C43EA7C
:10406C00D213237010BD62795C495300DBB26371CB
:10407C00CB5C43EAD213237010BD2279574953000D
:10408C00DBB22371CB5C43EAD213237010BDE2790F
:10409C0052495300DBB2E371CB5C43EAD213237079
:1040AC0010BDA2794D495300DBB2A371CB5C43EA3E
:1040BC00D213237010BDE088FFF7DEF8474B4100A8
:1040CC00C9B25B5C43EAD0102070E088BDE81040B8
:1040DC00FFF7ACB8627841495300DBB26370CB5C3C
:1040EC0043EAD213237010BDE3783C4923F07F02DE
:1040FC0042EA530203F00103E2708A5C134323701B
:10410C0010BDA378354923F07F0242EA530203F035
:10411C000103A2708A5C1343237010BD63792F498D
:10412C0023F07F0242EA530203F0010362718A5CBE
:10413C001343237010BD2379284923F07F0242EAF0
:10414C00530203F0010322718A5C1343237010BDE8
:10415C00E379224923F07F0242EA530203F0010380
:10416C00E2718A5C1343237010BDA3791B4923F0C1
:10417C007F0242EA530203F00103A2718A5C1343EB
:10418C00237010BDE088FFF777F820F07F01134B08
:10419C0041EA500100F00100C9B25B5C1843207089
:1041AC00E088BDE81040FFF741B863780B4923F075
:1041BC007F0242EA530203F0010362708A5C1343EC
:1041CC00237010BDE2780549530043F00103DBB2C4
:1041DC00E370CB5C43EAD213237010BD042700209C
:1041EC00A278B349530043F00103DBB2A370CB5C5C
:1041FC0043EAD213237010BD6279AD49530043F0EA
:10420C000103DBB26371CB5C43EAD213237010BDA4
:10421C002279A749530043F00103DBB22371CB5C35
:10422C0043EAD213237010BDE279A149530043F045
:10423C000103DBB2E371CB5C43EAD213237010BDF4
:10424C00A2799B49530043F00103DBB2A371CB5C11
:10425C0043EAD213237010BDE088FFF70DF8944B9E
:10426C00410041F00101C9B25B5C43EAD0102070FF
:10427C00E088BDE81040FEF7D9BF62788C49530046
:10428C0043F00103DBB26370CB5C43EAD2132370BF
:10429C0010BDE37886495A0803F00103E2708A5C8A
:1042AC001343237010BDA37881495A0803F001030E
:1042BC00A2708A5C1343237010BD63797C495A0841
:1042CC0003F0010362718A5C1343237010BD2379E0
:1042DC0077495A0803F0010322718A5C1343237057
:1042EC0010BDE37972495A0803F00103E2718A5C4C
:1042FC001343237010BDA3796D495A0803F00103D1
:10430C00A2718A5C1343237010BDE088FEF7B4FFE2
:10431C00674BC0F3470100F001005B5C1843207051
:10432C00E088BDE81040FEF781BF637860495A0809
:10433C0003F0010362708A5C1343237010BDE278B2
:10434C00237812F0010F23F0520314BF00224022F5
:10435C0043F010031343237010BDA278237812F09E
:10436C00010F23F0520314BF0022402243F010032C
:10437C001343237010BD6279237812F0010F23F0E0
:10438C00520314BF0022402243F010031343237046
:10439C0010BD2279237812F0010F23F0520314BFC1
:1043AC000022402243F010031343237010BDE27926
:1043BC00237812F0010F23F0520314BF0022402285
:1043CC0043F010031343237010BDA279237812F02D
:1043DC00010F23F0520314BF0022402243F01003BC
:1043EC001343237010BDE088FEF746FF237810F0CE
:1043FC00010F23F0520314BF0022402243F010039C
:10440C001343237010BD6278237812F0010F23F050
:10441C00520314BF0022402243F0100313432370B5
:10442C0010BDE278237812F0020F23F0520314BF70
:10443C000022402243F010031343237010BDA278D6
:10444C00237812F0020F23F0520314BF00224022F3
:10445C0043F010031343237010BD6279237812F0DC
:10446C00020F23F0520314BF0022402243F010032A
:10447C001343237010BD2279237812F0020F23F01E
:10448C00520314BF0022402243F010031343237045
:10449C0010BDE279237812F0020F23F0520314BFFF
:1044AC000022402243F010031343237010BD00BFC1
:1044BC0004270020A279237812F0020F23F0520374
:1044CC0014BF0022402243F010031343237010BD8D
:1044DC00E088FEF7D1FE237810F0020F23F0520390
:1044EC0014BF0022402243F010031343237010BD6D
:1044FC006278237812F0020F23F0520314BF0022CB
:10450C00402243F010031343237010BDE27823784C
:10451C0012F0040F23F0520314BF0022402243F088
:10452C0010031343237010BDA278237812F0040FEC
:10453C0023F0520314BF0022402243F01003134314
:10454C00237010BD6279237812F0040F23F052030C
:10455C0014BF0022402243F010031343237010BDFC
:10456C002279237812F0040F23F0520314BF002297
:10457C00402243F010031343237010BDE2792378DB
:10458C0012F0040F23F0520314BF0022402243F018
:10459C0010031343237010BDA279237812F0040F7B
:1045AC0023F0520314BF0022402243F010031343A4
:1045BC00237010BDE088FEF75FFE237810F0040F27
:1045CC0023F0520314BF0022402243F01003134384
:1045DC00237010BD6278237812F0040F23F052037D
:1045EC0014BF0022402243F010031343237010BD6C
:1045FC00E278237812F0080F23F0520314BF002244
:10460C00402243F010031343237010BDA27823788B
:10461C0012F0080F23F0520314BF0022402243F083
:10462C0010031343237010BD6279237812F0080F26
:10463C0023F0520314BF0022402243F01003134313
:10464C00237010BD2279237812F0080F23F0520347
:10465C0014BF0022402243F010031343237010BDFB
:10466C00E279237812F0080F23F0520314BF0022D2
:10467C00402243F010031343237010BDA27923781A
:10468C0012F0080F23F0520314BF0022402243F013
:10469C0010031343237010BDE088FEF7EDFD237863
:1046AC0010F0080F23F0520314BF0022402243F0F5
:1046BC0010031343237010BD6278237812F0080F97
:1046CC0023F0520314BF0022402243F01003134383
:1046DC00237010BDE278237812F0100F23F05203F0
:1046EC0014BF0022402243F010031343237010BD6B
:1046FC00A278237812F0100F23F0520314BF00227B
:10470C00402243F010031343237010BD62792378C9
:10471C0012F0100F23F0520314BF0022402243F07A
:10472C0010031343237010BD2279237812F0100F5D
:10473C0023F0520314BF0022402243F01003134312
:10474C00237010BDE279237812F0100F23F052037E
:10475C0014BF0022402243F010031343237010BDFA
:10476C00A279237812F0100F23F0520314BF002209
:10477C00402243F010031343237010BDE088FEF772
:10478C007BFD237810F0100F23F0520314BF00228E
:10479C00402243F010031343237010BD627823783A
:1047AC0012F0100F23F0520314BF0022402243F0EA
:1047BC0010031343237010BDE278237812F0200FFE
:1047CC0023F0520314BF0022402243F01003134382
:1047DC00237010BDA278237812F0200F23F052031F
:1047EC0014BF0022402243F010031343237010BD6A
:1047FC006279237812F0200F23F0520314BF0022A9
:10480C00402243F010031343237010BD2279237808
:10481C0012F0200F23F0520314BF0022402243F069
:10482C0010031343237010BDE279237812F0200F8C
:10483C0023F0520314BF0022402243F01003134311
:10484C00237010BDA279237812F0200F23F05203AD
:10485C0014BF0022402243F010031343237010BDF9
:10486C00E088FEF709FD237810F0200F23F05203A7
:10487C0014BF0022402243F010031343237010BDD9
:10488C006278237812F0200F23F0520314BF002219
:10489C00402243F010031343237010BDE2782378B9
:1048AC0012F0400F23F0520314BF0022402243F0B9
:1048BC0010031343237010BDA278237812F0400F1D
:1048CC0023F0520314BF0022402243F01003134381
:1048DC00237010BD6279237812F0400F23F052033D
:1048EC0014BF0022402243F010031343237010BD69
:1048FC002279237812F0400F23F0520314BF0022C8
:10490C00402243F010031343237010BDE279237847
:10491C0012F0400F23F0520314BF0022402243F048
:10492C0010031343237010BDA279237812F0400FAB
:10493C0023F0520314BF0022402243F01003134310
:10494C00237010BDE088FEF797FC237810F0400F21
:10495C0023F0520314BF0022402243F010031343F0
:10496C00237010BD6278237812F0400F23F05203AD
:10497C0014BF0022402243F010031343237010BDD8
:10498C0094F903202378002A23F05203B4BF0022A9
:10499C00402243F010031343237010BD94F90220FE
:1049AC002378002A23F05203B4BF0022402243F0A4
:1049BC0010031343237010BD94F905202378002AAB
:1049CC0023F05203B4BF0022402243F010031343E0
:1049DC00237010BD94F904202378002A23F052038D
:1049EC00B4BF0022402243F010031343237010BDC8
:1049FC0094F907202378002A23F05203B4BF002235
:104A0C00402243F010031343237010BD94F9062089
:104A1C002378002A23F05203B4BF0022402243F033
:104A2C0010031343237010BDE088FEF725FC237898
:104A3C0010F0800F23F0520314BF0022402243F0E9
:104A4C0010031343237010BD94F901202378002A1E
:104A5C0023F05203B4BF0022402243F0100313434F
:104A6C00237010BDE37823F00103E37010BDA3782D
:104A7C0023F00103A37010BD637923F0010363716C
:104A8C0010BD237923F00103237110BDE37923F0CA
:104A9C000103E37110BDA37923F00103A37110BDD1
:104AAC00E088FEF7E9FB00F0FE01E088BDE810406D
:104ABC00FEF7BCBB637823F00103637010BDE37891
:104ACC0023F00203E37010BDA37823F00203A3705C
:104ADC0010BD637923F00203637110BD237923F0B9
:104AEC000203237110BDE37923F00203E37110BDBF
:104AFC00A37923F00203A37110BDE088FEF7BCFB81
:104B0C0000F0FD01E088BDE81040FEF78FBB637834
:104B1C0023F00203637010BDE37823F00403E37009
:104B2C0010BDA37823F00403A37010BD637923F0A8
:104B3C000403637110BD237923F00403237110BDAA
:104B4C00E37923F00403E37110BDA37923F004038C
:104B5C00A37110BDE088FEF78FFB00F0FB01E0882D
:104B6C00BDE81040FEF762BB637823F0040363706A
:104B7C0010BDE37823F00803E37010BDA37823F095
:104B8C000803A37010BD637923F00803637110BD93
:104B9C00237923F00803237110BDE37923F0080374
:104BAC00E37110BDA37923F00803A37110BDE08855
:104BBC00FEF762FB00F0F701E088BDE81040FEF75D
:104BCC0035BB637823F00803637010BDE37823F0E2
:104BDC001003E37010BDA37823F01003A37010BD75
:104BEC00637923F01003637110BD237923F0100354
:104BFC00237110BDE37923F01003E37110BDA37989
:104C0C0023F01003A37110BDE088FEF735FB00F014
:104C1C00EF01E088BDE81040FEF708BB637823F095
:104C2C001003637010BDE37823F02003E37010BD14
:104C3C00A37823F02003A37010BD637923F0200325
:104C4C00637110BD237923F02003237110BDE37928
:104C5C0023F02003E37110BDA37923F02003A3718B
:104C6C0010BDE088FEF708FB00F0DF01E088BDE82E
:104C7C001040FEF7DBBA637823F02003637010BD9D
:104C8C00E37823F04003E37010BDA37823F04003D6
:104C9C00A37010BD637923F04003637110BD2379B9
:104CAC0023F04003237110BDE37923F04003E3713B
:104CBC0010BDA37923F04003A37110BDE088FEF76B
:104CCC00DBFA00F0BF01E088BDE81040FEF7AEBA99
:104CDC00637823F04003637010BDE37803F07F0327
:104CEC00E37010BDA37803F07F03A37010BD63794C
:104CFC0003F07F03637110BD237903F07F032371ED
:104D0C0010BDE37903F07F03E37110BDA37903F0C9
:104D1C007F03A37110BDE088FEF7AEFA00F07F01AF
:104D2C00E088BDE81040FEF781BA637803F07F039A
:104D3C00637010BDE37843F00103E37010BDA378FA
:104D4C0043F00103A37010BD637943F00103637159
:104D5C0010BD237943F00103237110BDE37943F0B7
:104D6C000103E37110BDA37943F00103A37110BDDE
:104D7C00E088FEF781FA40F00101E088C9B2BDE895
:104D8C001040FEF753BA637843F00103637010BD13
:104D9C00E37843F00203E37010BDA37843F0020301
:104DAC00A37010BD637943F00203637110BD2379C6
:104DBC0043F00203237110BDE37943F00203E37166
:104DCC0010BDA37943F00203A37110BDE088FEF778
:104DDC0053FA40F00201E088C9B2BDE81040FEF77A
:104DEC0025BA637843F00203637010BDE37843F097
:104DFC000403E37010BDA37843F00403A37010BD4B
:104E0C00637943F00403637110BD237943F0040309
:104E1C00237110BDE37943F00403E37110BDA37952
:104E2C0043F00403A37110BDE088FEF725FA40F0AF
:104E3C000401E088C9B2BDE81040FEF7F7B9637809
:104E4C0043F00403637010BDE37843F00803E37090
:104E5C0010BDA37843F00803A37010BD637943F031
:104E6C000803637110BD237943F00803237110BD4F
:104E7C00E37943F00803E37110BDA37943F0080311
:104E8C00A37110BDE088FEF7F7F940F00801E08847
:104E9C00C9B2BDE81040FEF7C9B9637843F0080306
:104EAC00637010BDE37843F01003E37010BDA3787A
:104EBC0043F01003A37010BD637943F010036371CA
:104ECC0010BD237943F01003237110BDE37943F037
:104EDC001003E37110BDA37943F01003A37110BD4F
:104EEC00E088FEF7C9F940F01001E088C9B2BDE8CE
:104EFC001040FEF79BB9637843F01003637010BD4C
:104F0C00E37843F02003E37010BDA37843F0200353
:104F1C00A37010BD637943F02003637110BD237936
:104F2C0043F02003237110BDE37943F02003E371B8
:104F3C0010BDA37943F02003A37110BDE088FEF7E8
:104F4C009BF940F02001E088C9B2BDE81040FEF7A3
:104F5C006DB9637843F02003637010BDE37843F0C0
:104F6C004003E37010BDA37843F04003A37010BD61
:104F7C00637943F04003637110BD237943F0400320
:104F8C00237110BDE37943F04003E37110BDA379A5
:104F9C0043F04003A37110BDE088FEF76DF940F0BB
:104FAC004001E088C9B2BDE81040FEF73FB9637814
:104FBC0043F04003637010BDE37863F07F03E3704C
:104FCC0010BDA37863F07F03A37010BD637963F009
:104FDC007F03637110BD237963F07F03237110BDD0
:104FEC00E37963F07F03E37110BDA37963F07F0372
:104FFC00A37110BDE088FEF73FF960F07F01E088F7
:10500C00C9B2BDE81040FEF711B9637863F07F03B5
:10501C00637010BD70B504468089431CA381FEF7F4
:10502C002BF9034B1A5C0138236A9B1A236201E0AB
:10503C00F4240020FE2802F2FA80DFE810F00608C3
:10504C00670DB108B109C108CE0D970A820C4A0848
:10505C004008A108CB09DC08D50DB00AD10B130808
:10506C006D0DB508E509F708DC0DA20AF30B610814
:10507C004508A508FF091509E30DC00AFF00200823
:10508C00130EB908190A3009EA0D8F0E07017808BA
:10509C002F0EA908330A4B09F10D300C14012D0801
:1050AC005F0EBD08690A8109FF0D290C18018A08D9
:1050BC004A0EAD084D0A6609F80D630CF810A70CE2
:1050CC00C70CE70C070D270D730D470D870CF81057
:1050DC00CA0CEA0C0A0D2A0D800D4A0D8A0CAA0C7A
:1050EC00F810ED0C0D0D2D0D8D0D4D0D8D0CAD0C19
:1050FC00CD0CF810100D300D9A0D500D900CB00C0D
:10510C00D00CF00CF810330DA70D530D930CB30C01
:10511C00D30CF30C130DF810B40D560D990CB90CEF
:10512C00D90CF90C190D390DEF10590D960CB60C54
:10513C00D60CF60C160D360DC10DF810CA01E50192
:10514C0000021B023602510280026C027A049D049A
:10515C00BC04DB04FA04190552053805C802E40244
:10516C0000031C033B03570378037303A205C2051A
:10517C00E20502062506450677066506C003CA0346
:10518C00D403DE03E803F2030304FC03C706CF06D3
:10519C00D706DF06E706EF06FC06F70625042D0406
:1051AC0035043D0445044D045A0455041C073607C8
:1051BC0050076A078407A307C007BD0752019A0B63
:1051CC001C01E30B85015A0BA702D20A71011C0CBE
:1051DC004001A80EB601FC0B7D05E30A6401A70B88
:1051EC003801380C89016A0B9F03F40A7501700CA5
:1051FC004401430CBA01A40EA206050B6801B40BC2
:10520C003C01750EAD017A0B1704160B79013A08A7
:10521C0048017D0CBE01F8100F07270B6C01C10B68
:10522C0024014D0CB1018A0B6D04380B7F013D0834
:10523C004D01520CC401A40EE607490B237813F060
:10524C00400F07D0A3890133A38170BD237813F0DD
:10525C00400FF7D0A089FEF70FF8A38940B20130B8
:10526C001844A08170BD237813F0010FE9E723786F
:10527C0013F0010FEDE7237813F0400F07D0A3894B
:10528C000233A38170BD94F90030002BF7DBA089A9
:10529C004FF00005431CA381FDF7EEFF60F30705FB
:1052AC00A089FDF7E9FF60F30F25A58170BD237878
:1052BC0013F0010FE2E7237813F0040FDEE72378F5
:1052CC0013F0400F06E0237813F0010F02E023786F
:1052DC0013F0040FD3D0DAE794F90030002BCEDAB8
:1052EC00D5E7237813F0400F41F0A187E089431CE8
:1052FC00E381FDF7C1FF2073E089431CE381FDF7D7
:10530C00BBFF607370BD237813F0010FECE72378BB
:10531C0013F0040FE8E794F90030002BE6DA70BDC7
:10532C00237813F0400F06E0237813F0010F02E00E
:10533C00237813F0040F01F07A87D7E794F9003043
:10534C00002B81F27487D1E7237813F0400F02E031
:10535C00237813F0010F92D1A0894FF00005431C64
:10536C00A381FDF789FF60F30705A089431CA38186
:10537C00FDF782FF60F30F25E089617B013880B275
:10538C00E081FDF753FFE089217B013880B2E08199
:10539C00FDF74CFFA58170BD237813F0040FDAE7FD
:1053AC0094F90030002BD7DA69E7237813F0400F1B
:1053BC0006E0237813F0010F02E0237813F0040FBA
:1053CC003FF45DAFC8E794F90030002BBFF657AF40
:1053DC00C2E76378E27899185340C8B2C1F3072149
:1053EC004240607022F07F029A43B14A125C14BFB3
:1053FC0004250025114383EA000202F0100241EA61
:10540C0002032B43237070BD6378A2789918534024
:10541C00C8B2C1F307214240607022F07F029A4368
:10542C00A34A125C14BF04250025114383EA000231
:10543C0002F0100241EA02032B43237070BD637823
:10544C00627999185340C8B2C1F307214240607089
:10545C0022F07F029A43964A125C14BF0425002561
:10546C00114383EA000202F0100241EA02032B43CB
:10547C00237070BD6378227999185340C8B2C1F378
:10548C0007214240607022F07F029A43884A125CE6
:10549C0014BF04250025114383EA000202F0100218
:1054AC0041EA02032B43237070BD6378E27A9918AA
:1054BC005340C8B2C1F307214240607022F07F0212
:1054CC009A437B4A125C14BF04250025114383EADE
:1054DC00000202F0100241EA02032B43237070BD5C
:1054EC006378A27A99185340C8B2C1F3072142409D
:1054FC00607022F07F029A436D4A125C14BF04253F
:10550C000025114383EA000202F0100241EA020373
:10551C002B43237070BD62785300D9B24A4061703E
:10552C0012F0800F01F0100242EA1323604A14BFFC
:10553C0004200020525C13430343237070BDA089E8
:10554C006589431CA381FDF797FE45FA80F080B274
:10555C00FDF792FE637856491A184340D5B2C2F350
:10556C000722DBB26840495D657020EA03001143F5
:10557C0083EA050210F0800F02F0100214BF042021
:10558C00002041EA02030343237070BDA089431C31
:10559C00A381FDF771FE637845491A184340D5B2D3
:1055AC00C2F30722DBB26840495D657020EA030054
:1055BC00114383EA050210F0800F02F0100214BFB1
:1055CC000420002041EA02030343237070BD62787B
:1055DC00E378D11A5340C8B2C1F307214240494283
:1055EC0060701A4012F0800F314A125C14BF06250D
:1055FC000225114383EA000202F0100241EA020381
:10560C002B43237070BD6278A378D11A5340C8B273
:10561C00C1F307214240494260701A4012F0800FDA
:10562C00234A125C14BF06250225114383EA0002AB
:10563C0002F0100241EA02032B43237070BD627822
:10564C006379D11A5340C8B2C1F307214240494291
:10565C0060701A4012F0800F154A125C14BF0625B8
:10566C000225114383EA000202F0100241EA020310
:10567C002B43237070BD62782379D11A5340C8B282
:10568C00C1F307214240494260701A4012F0800F6A
:10569C00074A125C14BF06250225114383EA000257
:1056AC0002F0100241EA02032B43237070BD00BFCD
:1056BC000C2800206278E37AD11A5340C8B2C1F3A7
:1056CC0007214240494260701A4012F0800FA84AEC
:1056DC00125C14BF06250225114383EA000202F076
:1056EC00100241EA02032B43237070BD6278A37A47
:1056FC00D11A5340C8B2C1F30721424049426070ED
:10570C001A4012F0800F9A4A125C14BF062502252B
:10571C00114383EA000202F0100241EA02032B4318
:10572C00237070BD002363704223237070BDA08969
:10573C006589431CA381FDF79FFD45FA80F080B27B
:10574C00FDF79AFD63781A1A5840D1B2C2F30722BA
:10575C00C0B24B4052426170034013F0800F844B37
:10576C005B5C14BF062502251A4380EA010303F093
:10577C00100342EA03002843207070BDA089431C2B
:10578C00A381FDF779FD63781A1A5840D1B2C2F3A0
:10579C000722C0B24B4052426170034013F0800F9D
:1057AC00734B5B5C14BF062502251A4380EA010388
:1057BC0003F0100342EA03002843207070BD6278A6
:1057CC00E37813406B4A6370D35C43F0100323708F
:1057DC0070BD6278A3781340664A6370D35C43F063
:1057EC001003237070BD627863791340614A637053
:1057FC00D35C43F01003237070BD6278237913409F
:10580C005C4A6370D35C43F01003237070BD627804
:10581C00E37A1340574A6370D35C43F01003237050
:10582C0070BD6278A37A1340524A6370D35C43F024
:10583C001003237070BD63784E4AD35C43F01003A1
:10584C00237070BDA0896589431CA381FDF714FDED
:10585C0045FA80F080B2FDF70FFD63781840454B98
:10586C001B5C607043F01003237070BDA089431C57
:10587C00A381FDF701FD637818403E4B1B5C607003
:10588C0043F01003237070BD6278E3781343394AF8
:10589C006370D35C237070BD6278A3781343354A70
:1058AC006370D35C237070BD627863791343314AA3
:1058BC006370D35C237070BD6278237913432D4AD7
:1058CC006370D35C237070BD6278E37A1343294A0A
:1058DC006370D35C237070BD6278A37A1343254A3E
:1058EC006370D35C237070BD6378224AD35C2370E1
:1058FC0070BDA0896589431CA381FDF7BDFC45FAE9
:10590C0080F080B2FDF7B8FC63781843194BC0B235
:10591C001B5C6070237070BDA089431CA381FDF7D4
:10592C00ABFC63781843134BC0B21B5C60702370E4
:10593C0070BD6378E178227802F001005A184B4070
:10594C000244D0B2C2F307224140607021F07F01C3
:10595C0099430749095C14BF04250025114383EAC8
:10596C00000202F0100241EA02032B43237070BDC7
:10597C000C280020042700206378A178227802F0FC
:10598C0001005A184B400244D0B2C2F307224140E6
:10599C00607021F07F019943BA49095C14BF04255A
:1059AC000025114383EA000202F0100241EA0203CF
:1059BC002B43237070BD63786179227802F001006B
:1059CC005A184B400244D0B2C2F3072241406070D7
:1059DC0021F07F019943AB49095C14BF04250025D4
:1059EC00114383EA000202F0100241EA02032B4346
:1059FC00237070BD63782179227802F001005A1867
:105A0C004B400244D0B2C2F307224140607021F0F7
:105A1C007F0199439B49095C14BF04250025114360
:105A2C0083EA000202F0100241EA02032B432370C6
:105A3C0070BD6378E17A227802F001005A184B406D
:105A4C000244D0B2C2F307224140607021F07F01C2
:105A5C0099438C49095C14BF04250025114383EA42
:105A6C00000202F0100241EA02032B43237070BDC6
:105A7C006378A17A227802F001005A184B40024454
:105A8C00D0B2C2F307224140607021F07F019943EC
:105A9C007C49095C14BF04250025114383EA0002EC
:105AAC0002F0100241EA02032B43237070BD2378ED
:105ABC00627803F0010303EB4203D9B2C3F307236B
:105ACC004A40617012F0800F01F0100243EA0203A9
:105ADC006C4A14BF04200020525C13430343237010
:105AEC0070BDA0896589431CA381FDF7C5FB45FAF0
:105AFC0080F080B2FDF7C0FB2278637802F00102DF
:105B0C0060491A4443400244DBB2D5B2C2F30722C7
:105B1C006840495D657020EA0300114383EA050281
:105B2C0010F0800F02F0100214BF0420002041EA94
:105B3C0002030343237070BDA089431CA381FDF7AE
:105B4C009BFB2278637802F001024E491A444340D1
:105B5C000244DBB2D5B2C2F307226840495D6570DE
:105B6C0020EA0300114383EA050210F0800F02F0D3
:105B7C00100214BF0420002041EA020303432370E7
:105B8C0070BD6078E3782278C11A434002F00102BC
:105B9C008A1AD1B2C2F307224840524261701840AF
:105BAC0010F0800F3748405C14BF062502251043C7
:105BBC0083EA010202F0100240EA02032B43237035
:105BCC0070BD6078A3782278C11A434002F00102BC
:105BDC008A1AD1B2C2F3072248405242617018406F
:105BEC0010F0800F2748405C14BF06250225104397
:105BFC0083EA010202F0100240EA02032B432370F5
:105C0C0070BD607863792278C11A434002F00102BA
:105C1C008A1AD1B2C2F3072248405242617018402E
:105C2C0010F0800F1748405C14BF06250225104366
:105C3C0083EA010202F0100240EA02032B432370B4
:105C4C0070BD607823792278C11A434002F00102BA
:105C5C008A1AD1B2C2F307224840524261701840EE
:105C6C0010F0800F0748405C14BF06250225104336
:105C7C0083EA010202F0100240EA02032B43237074
:105C8C0070BD00BF0C2800206078E37A2278C11A1E
:105C9C00434002F001028A1AD1B2C2F307224840F3
:105CAC0052426170184010F0800FB448405C14BF31
:105CBC0006250225104383EA010202F0100240EA95
:105CCC0002032B43237070BD6078A37A2278C11A2B
:105CDC00434002F001028A1AD1B2C2F307224840B3
:105CEC0052426170184010F0800FA448405C14BF01
:105CFC0006250225104383EA010202F0100240EA55
:105D0C0002032B43237070BD237843F30003D9B2F5
:105D1C00C3F3072301F010025B4261701343974AEF
:105D2C0043F00203525C1343237070BDA089658954
:105D3C00431CA381FDF7A0FA45FA80F080B2FDF771
:105D4C009BFA617823780A1A484003F00103C0B229
:105D5C00D31ADAB2C3F3072351405B42627001409D
:105D6C0011F0800F8549895C14BF06250225194363
:105D7C0080EA020303F0100341EA03002843207079
:105D8C0070BDA089431CA381FDF776FA6178237856
:105D9C000A1A484003F00103C0B2D31ADAB2C3F3B3
:105DAC00072351405B426270014011F0800F734930
:105DBC00895C14BF06250225194380EA020303F00F
:105DCC00100341EA03002843207070BD6278E37829
:105DDC0053406B4A6370D35C237070BD6278A378B8
:105DEC005340674A6370D35C237070BD62786379EB
:105DFC005340634A6370D35C237070BD627823791F
:105E0C0053405F4A6370D35C237070BD6278E37A51
:105E1C0053405B4A6370D35C237070BD6278A37A85
:105E2C005340574A6370D35C237070BD002363707A
:105E3C004423237070BDA0896589431CA381FDF7A1
:105E4C001BFA45FA80F080B2FDF716FA63785840D9
:105E5C004B4BC0B21B5C6070237070BDA089431C9F
:105E6C00A381FDF709FA63785840454BC0B21B5C1F
:105E7C006070237070BD6178E278881A4A40C3B2B2
:105E8C00C0F307205940404211405A4011F0800F96
:105E9C003A4902F01002C95C14BF062502250843DA
:105EAC0040EA02032B43237070BD6178A278881AF4
:105EBC004A40C3B2C0F307205940404211405A40F7
:105ECC0011F0800F2D4902F01002C95C14BF062599
:105EDC000225084340EA02032B43237070BD61780E
:105EEC006279881A4A40C3B2C0F307205940404235
:105EFC0011405A4011F0800F204902F01002C95C89
:105F0C0014BF06250225084340EA02032B432370E5
:105F1C0070BD61782279881A4A40C3B2C0F3072059
:105F2C005940404211405A4011F0800F134902F081
:105F3C001002C95C14BF06250225084340EA02037F
:105F4C002B43237070BD6178E27A881A4A40C3B241
:105F5C00C0F307205940404211405A4011F0800FC5
:105F6C00064902F01002C95C14BF0625022508433D
:105F7C0040EA02032B43237070BD00BF0C280020A5
:105F8C00042700206178A27A881A4A40C3B2C0F371
:105F9C0007205940404211405A4011F0800FB1493E
:105FAC0002F01002C95C14BF06250225084340EA22
:105FBC0002032B43237070BD4223237070BDA08954
:105FCC006589431CA381FDF757F945FA80F080B22F
:105FDC00FDF752F961780D1A80EA0102EBB2C5F3B4
:105FEC000725D2B259406D4211405A4011F0800F32
:105FFC009C4902F01002C95C14BF062002200D431C
:10600C0045EA02030343237070BDA089431CA3819E
:10601C00FDF732F961780D1A80EA0102EBB2C5F393
:10602C000725D2B259406D4211405A4011F0800FF1
:10603C008C4902F01002C95C14BF062002200D43EB
:10604C0045EA02030343237070BDA089431CA3815E
:10605C00FDF712F9A070A089431CA381FDF70CF980
:10606C00E07070BDA089431CA381FDF705F9207178
:10607C00A089431CA381FDF7FFF8607170BDA08956
:10608C00431CA381FDF7F8F8A072A089431CA381DF
:10609C00FDF7F2F8E07270BDA089431CA381FDF7F7
:1060AC00EBF8A073A089431CA381FDF7E5F8E0731E
:1060BC0070BD6389A38170BD6389E38170BD608805
:1060CC00FDF7DAF8607070BDA088FDF7D5F8607048
:1060DC0070BD6589628894F90010AB186A4021F094
:1060EC00130198B24240608112F4805FC3F3004206
:1060FC0014BF1025002541EA02032B43237070BD09
:10610C006589A28894F90010AB186A4021F013013C
:10611C0098B24240608112F4805FC3F3004214BF16
:10612C001025002541EA02032B43237070BD6389BF
:10613C0094F900205B0022F0130299B242EA134357
:10614C0011F4805F618114BF102000200343237081
:10615C0070BD6589E28994F90010AB186A4021F092
:10616C00130198B24240608112F4805FC3F3004285
:10617C0014BF1025002541EA02032B43237070BD88
:10618C006388013B638070BDA388013BA38070BD15
:10619C006389013B638170BDE389013BE38170BD81
:1061AC0063880133638070BDA3880133A38070BD05
:1061BC0063890133638170BDE3890133E38170BD71
:1061CC00E17822780139274B02F00102C9B242F082
:1061DC000202585C7F29E17001F00F010CBF04230F
:1061EC00002302430F2943EA02030CBF10210021B4
:1061FC000B43237070BDA17822780139194B02F042
:10620C000102C9B242F00202585C7F29A17001F070
:10621C000F010CBF0423002302430F2943EA02039E
:10622C000CBF102100210B43237070BD61792278C3
:10623C0001390C4B02F00102C9B242F00202585C67
:10624C007F29617101F00F010CBF0423002302436D
:10625C000F2943EA02030CBF102100210B432370CA
:10626C0070BD00BF0C280020217922780139A74B82
:10627C0002F00102C9B242F00202585C7F2921717E
:10628C0001F00F010CBF0423002302430F2943EA42
:10629C0002030CBF102100210B43237070BDE17A67
:1062AC0022780139994B02F00102C9B242F0020284
:1062BC00585C7F29E17201F00F010CBF042300230D
:1062CC0002430F2943EA02030CBF102100210B43A8
:1062DC00237070BDA17A227801398C4B02F0010237
:1062EC00C9B242F00202585C7F29A17201F00F0181
:1062FC000CBF0423002302430F2943EA02030CBF03
:10630C00102100210B43237070BD61782278013974
:10631C007E4B02F00102C9B242F00202585C7F29A6
:10632C00617001F00F010CBF0423002302430F29FD
:10633C0043EA02030CBF102100210B43237070BDF4
:10634C006589A089FCF798FF45FA80F080B2FCF7CC
:10635C0093FF227801386D4B02F001026689C5B2B9
:10636C00A08942F00202595D7F2D42EA010205F03C
:10637C000F010CBF042300230F2943EA02030CBFB7
:10638C00102100210B432370431CA381FCF774FFE5
:10639C0046FA80F0294680B2BDE87040FCF746BF53
:1063AC00E17823780131594A03F00103C9B2525CF8
:1063BC008029E17043EA02030CBF0422002211F091
:1063CC000F0F5BB243EA020314BF002210221343E7
:1063DC00237070BDA178237801314C4A03F001037E
:1063EC00C9B2525C8029A17043EA02030CBF04229B
:1063FC00002211F00F0F5BB243EA020314BF00221C
:10640C0010221343237070BD6179237801313F4A08
:10641C0003F00103C9B2525C8029617143EA0203A3
:10642C000CBF0422002211F00F0F5BB243EA0203EF
:10643C0014BF002210221343237070BD21792378DE
:10644C000131324A03F00103C9B2525C8029217137
:10645C0043EA02030CBF0422002211F00F0F5BB2BF
:10646C0043EA020314BF002210221343237070BDB1
:10647C00E17A23780131254A03F00103C9B2525C59
:10648C008029E17243EA02030CBF0422002211F0BE
:10649C000F0F5BB243EA020314BF00221022134316
:1064AC00237070BDA17A23780131184A03F00103DF
:1064BC00C9B2525C8029A17243EA02030CBF0422C8
:1064CC00002211F00F0F5BB243EA020314BF00224B
:1064DC0010221343237070BD6178237801310B4A6D
:1064EC0003F00103C9B2525C8029617043EA0203D4
:1064FC000CBF0422002211F00F0F5BB243EA02031F
:10650C0014BF002210221343237070BD0C280020EE
:10651C006589A089FCF7B0FE45FA80F080B2FCF7E3
:10652C00ABFE01302378C5B2AC4A03F00103A0895D
:10653C00525D802D668943EA02030CBF04220022BF
:10654C0015F00F0F5BB243EA020314BF00221022B6
:10655C0013432370431CA381FCF78EFE46FA80F094
:10656C00294680B2BDE87040FCF760BE62782378A3
:10657C00D10923F0130341EA42020B4362702370EA
:10658C0070BD94F90030617803F0010223F013031D
:10659C0042EA410243EAD1136270237070BD617804
:1065AC0011F0010214BF6FF07F03002343EA510383
:1065BC006370237823F013031343237070BD237887
:1065CC00607813F0010F23F0130300F0010214BFE5
:1065DC006FF07F010021134341EA50012370617079
:1065EC0070BDE089617B013880B2E081FCF71EFE52
:1065FC00E089217B013880B2E081FCF717FE002393
:10660C00A38170BDE089617B013880B2E081FCF729
:10661C000DFEE089217B013880B2E081FCF706FE9B
:10662C000823A38170BDE089617B013880B2E081D1
:10663C00FCF7FCFDE089217B013880B2E081FCF79E
:10664C00F5FD1023A38170BDE089617B013880B218
:10665C00E081FCF7EBFDE089217B013880B2E08121
:10666C00FCF7E4FD1823A38170BDE089617B013840
:10667C0080B2E081FCF7DAFDE089217B013880B241
:10668C00E081FCF7D3FD2023A38170BDE089617B01
:10669C00013880B2E081FCF7C9FDE089217B01382B
:1066AC0080B2E081FCF7C2FD2823A38170BDE08994
:1066BC00617B013880B2E081FCF7B8FDE089217B79
:1066CC00013880B2E081FCF7B1FD3023A38170BDAD
:1066DC00E089617B013880B2E081FCF7A7FDE0899D
:1066EC00217B013880B2E081FCF7A0FD3823A38127
:1066FC0070BDE089E178013880B2E081FCF796FD4D
:10670C00E089A178013880B2E081BDE87040FCF7E7
:10671C008DBDE0896179013880B2E081FCF786FD9E
:10672C00E0892179013880B2E081BDE87040FCF746
:10673C007DBDE089E17A013880B2E081FCF776FD1D
:10674C00E089A17A013880B2E081BDE87040FCF7A5
:10675C006DBDE0896178013880B2E081FCF766FD9F
:10676C00E0892178013880B2E081BDE87040FCF707
:10677C005DBDE089431CE381FCF77EFDA070E089E0
:10678C00431CE381FCF778FDE07070BDE089431C8D
:10679C00E381FCF771FD2071E089431CE381FCF778
:1067AC006BFD607170BDE089431CE381FCF764FDF7
:1067BC00A072E089431CE381FCF75EFDE07270BDC2
:1067CC00E089431CE381FCF757FD2070E089431CF2
:1067DC00E381FCF751FD607070BD00BF0C280020F8
:1067EC00E378013BDBB2E37043B1A089FCF744FDD5
:1067FC00A38940B201301844A08170BDA389013334
:10680C00A38170BDA0894FF00005431CA381FCF748
:10681C0033FD60F30705A089FCF72EFD60F30F250F
:10682C00A58170BDA089FCF727FDA38940B201307A
:10683C001844A08170BDA0894FF00005431CA381B2
:10684C00FCF71AFD60F30705A089431CA381FCF734
:10685C0013FD60F30F25E089617B013880B2E08184
:10686C00FCF7E4FCE089217B013880B2E081FCF785
:10687C00DDFCA58170BDE089431CE381FCF7FCFCC9
:10688C002073E089431CE381FCF7F6FC607370BD58
:10689C00237823F0120343F00103237070BD637857
:1068AC00DB436370237843F01203237070BDA0891F
:1068BC00431CA381FCF7E0FC617880B2BDE870401A
:1068CC00FCF730BDA089431CA381FCF7D5FC80B23A
:1068DC00FCF7E2FC607070BD237E23F0010323768D
:1068EC0070BD227E208D42F0010121764FF6FF71A2
:1068FC00884200F09C8442F02102636201232276DC
:10690C00236270BD237883F0010313F0010F23F091
:10691C00120214BF002310231343237070BD63882D
:10692C00628A63826280A388A28AA382A280E3889F
:10693C00E28AE382E28070BDA388E288E380A280D1
:10694C0070BD2388228A2382228070BDE378A370D5
:10695C0070BDE378637170BDE378237170BDE3782B
:10696C00E37270BDE378A37270BDE378637070BDA1
:10697C00A0896589431CA381FCF77EFC45FA80F055
:10698C00E17880B2BDE87040FCF750BCA378E370AE
:10699C0070BDA378637170BDA378237170BDA378AB
:1069AC00E37270BDA378A37270BDA378637070BDE1
:1069BC00A0896589431CA381FCF75EFC45FA80F035
:1069CC00A17880B2BDE87040FCF730BC6379E3700D
:1069DC0070BD6379A37070BD6379237170BD6379E9
:1069EC00E37270BD6379A37270BD6379637070BD1F
:1069FC00A0896589431CA381FCF73EFC45FA80F015
:106A0C00617980B2BDE87040FCF710BC2379E3706B
:106A1C0070BD2379A37070BD2379637170BD237928
:106A2C00E37270BD2379A37270BD2379637070BD5E
:106A3C00A0896589431CA381FCF71EFC45FA80F0F4
:106A4C00217980B2BDE87040FCF7F0BBE37AE370CB
:106A5C0070BDE37AA37070BDE37A637170BDE37AA5
:106A6C00237170BDE37AA37270BDE37A637070BD5D
:106A7C00A0896589431CA381FCF7FEFB45FA80F0D5
:106A8C00E17980B2BDE87040FCF7D0BBA37AE3702B
:106A9C0070BDA37AA37070BDA37A637170BDA37A25
:106AAC00237170BDA37AE37270BDA37A637070BD5D
:106ABC00A0896589431CA381FCF7DEFB45FA80F0B5
:106ACC00A17980B2BDE87040FCF7B0BB6378E3708D
:106ADC0070BD6378A37070BD6378637170BD6378AB
:106AEC00237170BD6378E37270BD6378A37270BD5F
:106AFC00A0896589431CA381FCF7BEFB45FA80F095
:106B0C00617880B2BDE87040FCF790BB617860881A
:106B1C00BDE87040FCF78ABB6178A088BDE8704086
:106B2C00FCF784BBA0896589431CA381FCF7A4FBFB
:106B3C0045FA80F080B2FCF79FFBE07070BDA08935
:106B4C006589431CA381FCF797FB45FA80F080B262
:106B5C00FCF792FBA07070BDA0896589431CA381D2
:106B6C00FCF78AFB45FA80F080B2FCF785FB60717C
:106B7C0070BDA0896589431CA381FCF77DFB45FA98
:106B8C0080F080B2FCF778FB207170BDA08965891C
:106B9C00431CA381FCF770FB45FA80F080B2FCF734
:106BAC006BFBE07170BDA0896589431CA381FCF768
:106BBC0063FB45FA80F080B2FCF75EFBA07170BD00
:106BCC00A0896589431CA381FCF756FB45FA80F02C
:106BDC0080B2FCF751FB607070BDA089431CA3818F
:106BEC00FCF74AFBE07070BDA089431CA381FCF745
:106BFC0043FBA07070BDA089431CA381FCF73CFB38
:106C0C00607170BDA089431CA381FCF735FB20711A
:106C1C0070BDA089431CA381FCF72EFBE07270BDF4
:106C2C00A089431CA381FCF727FBA07270BDA0892F
:106C3C00431CA381FCF720FB607070BDA0896589A3
:106C4C00431CA381FCF718FB45FA80F085B2A089A0
:106C5C00431CA381FCF710FB01462846BDE870409D
:106C6C00FCF7E4BAA0894FF00005431CA381FCF7A4
:106C7C0003FB60F30705A089431CA381FCF7FCFA16
:106C8C0060F30F25A17AADB22846FCF7CFFA681C49
:106C9C00E17A80B2BDE87040FCF7C8BAA0894FF029
:106CAC000005431CA381FCF7E7FA60F30705A089F4
:106CBC00431CA381FCF7E0FA60F30F25ADB2284624
:106CCC00FCF7DAFAA072681C80B2FCF7D5FAE07215
:106CDC0070BDA0894FF00005431CA381FCF7CCFAD2
:106CEC0060F30705A089431CA381FCF7C5FA60F388
:106CFC000F25A8B2FCF7C0FA607070BDA0894FF0E8
:106D0C000005431CA381FCF7B7FA60F30705A089C3
:106D1C00431CA381FCF7B0FA60F30F256178A8B28D
:106D2C00BDE87040FCF782BA4FF00005E089FCF733
:106D3C00A3FAA17A60F30705E089431CE381FCF711
:106D4C0075FAE089FCF798FA60F30F25E089E17A8F
:106D5C00431EE381FCF76AFA658170BD2378627883
:106D6C00D907154648BF42F48075DA0648BF45F48A
:106D7C0000759B07CA4B48BF45F48065ADB233F82C
:106D8C001530238070BDA389013BA38170BDA08900
:106D9C006589431CA381FCF76FFA45FA80F085B234
:106DAC00A089431CA381FCF767FABE4B6F281A5CC1
:106DBC00236AA3EB020323625CD8682880F050811D
:106DCC0047282FD8402880F01B811E2800F0BF8058
:106DDC0019D80E2800F09180162800F0A080062803
:106DEC0040F025822846FCF747FAC0F3C712AE4B99
:106DFC0042EA40012846C9B25B5C13432370BDE8EC
:106E0C007040FCF713BA2E2800F0C68003D8262851
:106E1C0000F0B38070BD362800F0D1803E2800F021
:106E2C00DF8070BD572812D8502880F0F980284692
:106E3C00FCF722FA237810F0020F23F0520314BF50
:106E4C000022402243F010031343237070BD5F28CF
:106E5C0000F2F6802846FCF70FFA237810F0080FA2
:106E6C0023F0520314BF0022402243F010031343BB
:106E7C00237070BDAE2800F05B8119D8862800F015
:106E8C00258106D8772840F2FB807F2840F20E81BE
:106E9C0070BD962800F02E8103D88E2800F020813A
:106EAC0070BD9E2800F03081A62800F0378170BD9F
:106EBC00D62800F071810ED8BE2800F04D8103D881
:106ECC00B62800F03F8170BDC62800F04F81CE2857
:106EDC0000F0578170BDEE2800F07F8106D8DE28C7
:106EEC0000F06581E62800F06D8170BDF62800F099
:106EFC007F81FE2800F0878170BD2846FCF7BCF925
:106F0C0000F00102C0F34701674B284641EAC21169
:106F1C005B5C13432370BDE87040FCF787B92846CF
:106F2C00FCF7AAF9217810F0800F4FEA400001F02D
:106F3C0001015D4B41EA00012846C9B25B5C18BFF8
:106F4C0043F001032370BDE87040FCF76FB928468D
:106F5C00FCF792F9217810F0010F4FEA5000524BD8
:106F6C0040EAC1112846C9B25B5C18BF43F001036B
:106F7C002370BDE87040FCF759B92846FCF77CF942
:106F8C00494B4100C9B25B5C43EAD01020702846E3
:106F9C00BDE87040FCF74AB92846FCF76DF920F0C3
:106FAC007F01414B41EA500100F00100C9B25B5C2A
:106FBC00184320702846BDE87040FCF737B92846C6
:106FCC00FCF75AF9384B410041F00101C9B25B5C46
:106FDC0043EAD01020702846BDE87040FCF726B973
:106FEC002846FCF749F9304BC0F3470100F001008B
:106FFC005B5C184320702846BDE87040FCF716B95E
:10700C002846FCF739F9237810F0010F23F05203CE
:10701C0014BF0022402243F010031343237070BDB1
:10702C002846FCF729F9237810F0040F23F05203BB
:10703C0014BF0022402243F010031343237070BD91
:10704C002846FCF719F9237810F0100F23F052039F
:10705C0014BF0022402243F010031343237070BD71
:10706C002846FCF709F9237810F0200F23F052037F
:10707C0014BF0022402243F010031343237070BD51
:10708C002846FCF7F9F8237810F0400F23F0520350
:10709C0014BF0022402243F010031343237070BD31
:1070AC00180B0020F4250020042700202846FCF7AC
:1070BC00E3F8237810F0800F23F0520314BF002262
:1070CC00402243F010031343237070BD2846FCF795
:1070DC00D3F800F0FE012846BDE87040FCF7A6B8D6
:1070EC002846FCF7C9F800F0FD012846BDE87040C1
:1070FC00FCF79CB82846FCF7BFF800F0FB012846CB
:10710C00BDE87040FCF792B82846FCF7B5F800F0E3
:10711C00F7012846BDE87040FCF788B82846FCF714
:10712C00ABF800F0EF012846BDE87040FCF77EB8E4
:10713C002846FCF7A1F800F0DF012846BDE87040B6
:10714C00FCF774B82846FCF797F800F0BF01284606
:10715C00BDE87040FCF76AB82846FCF78DF800F0E3
:10716C007F012846BDE87040FCF760B82846FCF764
:10717C0083F840F001012846C9B2BDE87040FCF725
:10718C0055B82846FCF778F840F002012846C9B2F9
:10719C00BDE87040FCF74AB82846FCF76DF840F0A3
:1071AC0004012846C9B2BDE87040FCF73FB8284638
:1071BC00FCF762F840F008012846C9B2BDE87040FF
:1071CC00FCF734B82846FCF757F840F01001284675
:1071DC00C9B2BDE87040FCF729B82846FCF74CF85A
:1071EC0040F020012846C9B2BDE87040FCF71EB83B
:1071FC002846FCF741F840F040012846C9B2BDE8EA
:10720C007040FCF713B82846FCF736F860F07F01A5
:10721C002846C9B2BDE87040FCF708B8A389013B09
:10722C00A381237E63F07F0323760023236270BD4A
:10723C0070B504468089431CA381FCF71DF8034BF1
:10724C001A5C0138236A9B1A236201E0F4240020A3
:10725C00FE2802F2FA80DFE810F00608670DB1088C
:10726C00B109C108CE0D970A820C4A084008A10842
:10727C00CB09DC08D50DB00AD10B13086D0DB50880
:10728C00E509F708DC0DA20AF30B61084508A5080F
:10729C00FF091509E30DC00AFF002008130EB908F9
:1072AC00190A3009EA0D8F0E070178082F0EA9086C
:1072BC00330A4B09F10D300C14012D085F0EBD087B
:1072CC00690A8109FF0D290C18018A084A0EAD08BC
:1072DC004D0A6609F80D630CF810A70CC70CE70CE7
:1072EC00070D270D730D470D870CF810CA0CEA0C0F
:1072FC000A0D2A0D800D4A0D8A0CAA0CF810ED0C03
:10730C000D0D2D0D8D0D4D0D8D0CAD0CCD0CF810F6
:10731C00100D300D9A0D500D900CB00CD00CF00CD3
:10732C00F810330DA70D530D930CB30CD30CF30CB9
:10733C00130DF810B40D560D990CB90CD90CF90CA1
:10734C00190D390DEF10590D960CB60CD60CF60C18
:10735C00160D360DC10DF810CA01E50100021B0215
:10736C003602510280026C027A049D04BC04DB04D8
:10737C00FA04190552053805C802E40200031C037F
:10738C003B03570378037303A205C205E20502060B
:10739C002506450677066506C003CA03D403DE033B
:1073AC00E803F2030304FC03C706CF06D706DF0687
:1073BC00E706EF06FC06F70625042D0435043D040C
:1073CC0045044D045A0455041C07360750076A0738
:1073DC008407A307C007BD0752019A0B1C01E30BDE
:1073EC0085015A0BA702D20A71011C0C4001A80E90
:1073FC00B601FC0B7D05E30A6401A70B3801380CC0
:10740C0089016A0B9F03F40A7501700C4401430C4B
:10741C00BA01A40EA206050B6801B40B3C01750E53
:10742C00AD017A0B1704160B79013A0848017D0C53
:10743C00BE01F8100F07270B6C01C10B24014D0C7A
:10744C00B1018A0B6D04380B7F013D084D01520CC4
:10745C00C401A40EE607490B237813F0400F07D0A4
:10746C00A3890133A38170BD237813F0400FF7D0AB
:10747C00A089FBF701FFA38940B201301844A08119
:10748C0070BD237813F0010FE9E7237813F0010F97
:10749C00EDE7237813F0400F07D0A3890233A381C3
:1074AC0070BD94F90030002BF7DBA0894FF000057C
:1074BC00431CA381FBF7E0FE60F30705A089FBF7F3
:1074CC00DBFE60F30F25A58170BD237813F0010F4F
:1074DC00E2E7237813F0040FDEE7237813F0400F74
:1074EC0006E0237813F0010F02E0237813F0040F69
:1074FC00D3D0DAE794F90030002BCEDAD5E7237835
:10750C0013F0400F41F0A187E089431CE381FBF7A6
:10751C00B3FE2073E089431CE381FBF7ADFE60737F
:10752C0070BD237813F0010FECE7237813F0040FF0
:10753C00E8E794F90030002BE6DA70BD237813F0FD
:10754C00400F06E0237813F0010F02E0237813F0CC
:10755C00040F01F07A87D7E794F90030002B81F201
:10756C007487D1E7237813F0400F02E0237813F0EF
:10757C00010F92D1A0894FF00005431CA381FBF7AA
:10758C007BFE60F30705A089431CA381FBF774FE07
:10759C0060F30F25E089617B013880B2E081FBF755
:1075AC0045FEE089217B013880B2E081FBF73EFE8D
:1075BC00A58170BD237813F0040FDAE794F900303D
:1075CC00002BD7DA69E7237813F0400F06E0237815
:1075DC0013F0010F02E0237813F0040F3FF45DAFBA
:1075EC00C8E794F90030002BBFF657AFC2E76378B9
:1075FC00E27899185340C8B2C1F307214240607039
:10760C0022F07F029A43B14A125C14BF0425002574
:10761C00114383EA000202F0100241EA02032B43F9
:10762C00237070BD6378A27899185340C8B2C1F327
:10763C0007214240607022F07F029A43A34A125CF9
:10764C0014BF04250025114383EA000202F0100246
:10765C0041EA02032B43237070BD63786279991859
:10766C005340C8B2C1F307214240607022F07F0240
:10767C009A43964A125C14BF04250025114383EAF1
:10768C00000202F0100241EA02032B43237070BD8A
:10769C006378227999185340C8B2C1F3072142404C
:1076AC00607022F07F029A43884A125C14BF042552
:1076BC000025114383EA000202F0100241EA0203A2
:1076CC002B43237070BD6378627A99185340C8B20B
:1076DC00C1F307214240607022F07F029A437B4A3B
:1076EC00125C14BF04250025114383EA000202F04A
:1076FC00100241EA02032B43237070BD6378227A97
:10770C0099185340C8B2C1F307214240607022F06F
:10771C007F029A436D4A125C14BF04250025114365
:10772C0083EA000202F0100241EA02032B432370A9
:10773C0070BD62785300D9B24A40617012F0800F6C
:10774C0001F0100242EA1323604A14BF0420002007
:10775C00525C13430343237070BDA0892589431CDD
:10776C00A381FBF789FD45FA80F080B2FBF784FD1D
:10777C00637856491A184340D5B2C2F30722DBB2DC
:10778C006840495D657020EA0300114383EA0502F5
:10779C0010F0800F02F0100214BF0420002041EA08
:1077AC0002030343237070BDA089431CA381FBF724
:1077BC0063FD637845491A184340D5B2C2F30722DA
:1077CC00DBB26840495D657020EA0300114383EA2F
:1077DC00050210F0800F02F0100214BF04200020EC
:1077EC0041EA02030343237070BD6278E378D11A37
:1077FC005340C8B2C1F307214240494260701A405D
:10780C0012F0800F314A125C14BF06250225114379
:10781C0083EA000202F0100241EA02032B432370B8
:10782C0070BD6278A378D11A5340C8B2C1F3072156
:10783C004240494260701A4012F0800F234A125C99
:10784C0014BF06250225114383EA000202F0100240
:10785C0041EA02032B43237070BD62786379D11A1D
:10786C005340C8B2C1F307214240494260701A40EC
:10787C0012F0800F154A125C14BF06250225114325
:10788C0083EA000202F0100241EA02032B43237048
:10789C0070BD62782379D11A5340C8B2C1F3072165
:1078AC004240494260701A4012F0800F074A125C45
:1078BC0014BF06250225114383EA000202F01002D0
:1078CC0041EA02032B43237070BD00BF0C2800203B
:1078DC006278637AD11A5340C8B2C1F3072142408F
:1078EC00494260701A4012F0800FA84A125C14BF13
:1078FC0006250225114383EA000202F0100241EA38
:10790C0002032B43237070BD6278237AD11A534043
:10791C00C8B2C1F307214240494260701A4012F0CC
:10792C00800F9A4A125C14BF06250225114383EA84
:10793C00000202F0100241EA02032B43237070BDD7
:10794C00002363704223237070BDA0892589431CDA
:10795C00A381FBF791FC45FA80F080B2FBF78CFC1D
:10796C0063781A1A5840D1B2C2F30722C0B24B4006
:10797C0052426170034013F0800F844B5B5C14BF68
:10798C00062502251A4380EA010303F0100342EA9C
:10799C0003002843207070BDA089431CA381FBF712
:1079AC006BFC63781A1A5840D1B2C2F30722C0B2EA
:1079BC004B4052426170034013F0800F734B5B5C81
:1079CC0014BF062502251A4380EA010303F01003B5
:1079DC0042EA03002843207070BD6278E3781340BC
:1079EC006B4A6370D35C43F01003237070BD6278F4
:1079FC00A3781340664A6370D35C43F01003237082
:107A0C0070BD627863791340614A6370D35C43F054
:107A1C001003237070BD6278237913405C4A637045
:107A2C00D35C43F01003237070BD6278637A13400B
:107A3C00574A6370D35C43F01003237070BD6278B7
:107A4C00237A1340524A6370D35C43F010032370C3
:107A5C0070BD63784E4AD35C43F01003237070BD45
:107A6C00A0892589431CA381FBF706FC45FA80F00D
:107A7C0080B2FBF701FC63781840454B1B5C6070CF
:107A8C0043F01003237070BDA089431CA381FBF746
:107A9C00F3FB637818403E4B1B5C607043F01003A3
:107AAC00237070BD6278E3781343394A6370D35CFA
:107ABC00237070BD6278A3781343354A6370D35C2E
:107ACC00237070BD627863791343314A6370D35C61
:107ADC00237070BD6278237913432D4A6370D35C95
:107AEC00237070BD6278637A1343294A6370D35C48
:107AFC00237070BD6278237A1343254A6370D35C7C
:107B0C00237070BD6378224AD35C237070BDA0894A
:107B1C002589431CA381FBF7AFFB45FA80F080B2AB
:107B2C00FBF7AAFB63781843194BC0B21B5C60705F
:107B3C00237070BDA089431CA381FBF79DFB637868
:107B4C001843134BC0B21B5C6070237070BD63781C
:107B5C00E178227802F001005A184B400244D0B26E
:107B6C00C2F307224140607021F07F01994307491D
:107B7C00095C14BF04250025114383EA000202F0BE
:107B8C00100241EA02032B43237070BD0C28002025
:107B9C00042700206378A178227802F001005A189B
:107BAC004B400244D0B2C2F307224140607021F036
:107BBC007F019943BA49095C14BF04250025114380
:107BCC0083EA000202F0100241EA02032B43237005
:107BDC0070BD63786179227802F001005A184B402D
:107BEC000244D0B2C2F307224140607021F07F0101
:107BFC009943AB49095C14BF04250025114383EA62
:107C0C00000202F0100241EA02032B43237070BD04
:107C1C0063782179227802F001005A184B40024413
:107C2C00D0B2C2F307224140607021F07F0199432A
:107C3C009B49095C14BF04250025114383EA00020B
:107C4C0002F0100241EA02032B43237070BD6378EB
:107C5C00617A227802F001005A184B400244D0B2EB
:107C6C00C2F307224140607021F07F0199438C4997
:107C7C00095C14BF04250025114383EA000202F0BD
:107C8C00100241EA02032B43237070BD6378217A02
:107C9C00227802F001005A184B400244D0B2C2F3D1
:107CAC0007224140607021F07F0199437C49095CB7
:107CBC0014BF04250025114383EA000202F01002D0
:107CCC0041EA02032B43237070BD2378627803F0E2
:107CDC00010303EB4203D9B2C3F307234A4061709B
:107CEC0012F0800F01F0100243EA02036C4A14BF39
:107CFC0004200020525C13430343237070BDA08901
:107D0C002589431CA381FBF7B7FA45FA80F080B2B2
:107D1C00FBF7B2FA2278637802F0010260491A4448
:107D2C0043400244DBB2D5B2C2F307226840495D3E
:107D3C00657020EA0300114383EA050210F0800FFE
:107D4C0002F0100214BF0420002041EA0203034396
:107D5C00237070BDA089431CA381FBF78DFA227898
:107D6C00637802F001024E491A4443400244DBB2EC
:107D7C00D5B2C2F307226840495D657020EA030062
:107D8C00114383EA050210F0800F02F0100214BFB9
:107D9C000420002041EA02030343237070BD607885
:107DAC00E3782278C11A434002F001028A1AD1B258
:107DBC00C2F30722484052426170184010F0800F05
:107DCC003748405C14BF06250225104383EA0102A4
:107DDC0002F0100240EA02032B43237070BD60785E
:107DEC00A3782278C11A434002F001028A1AD1B258
:107DFC00C2F30722484052426170184010F0800FC5
:107E0C002748405C14BF06250225104383EA010273
:107E1C0002F0100240EA02032B43237070BD60781D
:107E2C0063792278C11A434002F001028A1AD1B256
:107E3C00C2F30722484052426170184010F0800F84
:107E4C001748405C14BF06250225104383EA010243
:107E5C0002F0100240EA02032B43237070BD6078DD
:107E6C0023792278C11A434002F001028A1AD1B256
:107E7C00C2F30722484052426170184010F0800F44
:107E8C000748405C14BF06250225104383EA010213
:107E9C0002F0100240EA02032B43237070BD00BFB6
:107EAC000C2800206078637A2278C11A434002F0D3
:107EBC0001028A1AD1B2C2F30722484052426170C1
:107ECC00184010F0800FB448405C14BF0625022502
:107EDC00104383EA010202F0100240EA02032B4332
:107EEC00237070BD6078237A2278C11A434002F067
:107EFC0001028A1AD1B2C2F3072248405242617081
:107F0C00184010F0800FA448405C14BF06250225D1
:107F1C00104383EA010202F0100240EA02032B43F1
:107F2C00237070BD237843F30003D9B2C3F3072346
:107F3C0001F010025B4261701343974A43F0020355
:107F4C00525C1343237070BDA0892589431CA38107
:107F5C00FBF792F945FA80F080B2FBF78DF9617866
:107F6C0023780A1A484003F00103C0B2D31ADAB2DC
:107F7C00C3F3072351405B426270014011F0800F44
:107F8C008549895C14BF06250225194380EA020342
:107F9C0003F0100341EA03002843207070BDA08950
:107FAC00431CA381FBF768F9617823780A1A4840CF
:107FBC0003F00103C0B2D31ADAB2C3F30723514062
:107FCC005B426270014011F0800F7349895C14BFF1
:107FDC0006250225194380EA020303F0100341EA47
:107FEC0003002843207070BD6278E37853406B4ADD
:107FFC006370D35C237070BD6278A3785340674A7A
:10800C006370D35C237070BD627863795340634AAC
:10801C006370D35C237070BD6278237953405F4AE0
:10802C006370D35C237070BD6278637A53405B4A93
:10803C006370D35C237070BD6278237A5340574AC7
:10804C006370D35C237070BD002363704423237072
:10805C0070BDA0892589431CA381FBF70DF945FA56
:10806C0080F080B2FBF708F9637858404B4BC0B2F4
:10807C001B5C6070237070BDA089431CA381FBF74F
:10808C00FBF863785840454BC0B21B5C60702370A2
:10809C0070BD6178E278881A4A40C3B2C0F30720F9
:1080AC005940404211405A4011F0800F3A4902F0B9
:1080BC001002C95C14BF06250225084340EA0203DE
:1080CC002B43237070BD6178A278881A4A40C3B2E2
:1080DC00C0F307205940404211405A4011F0800F24
:1080EC002D4902F01002C95C14BF06250225084375
:1080FC0040EA02032B43237070BD61786279881AC1
:10810C004A40C3B2C0F307205940404211405A4084
:10811C0011F0800F204902F01002C95C14BF062533
:10812C000225084340EA02032B43237070BD61789B
:10813C002279881A4A40C3B2C0F307205940404202
:10814C0011405A4011F0800F134902F01002C95C23
:10815C0014BF06250225084340EA02032B43237073
:10816C0070BD6178627A881A4A40C3B2C0F30720A6
:10817C005940404211405A4011F0800F064902F01C
:10818C001002C95C14BF06250225084340EA02030D
:10819C002B43237070BD00BF0C2800200427002047
:1081AC006178227A881A4A40C3B2C0F3072059403A
:1081BC00404211405A4011F0800FB14902F01002B8
:1081CC00C95C14BF06250225084340EA02032B4371
:1081DC00237070BD4223237070BDA0892589431C78
:1081EC00A381FBF749F845FA80F080B2FBF744F81D
:1081FC0061780D1A80EA0102EBB2C5F30725D2B201
:10820C0059406D4211405A4011F0800F9C4902F0C8
:10821C001002C95C14BF062002200D4345EA02037C
:10822C000343237070BDA089431CA381FBF724F882
:10823C0061780D1A80EA0102EBB2C5F30725D2B2C0
:10824C0059406D4211405A4011F0800F8C4902F098
:10825C001002C95C14BF062002200D4345EA02033C
:10826C000343237070BDA089431CA381FBF704F862
:10827C00A070A089431CA381FAF7FEFFE07070BDCB
:10828C00A089431CA381FAF7F7FF2071A089431C36
:10829C00A381FAF7F1FF607170BDA089431CA38123
:1082AC00FAF7EAFF2072A089431CA381FAF7E4FFD6
:1082BC00607270BDA089431CA381FAF7DDFFA07327
:1082CC00A089431CA381FAF7D7FFE07370BD238903
:1082DC00A38170BD2389E38170BD6088FAF7CCFF60
:1082EC00607070BDA088FAF7C7FF607070BD2589FB
:1082FC00628894F90010AB186A4021F0130198B20F
:10830C004240208112F4805FC3F3004214BF102559
:10831C00002541EA02032B43237070BD2589A288F6
:10832C0094F90010AB186A4021F0130198B2424046
:10833C00208112F4805FC3F3004214BF1025002586
:10834C0041EA02032B43237070BD238994F900206A
:10835C005B0022F0130299B242EA134311F4805FDE
:10836C00218114BF102000200343237070BD258988
:10837C00E28994F90010AB186A4021F0130198B20D
:10838C004240208112F4805FC3F3004214BF1025D9
:10839C00002541EA02032B43237070BD6388013B27
:1083AC00638070BDA388013BA38070BD2389013B12
:1083BC00238170BDE389013BE38170BD6388013388
:1083CC00638070BDA3880133A38070BD2389013302
:1083DC00238170BDE3890133E38170BDE17822789C
:1083EC000139274B02F00102C9B242F00202585C7B
:1083FC007F29E17001F00F010CBF0423002302431D
:10840C000F2943EA02030CBF102100210B432370F8
:10841C0070BDA17822780139194B02F00102C9B262
:10842C0042F00202585C7F29A17001F00F010CBFD1
:10843C000423002302430F2943EA02030CBF10213B
:10844C0000210B43237070BD6179227801390C4BEC
:10845C0002F00102C9B242F00202585C7F2961713C
:10846C0001F00F010CBF0423002302430F2943EA40
:10847C0002030CBF102100210B43237070BD00BF01
:10848C000C280020217922780139A74B02F0010237
:10849C00C9B242F00202585C7F29217101F00F0130
:1084AC000CBF0423002302430F2943EA02030CBF31
:1084BC00102100210B43237070BD617A22780139A1
:1084CC00994B02F00102C9B242F00202585C7F29BA
:1084DC00617201F00F010CBF0423002302430F292A
:1084EC0043EA02030CBF102100210B43237070BD23
:1084FC00217A227801398C4B02F00102C9B242F088
:10850C000202585C7F29217201F00F010CBF042379
:10851C00002302430F2943EA02030CBF1021002160
:10852C000B43237070BD6178227801397E4B02F0C9
:10853C000102C9B242F00202585C7F29617001F05D
:10854C000F010CBF0423002302430F2943EA02034B
:10855C000CBF102100210B43237070BD2589A0890D
:10856C00FAF78AFE45FA80F080B2FAF785FE227897
:10857C0001386D4B02F001022689C5B2A08942F088
:10858C000202595D7F2D42EA010205F00F010CBF7A
:10859C00042300230F2943EA02030CBF10210021FE
:1085AC000B432370431CA381FAF766FE46FA80F056
:1085BC00294680B2BDE87040FAF738BEE1782378DE
:1085CC000131594A03F00103C9B2525C8029E170B0
:1085DC0043EA02030CBF0422002211F00F0F5BB21E
:1085EC0043EA020314BF002210221343237070BD10
:1085FC00A178237801314C4A03F00103C9B2525CD3
:10860C008029A17043EA02030CBF0422002211F05E
:10861C000F0F5BB243EA020314BF00221022134374
:10862C00237070BD6179237801313F4A03F0010357
:10863C00C9B2525C8029617143EA02030CBF042267
:10864C00002211F00F0F5BB243EA020314BF0022A9
:10865C0010221343237070BD217923780131324AE3
:10866C0003F00103C9B2525C8029217143EA020371
:10867C000CBF0422002211F00F0F5BB243EA02037D
:10868C0014BF002210221343237070BD617A23782B
:10869C000131254A03F00103C9B2525C8029617291
:1086AC0043EA02030CBF0422002211F00F0F5BB24D
:1086BC0043EA020314BF002210221343237070BD3F
:1086CC00217A23780131184A03F00103C9B2525CB4
:1086DC008029217243EA02030CBF0422002211F00C
:1086EC000F0F5BB243EA020314BF002210221343A4
:1086FC00237070BD6178237801310B4A03F00103BC
:10870C00C9B2525C8029617043EA02030CBF042297
:10871C00002211F00F0F5BB243EA020314BF0022D8
:10872C0010221343237070BD0C2800202589A089CA
:10873C00FAF7A2FD45FA80F080B2FAF79DFD013000
:10874C002378C5B2AC4A03F00103A089525D802D99
:10875C00268943EA02030CBF0422002215F00F0FF6
:10876C005BB243EA020314BF0022102213432370AE
:10877C00431CA381FAF780FD46FA80F0294680B2AB
:10878C00BDE87040FAF752BD62782378D10923F026
:10879C00130341EA42020B436270237070BD94F9DB
:1087AC000030617803F0010223F0130342EA410226
:1087BC0043EAD1136270237070BD617811F001022D
:1087CC0014BF6FF07F03002343EA510363702378D7
:1087DC0023F013031343237070BD2378607813F0D8
:1087EC00010F23F0130300F0010214BF6FF07F019F
:1087FC000021134341EA50012370617070BDE08980
:10880C00617B013880B2E081FAF710FDE089217BB1
:10881C00013880B2E081FAF709FD0023A38170BD15
:10882C00E089617B013880B2E081FAF7FFFCE089D6
:10883C00217B013880B2E081FAF7F8FC0823A38190
:10884C0070BDE089617B013880B2E081FAF7EEFC03
:10885C00E089217B013880B2E081FAF7E7FC102334
:10886C00A38170BDE089617B013880B2E081FAF7A9
:10887C00DDFCE089217B013880B2E081FAF7D6FC7F
:10888C001823A38170BDE089617B013880B2E0813F
:10889C00FAF7CCFCE089217B013880B2E081FAF751
:1088AC00C5FC2023A38170BDE089617B013880B2B7
:1088BC00E081FAF7BBFCE089217B013880B2E081D2
:1088CC00FAF7B4FC2823A38170BDE089617B0138E1
:1088DC0080B2E081FAF7AAFCE089217B013880B2F2
:1088EC00E081FAF7A3FC3023A38170BDE089617BA2
:1088FC00013880B2E081FAF799FCE089217B0138DC
:10890C0080B2E081FAF792FC3823A38170BDE08934
:10891C00E178013880B2E081FAF788FCE089A1782F
:10892C00013880B2E081BDE87040FAF77FBCE08985
:10893C006179013880B2E081FAF778FCE08921791D
:10894C00013880B2E081BDE87040FAF76FBCE08975
:10895C00617A013880B2E081FAF768FCE089217A0B
:10896C00013880B2E081BDE87040FAF75FBCE08965
:10897C006178013880B2E081FAF758FCE0892178FF
:10898C00013880B2E081BDE87040FAF74FBCE08955
:10899C00431CE381FAF770FCA070E089431CE3816F
:1089AC00FAF76AFCE07070BDE089431CE381FAF7CA
:1089BC0063FC2071E089431CE381FAF75DFC607174
:1089CC0070BDE089431CE381FAF756FC2072E08904
:1089DC00431CE381FAF750FC607270BDE089431CC4
:1089EC00E381FAF749FC2070E089431CE381FAF734
:1089FC0043FC607070BD00BF0C280020E378013B85
:108A0C00DBB2E37043B1A089FAF736FCA38940B21C
:108A1C0001301844A08170BDA3890133A38170BDBE
:108A2C00A0894FF00005431CA381FAF725FC60F3E5
:108A3C000705A089FAF720FC60F30F25A58170BD0E
:108A4C00A089FAF719FCA38940B201301844A0811F
:108A5C0070BDA0894FF00005431CA381FAF70CFCF4
:108A6C0060F30705A089431CA381FAF705FC60F3AA
:108A7C000F25E089617B013880B2E081FAF7D6FBE3
:108A8C00E089217B013880B2E081FAF7CFFBA58128
:108A9C0070BDE089431CE381FAF7EEFB2073E0899B
:108AAC00431CE381FAF7E8FB607370BD237823F075
:108ABC00120343F00103237070BD6378DB436370D2
:108ACC00237843F01203237070BDA089431CA3814B
:108ADC00FAF7D2FB617880B2BDE87040FAF722BC9D
:108AEC00A089431CA381FAF7C7FB80B2FAF7D4FB29
:108AFC00607070BD237E23F00103237670BD227E4F
:108B0C00208D42F0010121764FF6FF71884200F072
:108B1C009C8442F02102636201232276236270BDA1
:108B2C00237883F0010313F0010F23F0120214BF1A
:108B3C00002310231343237070BD6388628A638201
:108B4C006280A388A28AA382A280E388E28AE3825D
:108B5C00E28070BDA388E288E380A28070BD238888
:108B6C00228A2382228070BDE378A37070BDE378E3
:108B7C00637170BDE378237170BDE378637270BD6F
:108B8C00E378237270BDE378637070BDA08925898A
:108B9C00431CA381FAF770FB45FA80F0E17880B2B0
:108BAC00BDE87040FAF742BBA378E37070BDA378C0
:108BBC00637170BDA378237170BDA378637270BDAF
:108BCC00A378237270BDA378637070BDA0892589CA
:108BDC00431CA381FAF750FB45FA80F0A17880B2D0
:108BEC00BDE87040FAF722BB6379E37070BD63791E
:108BFC00A37070BD6379237170BD6379637270BDAE
:108C0C006379237270BD6379637070BDA089258907
:108C1C00431CA381FAF730FB45FA80F0617980B2EE
:108C2C00BDE87040FAF702BB2379E37070BD23797D
:108C3C00A37070BD2379637170BD2379637270BDAD
:108C4C002379237270BD2379637070BDA089258947
:108C5C00431CA381FAF710FB45FA80F0217980B20E
:108C6C00BDE87040FAF7E2BA637AE37070BD637ADC
:108C7C00A37070BD637A637170BD637A237170BD2C
:108C8C00637A237270BD637A637070BDA089258985
:108C9C00431CA381FAF7F0FA45FA80F0E17980B22F
:108CAC00BDE87040FAF7C2BA237AE37070BD237A3C
:108CBC00A37070BD237A637170BD237A237170BD6C
:108CCC00237A637270BD237A637070BDA089258985
:108CDC00431CA381FAF7D0FA45FA80F0A17980B24F
:108CEC00BDE87040FAF7A2BA6378E37070BD6378A0
:108CFC00A37070BD6378637170BD6378237170BDB0
:108D0C006378637270BD6378237270BDA089258906
:108D1C00431CA381FAF7B0FA45FA80F0617880B26F
:108D2C00BDE87040FAF782BA61786088BDE870409F
:108D3C00FAF77CBA6178A088BDE87040FAF776BA89
:108D4C00A0892589431CA381FAF796FA45FA80F08D
:108D5C0080B2FAF791FAE07070BDA0892589431CA6
:108D6C00A381FAF789FA45FA80F080B2FAF784FA0F
:108D7C00A07070BDA0892589431CA381FAF77CFAE9
:108D8C0045FA80F080B2FAF777FA607170BDA0896D
:108D9C002589431CA381FAF76FFA45FA80F080B25B
:108DAC00FAF76AFA207170BDA0892589431CA3814A
:108DBC00FAF762FA45FA80F080B2FAF75DFAE071E0
:108DCC0070BDA0892589431CA381FAF755FA45FA91
:108DDC0080F080B2FAF750FAA07170BDA089258995
:108DEC00431CA381FAF748FA45FA80F080B2FAF7EF
:108DFC0043FA607070BDA089431CA381FAF73CFA5A
:108E0C00E07070BDA089431CA381FAF735FAA070FD
:108E1C0070BDA089431CA381FAF72EFA607170BD56
:108E2C00A089431CA381FAF727FA207170BDA08991
:108E3C00431CA381FAF720FA607270BDA089431C11
:108E4C00A381FAF719FA207270BDA089431CA38183
:108E5C00FAF712FA607070BDA0892589431CA381B2
:108E6C00FAF70AFA45FA80F085B2A089431CA3816F
:108E7C00FAF702FA01462846BDE87040FAF7D6B96F
:108E8C00A0894FF00005431CA381FAF7F5F960F3B4
:108E9C000705A089431CA381FAF7EEF960F30F25AF
:108EAC00217AADB22846FAF7C1F9681C617A80B212
:108EBC00BDE87040FAF7BAB9A0894FF00005431C21
:108ECC00A381FAF7D9F960F30705A089431CA381A4
:108EDC00FAF7D2F960F30F25ADB22846FAF7CCF9C0
:108EEC002072681C80B2FAF7C7F9607270BDA08955
:108EFC004FF00005431CA381FAF7BEF960F3070598
:108F0C00A089431CA381FAF7B7F960F30F25A8B227
:108F1C00FAF7B2F9607070BDA0894FF00005431CE0
:108F2C00A381FAF7A9F960F30705A089431CA38173
:108F3C00FAF7A2F960F30F256178A8B2BDE870408A
:108F4C00FAF774B94FF00005E089FAF795F9217A30
:108F5C0060F30705E089431CE381FAF767F9E089C0
:108F6C00FAF78AF960F30F25E089617A431EE381F1
:108F7C00FAF75CF9258170BD23786278D90715461C
:108F8C0048BF42F48075DA0648BF45F400759B076C
:108F9C00CA4B48BF45F48065ADB233F81530238019
:108FAC0070BDA389013BA38170BDA0892589431C99
:108FBC00A381FAF761F945FA80F085B2A089431CC8
:108FCC00A381FAF759F9BE4B6F281A5C236AA3EBFD
:108FDC00020323625CD8682880F0508147282FD880
:108FEC00402880F01B811E2800F0BF8019D80E2865
:108FFC0000F09180162800F0A080062840F0258211
:10900C002846FAF739F9C0F3C712AE4B42EA4001D1
:10901C002846C9B25B5C13432370BDE87040FAF775
:10902C0005B92E2800F0C68003D8262800F0B3809E
:10903C0070BD362800F0D1803E2800F0DF8070BD76
:10904C00572812D8502880F0F9802846FAF714F9DE
:10905C00237810F0020F23F0520314BF0022402299
:10906C0043F010031343237070BD5F2800F2F680A9
:10907C002846FAF701F9237810F0080F23F0520371
:10908C0014BF0022402243F010031343237070BD21
:10909C00AE2800F05B8119D8862800F0258106D80F
:1090AC00772840F2FB807F2840F20E8170BD962815
:1090BC0000F02E8103D88E2800F0208170BD9E28F0
:1090CC0000F03081A62800F0378170BDD62800F062
:1090DC0071810ED8BE2800F04D8103D8B62800F05F
:1090EC003F8170BDC62800F04F81CE2800F057811B
:1090FC0070BDEE2800F07F8106D8DE2800F0658177
:10910C00E62800F06D8170BDF62800F07F81FE2806
:10911C0000F0878170BD2846FAF7AEF800F0010226
:10912C00C0F34701674B284641EAC2115B5C13430D
:10913C002370BDE87040FAF779B82846FAF79CF826
:10914C00217810F0800F4FEA400001F001015D4BD7
:10915C0041EA00012846C9B25B5C18BF43F0010329
:10916C002370BDE87040FAF761B82846FAF784F826
:10917C00217810F0010F4FEA5000524B40EAC11118
:10918C002846C9B25B5C18BF43F001032370BDE8ED
:10919C007040FAF74BB82846FAF76EF8494B410085
:1091AC00C9B25B5C43EAD01020702846BDE8704021
:1091BC00FAF73CB82846FAF75FF820F07F01414BEC
:1091CC0041EA500100F00100C9B25B5C1843207009
:1091DC002846BDE87040FAF729B82846FAF74CF84B
:1091EC00384B410041F00101C9B25B5C43EAD0103D
:1091FC0020702846BDE87040FAF718B82846FAF7F0
:10920C003BF8304BC0F3470100F001005B5C1843A6
:10921C0020702846BDE87040FAF708B82846FAF7DF
:10922C002BF8237810F0010F23F0520314BF002207
:10923C00402243F010031343237070BD2846FAF705
:10924C001BF8237810F0040F23F0520314BF0022F4
:10925C00402243F010031343237070BD2846FAF7E5
:10926C000BF8237810F0100F23F0520314BF0022D8
:10927C00402243F010031343237070BD2846F9F7C6
:10928C00FBFF237810F0200F23F0520314BF0022B1
:10929C00402243F010031343237070BD2846F9F7A6
:1092AC00EBFF237810F0400F23F0520314BF002281
:1092BC00402243F010031343237070BD180B0020A1
:1092CC00F4250020042700202846F9F7D5FF237841
:1092DC0010F0800F23F0520314BF0022402243F001
:1092EC0010031343237070BD2846F9F7C5FF00F037
:1092FC00FE012846BDE87040F9F798BF2846F9F7FB
:10930C00BBFF00F0FD012846BDE87040F9F78EBFA9
:10931C002846F9F7B1FF00F0FB012846BDE8704084
:10932C00F9F784BF2846F9F7A7FF00F0F7012846A4
:10933C00BDE87040F9F77ABF2846F9F79DFF00F0B9
:10934C00EF012846BDE87040F9F770BF2846F9F7E1
:10935C0093FF00F0DF012846BDE87040F9F766BFC7
:10936C002846F9F789FF00F0BF012846BDE8704098
:10937C00F9F75CBF2846F9F77FFF00F07F0128461C
:10938C00BDE87040F9F752BF2846F9F775FF40F079
:10939C0001012846C9B2BDE87040F9F747BF28461D
:1093AC00F9F76AFF40F002012846C9B2BDE87040E7
:1093BC00F9F73CBF2846F9F75FFF40F00401284657
:1093CC00C9B2BDE87040F9F731BF2846F9F754FF30
:1093DC0040F008012846C9B2BDE87040F9F726BF35
:1093EC002846F9F749FF40F010012846C9B2BDE8FC
:1093FC007040F9F71BBF2846F9F73EFF40F02001FB
:10940C002846C9B2BDE87040F9F710BF2846F9F7F5
:10941C0033FF40F040012846C9B2BDE87040F9F76F
:10942C0005BF2846F9F728FF60F07F012846C9B22E
:10943C00BDE87040F9F7FABEA389013BA381237EF6
:10944C0063F07F0323760023236270BDF8B50446D6
:10945C008089431CA381F9F70FFFBF4B6728195C68
:10946C00236AA3EB0101216200F0528200F2988082
:10947C00512800F001835BD8462800F08D8227D854
:10948C00422800F06D8106D8402800F0C4824128A3
:10949C0000F0ED82F8BD442800F0A48200F28D8229
:1094AC00A0894FF00005431CA381F9F7E5FE60F39A
:1094BC000705A089431CA381F9F7DEFE60F30F2595
:1094CC00A178ADB22846F9F7B1FE681CE178CCE181
:1094DC004A2800F0E78007D8482800F0A68200F25E
:1094EC00C88263786376F8BD4D2800F06E825028F0
:1094FC0000F0A0824B2840F02C84A0894FF000058E
:10950C00431CA381F9F7B8FE60F30705A089431C3F
:10951C00A381F9F7B1FE60F30F25ADB22846F9F738
:10952C00ABFEA070681C80B2F9F7A6FEE070F8BD27
:10953C005A2800F0BD801DD8562800F0318206D87C
:10954C00522800F03A81532800F07881F8BD582851
:10955C0000F0758200F29282217E627E11F0010F82
:10956C0023787E48627003F0010314BF04210021AC
:10957C00825CADE3602800F0678208D85E2800F0BA
:10958C00158200F2F2815B2800F08C81F8BD622814
:10959C0000F01981C0F07482632800F03781F8BDA7
:1095AC00A22800F0778248D8722800F029812ED8A2
:1095BC006A2800F0A68006D8682800F04A8269283C
:1095CC0000F06082F8BD6F2800F0BB81702800F0BD
:1095DC004A826B2840F0BD83A0894FF00005431CE4
:1095EC00A381F9F749FE60F30705A089431CA38109
:1095FC00F9F742FE60F30F25ADB22846F9F73CFEB1
:10960C00A071681C80B2F9F737FEE071F8BD7A28BA
:10961C0000F09C8008D8782800F0208200F2348278
:10962C00732800F02781F8BDA02800F0B88200F262
:10963C0017837B2800F05181F8BDB22800F03082EE
:10964C0015D8AA2800F0418208D8A82800F0CA82B0
:10965C0000F22083A32800F05B82F8BDB02800F054
:10966C00A68200F20483AB2800F06E82F8BDBA2803
:10967C0000F0398208D8B82800F0D08200F22D838F
:10968C00B32800F04C82F8BDED2800F05583FE287D
:10969C0003D0BB2840F05D836CE22046BDE8F84067
:1096AC00F9F7F8BD2278E18802F00102658804E040
:1096BC002278E18802F00102A5884B1969401A440E
:1096CC00CB4390B203F40043C2F300424540414007
:1096DC00E0802B4214BF0426002611F4805FC0F3F7
:1096EC00072121F07F0114BF10230023002842EA38
:1096FC00010214BF00254025324313432B43237032
:10970C00F8BD2278E38802F0010202EB430295B225
:10971C00C2F300426B4005F4805013F4004F83B247
:10972C0014BF0427002713B925B1184600E01020F8
:10973C00002601E028464026C5F3072121F07F01D1
:10974C000A433A4340EA0203334333E02278E18888
:10975C0002F00102E589B0E7F42300200C28002078
:10976C002378E08803F001026188431A41409B1A78
:10977C009DB213F4803F80EA050014BF032202223D
:10978C000840694010F4004F14BF0423002311F467
:10979C00805FC5F3072121F07F0114BF102600263E
:1097AC00002D42EA010214BF002040201A4346EA71
:1097BC00020303432370E580F8BD2378E08803F0AF
:1097CC000102A188D1E7237843F3000399B213F483
:1097DC00803FC1F3072201F4805314BF03250225F7
:1097EC0022F07F02002BE1800CBF0023102342EA01
:1097FC0005020CBF40200020134303432370F8BD27
:10980C002378E08803F00102E189AEE7A0894FF0EC
:10981C000005431CA381F9F72FFD60F30705A08910
:10982C00431CA381F9F728FD60F30F25A179ADB294
:10983C002846F9F7FBFC681CE17916E0A0894FF08B
:10984C000005431CA381F9F717FD60F30705A089F8
:10985C00431CA381F9F710FD60F30F252179ADB2FC
:10986C002846F9F7E3FC681C617980B2BDE8F84042
:10987C00F9F7DCBCA0894FF00005431CA381F9F774
:10988C00FBFC60F30705A089431CA381F9F7F4FCEA
:10989C0060F30F25A17BADB22846F9F7C7FC681C15
:1098AC00E17BE2E7A0894FF00005431CA381F9F7A7
:1098BC00E3FC60F30705A089431CA381F9F7DCFCEA
:1098CC0060F30F25ADB22846F9F7D6FC2071681C61
:1098DC0080B2F9F7D1FC6071F8BDA0894FF000059A
:1098EC00431CA381F9F7C8FC60F30705A089431C4E
:1098FC00A381F9F7C1FC60F30F25ADB22846F9F747
:10990C00BBFCA073681C80B2F9F7B6FCE073F8BD21
:10991C00E088F9F7B1FC617803090546E08843EA71
:10992C00011105F00F05C9B2F9F780FC637823F03B
:10993C000F031D43237803F00102A84B65705B5D98
:10994C0068E1E088F9F798FC6178054601F00F01B1
:10995C0041EA0011E088C9B2F9F768FC607820F0A0
:10996C000F0040EA1510C0B27BE0A27E0132D3B2E8
:10997C00227EA3765B1A12F0010F2178DBB2984A93
:10998C0001F0010118BF0420D25C08BF00206370F5
:10999C0041EA020303439DE1237E23F006030AE020
:1099AC00237E23F0060343F0020304E0237E23F01E
:1099BC00060343F004032376F8BD237E5A064CBFFE
:1099CC0043F0010323F001032376E089431CE38178
:1099DC00F9F752FC2073E089431CE381F9F74CFC46
:1099EC006073F8BD62785342D9B202EA01004A4072
:1099FC00617010F0800F7A4802F01002405C14BFC6
:109A0C00062502251043C3F30722524240EA020303
:109A1C002B432370F8BDA078F9F73EFCE070237857
:109A2C0003F001026D4B1B5CF4E0A078F9F734FCF9
:109A3C00A070F4E7A078F9F72FFC6071EFE7A0783D
:109A4C00F9F72AFC2071EAE7A078F9F725FCE07118
:109A5C00E5E7A078F9F720FCA071E0E7A078F9F72A
:109A6C001BFC6070DBE7A078F9F716FCD7E7E17810
:109A7C000BE0A178084609E0617906E0217904E061
:109A8C00E17902E0A17900E06178A078BDE8F840C6
:109A9C00F9F748BCE5886B1C19E0002940F35481A8
:109AAC00E588A0786B1CE380F9F7F6FB01462846A5
:109ABC00F9F7BCFBE378226A013BA2F11501DBB29A
:109ACC002162E370002BE8D139E1E5886B1EE3805D
:109ADC00A078F9F7E1FB01462846F9F7A7FB3DE032
:109AEC00002940F33181E588A0786B1EE380F9F7FB
:109AFC00D3FB01462846F9F799FBE378226A013B30
:109B0C00A2F11501DBB22162E370002BE8D116E162
:109B1C00E088A578431C1AE0002940F31581E08801
:109B2C00A578431CE380F9F7A7FB01462846F9F713
:109B3C00F9FBE378226A013BA2F11501DBB2216249
:109B4C00E370002BE8D1FAE0E088A578431EE380AF
:109B5C00F9F792FB01462846F9F7E4FBE378013B61
:109B6C00DBB2002BE37014BF02234223B2E00029C6
:109B7C0040F3EA80E088A578431EE380F9F77CFB8C
:109B8C0001462846F9F7CEFBE378226A013BA2F1A5
:109B9C001501DBB22162E370002BE8D1CFE0A58880
:109BAC00E0886B1CA380431C21E0002A4CDDA588B7
:109BBC00E0886B1CA380431CE380F9F75DFB014636
:109BCC002846F9F733FB6388216A013BA1F11502A2
:109BDC009BB222626380002BE7D135E00427002082
:109BEC000C280020A588E0886B1EA380431EE38010
:109BFC00F9F742FB01462846F9F718FB638894F9FC
:109C0C000020013B22F016029BB2002B638014BF94
:109C1C000423002313435DE0002A15DDA588E088AA
:109C2C006B1EA380431EE380F9F726FB01462846F2
:109C3C00F9F7FCFA6388216A013BA1F115029BB28A
:109C4C0022626380002BE7D1227802F0E9022270B5
:109C5C001BB142F00202227078E010392162F8BD8B
:109C6C00E088431C18E0002D49D0002A47DDE0882D
:109C7C00431CE380F9F700FB6788266A6378013F91
:109C8C00A6F115021D1ABFB22262EDB26780002F39
:109C9C00E9D134E0E088431EE380F9F7EDFA63780C
:109CAC00618822781D1A0139434002F00102EDB29D
:109CBC0089B242F00200274A002983EA0503525D6B
:109CCC00618003F0100342EA000214BF042100215A
:109CDC0013430B432370F8BD8DB1E088431EE38022
:109CEC00F9F7CAFA6788266A6378013FA6F115026C
:109CFC001D1ABFB22262EDB26780002FECD1227820
:109D0C004340002F02F0010283EA050342F00201F6
:109D1C00104A03F01003525D42EA010214BF042101
:109D2C00002143EA020343EA0103237000D06DB91A
:109D3C00A6F110032362F8BDA389013B08E042237E
:109D4C00103A23702262F8BD02232370A389023BD0
:109D5C00A381F8BD0C28002000234FF470428381AE
:109D6C00C380838043800380C382838243820382C7
:109D7C004381038143760376C369C28103624FF644
:109D8C00FF730385704738B5037E0D460446D9072B
:109D9C0001D4662D40D19A0123F0610302F04002F8
:109DAC0013435BB2DAB2002B227605DAA38902F0F8
:109DBC007F0201332276A381E089617B013880B276
:109DCC00E081F9F733FAE089217B013880B2E08138
:109DDC00F9F72CFA94F82A302BB1238DAB4204BF3F
:109DEC004FF6FF732385662D15D0237E5A070DD5AC
:109DFC00607EEDB245EA00252846F9F73DFA20735E
:109E0C00681C80B2F9F738FA607338BD9B0702D52D
:109E1C003823A38138BDA58138BD00002DE9F3415D
:109E2C00034D00230446034F2E46019304E000BF6C
:109E3C00A8670020F4210020A089431CA381F9F716
:109E4C001BFA226A3B5C0138D31A2362FE2802F209
:109E5C008280DFE810F04E0A860F1F0B1A0C350BB0
:109E6C00B30FF30CDF0E9A0A8E0A0B0B350C510B49
:109E7C00BA0F0C0D290E5C0A8B0F240B500C6D0BBA
:109E8C00C10FFE0C480EB90A940A100B6B0C890B0F
:109E9C00C80F1C0DFF006A0AF00F290B850CA50BCF
:109EAC00CF0F57102201D80A0710150BA10CC10BAC
:109EBC00D60F820E1301780A2F102E0BD50CF90B2E
:109ECC00E40F7B0E3101EC0A1E101A0BBB0CDD0BE0
:109EDC00DD0FBE0E8010FC0E130F2A0F410F580F12
:109EEC00900F6F0FE50E8010160F2D0F440F5B0FA8
:109EFC00950F720FE80EFF0E8010300F470F5E0F9C
:109F0C009A0F750FEB0E020F190F80104A0F610F8D
:109F1C009F0F780FEE0E050F1C0F330F8010640F80
:109F2C00A40F7B0FF10E080F1F0F360F4D0F801073
:109F3C00A90F7E0FF70E0E0F250F3C0F530F6A0F54
:109F4C009E0E810FF40E0B0F220F390F500F670F5F
:109F5C00AE0F80103903590379039903B903D90360
:109F6C001004F903370663068A06B106D806FF0605
:109F7C00420726075A047B049C04BD04E104020535
:109F8C00290523059007B807E0070B0833085B0881
:109F9C00960883087B05860591059C05A705B205E7
:109FAC00C505BD05E808F108FA0803090C091509EF
:109FBC0024091E09E105EA05F305FC0505060E0654
:109FCC001D0617063E095D097C099F09BE09DD09BE
:109FDC00000AFC097501F50D40013B0E1702B60D88
:109FEC0034042E0DC6016E0E63017110A802510EC1
:109FFC0068073F0D8901020E5B018A0E3B02C50DFD
:10A00C005105500DDA01CB0E6701940ECC027D1078
:10A01C00BE08610D9D010F0E5F0140105F02D40D53
:10A02C00D205720DEE01860A6B01D90EF002751085
:10A03C003009830DB1011C0E4901A80E8302E30DFA
:10A04C002906940D02028A0A7001AD0E14037910D0
:10A05C00260AA50D2278500604D5A3890133A381C5
:10A06C0001F079BF053BA0892362F9F705F9A389B3
:10A07C0040B201301844A08101F06DBF2278D107A5
:10A08C00EBD4053BA0892362F9F7F6F8A38940B21B
:10A09C0001301844A08101F05EBF22785206DCD555
:10A0AC00053BA0892362F9F7E7F8A38940B2013098
:10A0BC001844A08101F04FBF2278D007CDD5053BC5
:10A0CC00A0892362F9F7D8F8A38940B2013018446B
:10A0DC00A08101F040BF237813F0400F08D0A38972
:10A0EC000233A38101F037BF94F90030002BF6DB6B
:10A0FC00A089431CA381F9F7BFF82870A089F9F750
:10A10C00BBF868702B88A38101F025BF237813F06E
:10A11C00010FE3E7237813F0040FDFE7237813F044
:10A12C00400F06E0237813F0010F02E0237813F0C0
:10A13C00040FD4D0DCE794F90030002BCFDAD7E74A
:10A14C002278510601F10787E089063B2362431C04
:10A15C00E381F9F791F82073E089431CE381F9F767
:10A16C008BF8607301F0F7BE2278D20701F1F38609
:10A17C00E089063B2362431CE381F9F77DF82073E9
:10A18C00E089431CE381F9F777F8607301F0E3BED3
:10A19C002278500701F1DF86E089063B2362431CDD
:10A1AC00E381F9F769F82073E089431CE381F9F73F
:10A1BC0063F8607301F0CFBE94F90020002AC1F25D
:10A1CC00CA86E089063B2362431CE381F9F754F805
:10A1DC002073E089431CE381F9F74EF8607301F0BA
:10A1EC00BABE2278510641F1B686E089063B23625D
:10A1FC00431CE381F9F740F82073E089431CE381A9
:10A20C00F9F73AF8607301F0A6BE2278D20741F153
:10A21C00A286E089063B2362431CE381F9F72CF804
:10A22C002073E089431CE381F9F726F8607301F091
:10A23C0092BE2278500741F18E86E089063B23625C
:10A24C00431CE381F9F718F82073E089431CE38180
:10A25C00F9F712F8607301F07EBE94F90020002A21
:10A26C0081F27986E089063B2362431CE381F9F78E
:10A27C0003F82073E089431CE381F8F7FDFF60735A
:10A28C0001F069BE227851063FF529AFA089073B42
:10A29C002362431CA381F8F7EFFF2870A089431CAD
:10A2AC00A381F8F7E9FF6870E089617B013880B21F
:10A2BC00E081F8F7BBFFE089217B013880B2E081B7
:10A2CC00F8F7B4FF2B88A38101F045BE2278D207A2
:10A2DC003FF505AFA089073B2362431CA381F8F728
:10A2EC00CBFF2870A089431CA381F8F7C5FF6870C9
:10A2FC00E089617B013880B2E081F8F797FFE08953
:10A30C00217B013880B2E081F8F790FF2B88A38184
:10A31C0001F021BE227850073FF5E1AEA089073B42
:10A32C002362431CA381F8F7A7FF2870A089431C64
:10A33C00A381F8F7A1FF6870E089617B013880B2D6
:10A34C00E081F8F773FFE089217B013880B2E0816E
:10A35C00F8F76CFF2B88A38101F0FDBD94F9002068
:10A36C00002AFFF6BCAEA089073B2362431CA381E5
:10A37C00F8F782FF2870A089431CA381F8F77CFFB3
:10A38C006870E089617B013880B2E081F8F74EFF9C
:10A39C00E089217B013880B2E081F8F747FF2B88F8
:10A3AC00A38101F0D8BD227851067FF598AEA08923
:10A3BC00073B2362431CA381F8F75EFF2870A0893A
:10A3CC00431CA381F8F758FF6870E089617B013862
:10A3DC0080B2E081F8F72AFFE089217B013880B256
:10A3EC00E081F8F723FF2B88A38101F0B4BD22781C
:10A3FC00D2077FF574AEA089073B2362431CA3816F
:10A40C00F8F73AFF2870A089431CA381F8F734FFB2
:10A41C006870E089617B013880B2E081F8F706FF53
:10A42C00E089217B013880B2E081F8F7FFFE2B88B0
:10A43C00A38101F090BD227850077FF550AEA08922
:10A44C00073B2362431CA381F8F716FF2870A089F1
:10A45C00431CA381F8F710FF6870E089617B013819
:10A46C0080B2E081F8F7E2FEE089217B013880B20E
:10A47C00E081F8F7DBFE2B88A38101F06CBD94F929
:10A48C000020002ABFF62BAEA089073B2362431C99
:10A49C00A381F8F7F1FE2870A089431CA381F8F77B
:10A4AC00EBFE6870E089617B013880B2E081F8F7DF
:10A4BC00BDFEE089217B013880B2E081F8F7B6FE61
:10A4CC002B88A38101F047BD6378E278991853403B
:10A4DC00C8B22980C1F307214240607022F07F028C
:10A4EC009A43CC4A125C14BF4FF0040E4FF0000E8E
:10A4FC00114383EA000202F0100241EA02034EEA21
:10A50C000303237001F027BD6378A2789918534098
:10A51C00C8B22980C1F307214240607022F07F024B
:10A52C009A43BC4A125C14BF4FF0040E4FF0000E5D
:10A53C00114383EA000202F0100241EA02034EEAE0
:10A54C000303237001F007BD6378627999185340B7
:10A55C00C8B22980C1F307214240607022F07F020B
:10A56C009A43AC4A125C14BF4FF0040E4FF0000E2D
:10A57C00114383EA000202F0100241EA02034EEAA0
:10A58C000303237001F0E7BC6378227999185340D8
:10A59C00C8B22980C1F307214240607022F07F02CB
:10A5AC009A439C4A125C14BF4FF0040E4FF0000EFD
:10A5BC00114383EA000202F0100241EA02034EEA60
:10A5CC000303237001F0C7BC6378E27999185340F8
:10A5DC00C8B22980C1F307214240607022F07F028B
:10A5EC009A438C4A125C14BF4FF0040E4FF0000ECD
:10A5FC00114383EA000202F0100241EA02034EEA20
:10A60C000303237001F0A7BC6378A2799918534017
:10A61C00C8B22980C1F307214240607022F07F024A
:10A62C009A437C4A125C14BF4FF0040E4FF0000E9C
:10A63C00114383EA000202F0100241EA02034EEADF
:10A64C000303237001F087BC6278530003F0FE0112
:10A65C002B804A40617012F0800F01F0100242EA28
:10A66C0013236C4A14BF04200020525C1343034391
:10A67C00237001F070BCE088F8F7FEFD63781A18BF
:10A68C004340D1B22A80DBB2C2F30722484061704A
:10A69C0020EA030010F0800F5E48405C14BF4FF0BE
:10A6AC00040E4FF0000E104383EA010202F0100278
:10A6BC0040EA02034EEA0303237001F04CBCA0896C
:10A6CC00431CA381F8F7D8FD63781A184340D1B224
:10A6DC002A80DBB2C2F307224840617020EA0300F3
:10A6EC0010F0800F4B48405C14BF4FF0040E4FF03D
:10A6FC00000E104383EA010202F0100240EA02034A
:10A70C004EEA0303237001F026BC6078E278414BDB
:10A71C00811A42405FFA81FE2980C1F3072180EA49
:10A72C000E0013F80E30494284F801E0104082EA22
:10A73C000E020B4310F0800F02F0100214BF062023
:10A74C00022013430343237001F005BC6078A27808
:10A75C00304B811A42405FFA81FE2980C1F30721F8
:10A76C0080EA0E0013F80E30494284F801E01040E4
:10A77C0082EA0E020B4310F0800F02F0100214BF9D
:10A78C000620022013430343237001F0E4BB6078DE
:10A79C006279204B811A42405FFA81FE2980C1F315
:10A7AC00072180EA0E0013F80E30494284F801E0CC
:10A7BC00104082EA0E020B4310F0800F02F01002E0
:10A7CC0014BF0620022013430343237001F0C3BBC4
:10A7DC00607822790F4B811A42405FFA81FE298002
:10A7EC00C1F3072180EA0E0013F80E30494284F8B9
:10A7FC0001E0104082EA0E020B4310F0800F02F0D1
:10A80C00100214BF0620022013430343237001F0EF
:10A81C00A2BB00BF0C2800206078E279BD4B811AE6
:10A82C0042405FFA81FE2980C1F3072180EA0E00C5
:10A83C0013F80E30494284F801E0104082EA0E020F
:10A84C000B4310F0800F02F0100214BF0620022000
:10A85C0013430343237001F07EBB6078A279AD4BA8
:10A86C00811A42405FFA81FE2980C1F3072180EAF8
:10A87C000E0013F80E30494284F801E0104082EAD1
:10A88C000E020B4310F0800F02F0100214BF0620D2
:10A89C00022013430343237001F05DBB002363705C
:10A8AC004223237001F057BBE088F8F7E5FC94F8DD
:10A8BC0001E0984BC0EB0E0180EA0E025FFA81FCBE
:10A8CC002980D2B2C1F307218EEA0C0E13F80C309A
:10A8DC00494284F801C002EA0E0E82EA0C020B43D4
:10A8EC001EF0800F02F0100214BF0620022013434A
:10A8FC000343237001F02FBBA089431CA381F8F7FD
:10A90C00BBFC94F801E0834BC0EB0E0180EA0E0215
:10A91C005FFA81FC2980D2B2C1F307218EEA0C0EBA
:10A92C0013F80C30494284F801C002EA0E0E82EA98
:10A93C000C020B431EF0800F02F0100214BF062015
:10A94C00022013430343237001F005BB6278E378C4
:10A95C001340714A6370D35C43F01003237001F011
:10A96C00FABA6278A37813406B4A6370D35C43F0F5
:10A97C001003237001F0EFBA627863791340664AD2
:10A98C006370D35C43F01003237001F0E4BA627877
:10A99C0023791340604A6370D35C43F01003237037
:10A9AC0001F0D9BA6278E37913405B4A6370D35CE7
:10A9BC0043F01003237001F0CEBA6278A3791340F0
:10A9CC00554A6370D35C43F01003237001F0C3BA93
:10A9DC006378514AD35C43F01003237001F0BBBA87
:10A9EC00E088F8F749FC637818404B4B1B5C6070AF
:10A9FC0043F01003237001F0AEBAA089431CA3816D
:10AA0C00F8F73AFC63781840434B1B5C607043F0DA
:10AA1C001003237001F09FBA6278E37813433E4A27
:10AA2C006370D35C237001F096BA6278A3781343F9
:10AA3C00394A6370D35C237001F08DBA6278637904
:10AA4C001343354A6370D35C237001F084BA627887
:10AA5C0023791343304A6370D35C237001F07BBAC3
:10AA6C006278E37913432C4A6370D35C237001F052
:10AA7C0072BA6278A3791343274A6370D35C23704C
:10AA8C0001F069BA6378244AD35C237001F063BA8D
:10AA9C00E088F8F7F1FB637818431F4BC0B21B5CDE
:10AAAC006070237001F057BAA089431CA381F8F79A
:10AABC00E3FB63781843184BC0B21B5C60702370C7
:10AACC0001F049BA6278E078217801F0010E111892
:10AADC00424071445FFA81FE2980C1F3072180EA6C
:10AAEC000E0084F801E020F07F0030EA0203094BED
:10AAFC0082EA0E0213F80E3018BF042002F0100286
:10AB0C0008BF0020194341EA02030343237001F0FC
:10AB1C0022BA00BF0C280020042700206278A078FD
:10AB2C00217801F0010E1118424071445FFA81FE48
:10AB3C002980C1F3072180EA0E0084F801E020F09F
:10AB4C007F0030EA0203C84B82EA0E0213F80E3083
:10AB5C0018BF042002F0100208BF0020194341EA7C
:10AB6C0002030343237001F0F6B96278607921780F
:10AB7C0001F0010E1118424071445FFA81FE2980E8
:10AB8C00C1F3072180EA0E0084F801E020F07F0079
:10AB9C0030EA0203B44B82EA0E0213F80E3018BFEF
:10ABAC00042002F0100208BF0020194341EA0203FE
:10ABBC000343237001F0CFB962782079217801F03A
:10ABCC00010E1118424071445FFA81FE2980C1F3D5
:10ABDC00072180EA0E0084F801E020F07F0030EAC3
:10ABEC000203A14B82EA0E0213F80E3018BF0420A8
:10ABFC0002F0100208BF0020194341EA020303438C
:10AC0C00237001F0A8B96278E079217801F0010E87
:10AC1C001118424071445FFA81FE2980C1F307216B
:10AC2C0080EA0E0084F801E020F07F0030EA020395
:10AC3C008D4B82EA0E0213F80E3018BF042002F07E
:10AC4C00100208BF0020194341EA0203034323709A
:10AC5C0001F081B96278A079217801F0010E111808
:10AC6C00424071445FFA81FE2980C1F3072180EADA
:10AC7C000E0084F801E020F07F0030EA02037A4BEA
:10AC8C0082EA0E0213F80E3018BF042002F01002F4
:10AC9C0008BF0020194341EA02030343237001F06B
:10ACAC005AB92378627803F0010303EB4203D9B25B
:10ACBC002B80C3F307234A40617012F0800F01F020
:10ACCC00100243EA0203684A14BF04200020525CBD
:10ACDC0013430343237001F03EB9E088F8F7CCFA34
:10ACEC002278637802F001021A4443400244DBB23A
:10ACFC00D1B22A80C2F307224840617020EA0300D7
:10AD0C004B4010F0800F584803F01003405C14BF08
:10AD1C004FF0040E4FF0000E02431A434EEA0202AB
:10AD2C00227001F018B9A089431CA381F8F7A4FA8A
:10AD3C002278637802F001021A4443400244DBB2E9
:10AD4C00D1B22A80C2F307224840617020EA030086
:10AD5C004B4010F0800F444803F01003405C14BFCC
:10AD6C004FF0040E4FF0000E02431A434EEA02025B
:10AD7C00227001F0F0B894F801E0E2782178C2EB8F
:10AD8C000E00394B01F001018EEA0202411AC8B2E1
:10AD9C002980C1F307218EEA000E1B5C49426070CA
:10ADAC0002EA0E0E42400B431EF0800F02F010021E
:10ADBC0014BF4FF0060E4FF0020E13434EEA03037E
:10ADCC00237001F0C8B894F801E0A2782178C2EBA6
:10ADDC000E00254B01F001018EEA0202411AC8B2A5
:10ADEC002980C1F307218EEA000E1B5C494260707A
:10ADFC0002EA0E0E42400B431EF0800F02F01002CE
:10AE0C0014BF4FF0060E4FF0020E13434EEA03032D
:10AE1C00237001F0A0B894F801E062792178C2EBBC
:10AE2C000E00114B01F001018EEA0202411AC8B268
:10AE3C002980C1F307218EEA000E1B5C4942607029
:10AE4C0002EA0E0E42400B431EF0800F02F010027D
:10AE5C0014BF4FF0060E4FF0020E13434EEA0303DD
:10AE6C00237001F078B800BF0C28002094F801E0A2
:10AE7C0022792178C2EB0E00C44B01F001018EEA5D
:10AE8C000202411AC8B22980C1F307218EEA000ED2
:10AE9C001B5C4942607002EA0E0E42400B431EF0EE
:10AEAC00800F02F0100214BF4FF0060E4FF0020E8E
:10AEBC0013434EEA0303237001F04DB894F801E0FC
:10AECC00E2792178C2EB0E00B04B01F001018EEA61
:10AEDC000202411AC8B22980C1F307218EEA000E82
:10AEEC001B5C4942607002EA0E0E42400B431EF09E
:10AEFC00800F02F0100214BF4FF0060E4FF0020E3E
:10AF0C0013434EEA0303237001F025B894F801E0D3
:10AF1C00A2792178C2EB0E009C4B01F001018EEA64
:10AF2C000202411AC8B22980C1F307218EEA000E31
:10AF3C001B5C4942607002EA0E0E42400B431EF04D
:10AF4C00800F02F0100214BF4FF0060E4FF0020EED
:10AF5C0013434EEA0303237000F0FDBF237843F341
:10AF6C000003D9B22B801B0E01F0100261705B4202
:10AF7C001343864A43F00203525C1343237000F0E0
:10AF8C00EABFE088F8F778F9617823780A1A484024
:10AF9C0003F00103C0B2D31ADAB22B80C3F3072338
:10AFAC00514062705B42014011F0800F7749895C1F
:10AFBC0014BF4FF0060E4FF0020E194380EA020345
:10AFCC0003F0100341EA03004EEA0000207000F089
:10AFDC00C2BFA089431CA381F8F74EF9617823788E
:10AFEC000A1A484003F00103C0B2D31ADAB22B801C
:10AFFC00C3F30723514062705B42014011F0800F94
:10B00C006249895C14BF4FF0060E4FF0020E1943D3
:10B01C0080EA020303F0100341EA03004EEA000049
:10B02C00207000F098BF6278E3785340584A637000
:10B03C00D35C237000F08FBF6278A3785340544ADE
:10B04C006370D35C237000F086BF627863795340E1
:10B05C004F4A6370D35C237000F07DBF6278237914
:10B06C0053404B4A6370D35C237000F074BF62781A
:10B07C00E3795340464A6370D35C237000F06BBF96
:10B08C006278A3795340424A6370D35C237000F01A
:10B09C0062BF002363704423237000F05CBFE08820
:10B0AC00F8F7EAF863785840394BC0B21B5C607013
:10B0BC00237000F050BFA089431CA381F8F7DCF883
:10B0CC0063785840324BC0B21B5C6070237000F048
:10B0DC0042BF6078E2782D4B811A42405FFA81FEC4
:10B0EC002980C1F3072180EA0E0013F80E30494283
:10B0FC00104082EA0E020B4310F0800F02F0100297
:10B10C0014BF0620022013430343237000F023BF17
:10B11C006078A2781D4B811A42405FFA81FE29802B
:10B12C00C1F3072180EA0E0013F80E30494210409B
:10B13C0082EA0E020B4310F0800F02F0100214BFD3
:10B14C000620022013430343237000F004BF6078F1
:10B15C0062790E4B811A42405FFA81FE2980C1F35D
:10B16C00072180EA0E0013F80E304942104082EAA3
:10B17C000E020B4310F0800F02F0100214BF0620D9
:10B18C00022013430343237000F0E5BE0C2800207B
:10B19C000427002060782279C84B811A42405FFA5C
:10B1AC0081FE2980C1F3072180EA0E0013F80E30CE
:10B1BC004942104082EA0E020B4310F0800F02F05D
:10B1CC00100214BF0620022013430343237000F027
:10B1DC00C2BE6078E279B94B811A42405FFA81FEB7
:10B1EC002980C1F3072180EA0E0013F80E30494282
:10B1FC00104082EA0E020B4310F0800F02F0100296
:10B20C0014BF0620022013430343237000F0A3BE97
:10B21C006078A279A94B811A42405FFA81FE29809D
:10B22C00C1F3072180EA0E0013F80E30494210409A
:10B23C0082EA0E020B4310F0800F02F0100214BFD2
:10B24C000620022013430343237000F084BE4223E4
:10B25C00237000F080BEE088F8F70EF894F801E057
:10B26C00964BC0EB0E0180EA0E005FFA81FC298040
:10B27C00C2B2C1F307218EEA0C0E13F80C3049420E
:10B28C0002EA0E0E82EA0C020B431EF0800F02F053
:10B29C00100214BF0620022013430343237000F056
:10B2AC005ABEA089431CA381F7F7E6FF94F801E08E
:10B2BC00824BC0EB0E0180EA0E005FFA81FC298004
:10B2CC00C2B2C1F307218EEA0C0E13F80C304942BE
:10B2DC0002EA0E0E82EA0C020B431EF0800F02F003
:10B2EC00100214BF0620022013430343237000F006
:10B2FC0032BEA089431CA381F7F7BEFFA070A089C2
:10B30C00431CA381F7F7B8FFE07000F024BEA089BE
:10B31C00431CA381F7F7B0FF2071A089431CA381C4
:10B32C00F7F7AAFF607100F016BEA089431CA38139
:10B33C00F7F7A2FFA071A089431CA381F7F79CFF2C
:10B34C00E07100F008BEA089431CA381F7F794FFBD
:10B35C00A073A089431CA381F7F78EFFE07300F064
:10B36C00FABDE388A38100F0F6BDE388E38100F029
:10B37C00F2BD6088F7F780FF607000F0ECBDA0882C
:10B38C00F7F77AFF607000F0E6BDB4F806E062886B
:10B39C0094F900000EEB02038EEA020220F0130077
:10B3AC0099B24A402980E18012F4805FC3F30042D5
:10B3BC0014BF4FF0100E4FF0000E40EA02034EEA9D
:10B3CC000303237000F0C7BDB4F806E0A28894F91B
:10B3DC0000000EEB02038EEA020220F0130099B279
:10B3EC004A402980E18012F4805FC3F3004214BF0D
:10B3FC004FF0100E4FF0000E40EA02034EEA03032A
:10B40C00237000F0A8BDE38894F900205B0022F0C3
:10B41C00130299B242EA134311F4805F2980E18050
:10B42C0014BF102000200343237000F094BDB4F827
:10B43C0006E0E28994F900000EEB02038EEA0202A8
:10B44C0020F0130099B24A402980E18012F4805F09
:10B45C00C3F3004214BF4FF0100E4FF0000E40EA41
:10B46C0002034EEA0303237000F075BD6388013BB1
:10B47C00638000F070BDA388013BA38000F06BBD1E
:10B48C00E388013BE38000F066BDE389013BE38187
:10B49C0000F061BD63880133638000F05CBDA3885C
:10B4AC000133A38000F057BDE3880133E38000F043
:10B4BC0052BDE3890133E38100F04DBD0C2800201F
:10B4CC00E17822780139B34B02F00102C9B242F0A3
:10B4DC000202585C7F29E17001F00F010CBF0423BC
:10B4EC00002302430F2943EA02030CBF1021002161
:10B4FC000B43237000F02FBDA17822780139A54BA6
:10B50C0002F00102C9B242F00202585C7F29A1701C
:10B51C0001F00F010CBF0423002302430F2943EA5F
:10B52C0002030CBF102100210B43237000F013BD4C
:10B53C00617922780139974B02F00102C9B242F0CD
:10B54C000202585C7F29617101F00F010CBF0423CA
:10B55C00002302430F2943EA02030CBF10210021F0
:10B56C000B43237000F0F7BC217922780139894B09
:10B57C0002F00102C9B242F00202585C7F2921712B
:10B58C0001F00F010CBF0423002302430F2943EAEF
:10B59C0002030CBF102100210B43237000F0DBBC15
:10B5AC00E179227801397B4B02F00102C9B242F0F9
:10B5BC000202585C7F29E17101F00F010CBF0423DA
:10B5CC00002302430F2943EA02030CBF1021002180
:10B5DC000B43237000F0BFBCA179227801396D4B6D
:10B5EC0002F00102C9B242F00202585C7F29A1713B
:10B5FC0001F00F010CBF0423002302430F2943EA7F
:10B60C0002030CBF102100210B43237000F0A3BCDC
:10B61C006178227801395F4B02F00102C9B242F025
:10B62C000202585C7F29617001F00F010CBF0423EA
:10B63C00002302430F2943EA02030CBF102100210F
:10B64C000B43237000F087BCE088F7F715FE2278D7
:10B65C000138504B02F00102C1B242F00202585CB8
:10B66C007F2942EA000201F00F000CBF04230023E3
:10B67C000F2843EA02030CBF102000200343E0888C
:10B68C002370F7F7D3FD00F066BCE1782378013125
:10B69C00404A03F00103C9B2525C8029E17043EACD
:10B6AC0002030CBF0422002211F00F0F5BB243EA1D
:10B6BC00020314BF002210221343237000F04BBC72
:10B6CC00A17823780131334A03F00103C9B2525CEB
:10B6DC008029A17043EA02030CBF0422002211F05E
:10B6EC000F0F5BB243EA020314BF00221022134374
:10B6FC00237000F030BC617923780131254A03F0C6
:10B70C000103C9B2525C8029617143EA02030CBF88
:10B71C000422002211F00F0F5BB243EA020314BFA4
:10B72C00002210221343237000F015BC21792378DA
:10B73C000131184A03F00103C9B2525C802921710E
:10B74C0043EA02030CBF0422002211F00F0F5BB27C
:10B75C0043EA020314BF0022102213432370FAE3BE
:10B76C00E179237801310B4A03F00103C9B2525C31
:10B77C008029E17143EA02030CBF0422002211F07C
:10B78C000F0F5BB243EA020314BF002210221343D3
:10B79C002370E0E30C280020A17923780131A74A1B
:10B7AC0003F00103C9B2525C8029A17143EA020380
:10B7BC000CBF0422002211F00F0F5BB243EA02030C
:10B7CC0014BF0022102213432370C4E36178237842
:10B7DC0001319A4A03F00103C9B2525C80296170AD
:10B7EC0043EA02030CBF0422002211F00F0F5BB2DC
:10B7FC0043EA020314BF0022102213432370AAE36E
:10B80C00E088F7F739FD01302378C1B28B4A03F099
:10B81C000103E088525C802943EA02030CBF042236
:10B82C00002211F00F0F5BB243EA020314BF002297
:10B83C00102213432370F7F7F9FC8CE3627823781A
:10B84C00D10923F0130341EA42020B4362702370C7
:10B85C0081E394F90030617803F0010223F01303C3
:10B86C0042EA410243EAD1136270237073E36178B8
:10B87C0011F0010214BF6FF07F03002343EA510360
:10B88C006370237823F013031343237063E323784B
:10B89C00607813F0010F23F0130300F0010214BFC2
:10B8AC006FF07F010021134341EA50012370617056
:10B8BC0051E3E089617B013880B2E081F7F7B6FC97
:10B8CC00E089217B013880B2E081F7F7AFFC0023DF
:10B8DC00A38140E3E089617B013880B2E081F7F716
:10B8EC00A5FCE089217B013880B2E081F7F79EFC52
:10B8FC000823A3812FE3E089617B013880B2E081CA
:10B90C00F7F794FCE089217B013880B2E081F7F7EE
:10B91C008DFC1023A3811EE3E089617B013880B28A
:10B92C00E081F7F783FCE089217B013880B2E0816C
:10B93C00F7F77CFC1823A3810DE3E089617B0138C8
:10B94C0080B2E081F7F772FCE089217B013880B28C
:10B95C00E081F7F76BFC2023A381FCE2E089617B9B
:10B96C00013880B2E081F7F761FCE089217B013876
:10B97C0080B2E081F7F75AFC2823A381EBE2E0893F
:10B98C00617B013880B2E081F7F750FCE089217BC4
:10B99C00013880B2E081F7F749FC3023A381DAE269
:10B9AC00E089617B013880B2E081F7F73FFCE089E8
:10B9BC00217B013880B2E081F7F738FC3823A38172
:10B9CC00C9E2E089E178013880B2E081F7F72EFC1A
:10B9DC00E089A178013880B2E081F7F727FCBAE260
:10B9EC00E0896179013880B2E081F7F71FFCE089CA
:10B9FC002179013880B2E081F7F718FCABE2E089DD
:10BA0C00E179013880B2E081F7F710FCE089A17987
:10BA1C00013880B2E081F7F709FC9CE2E08961789B
:10BA2C00013880B2E081F7F701FCE0892178013818
:10BA3C0080B2E081F7F7FAFB8DE200BF0C28002002
:10BA4C00E089431CE381F7F717FCA070E089431CE5
:10BA5C00E381F7F711FCE0707DE2E089431CE381A0
:10BA6C00F7F70AFC2071E089431CE381F7F704FC2B
:10BA7C00607170E2E089431CE381F7F7FDFBA07174
:10BA8C00E089431CE381F7F7F7FBE07163E2E0899F
:10BA9C00431CE381F7F7F0FB2070E089431CE38142
:10BAAC00F7F7EAFB607056E2E378013BDBB2E37038
:10BABC0043B1A089F7F7E0FBA38940B201301844E9
:10BACC00A08148E2A3890133A38144E2A089431CED
:10BADC00A381F7F7D1FB2870A089F7F7CDFB68702D
:10BAEC002B88A38137E2A089F7F7C6FBA38940B264
:10BAFC0001301844A0812EE2A089431CA381F7F7E2
:10BB0C00BBFB2870A089431CA381F7F7B5FB6870B9
:10BB1C00E089617B013880B2E081F7F787FBE0892F
:10BB2C00217B013880B2E081F7F780FB2B88A38161
:10BB3C0011E2E089431CE381F7F79EFB2073E08957
:10BB4C00431CE381F7F798FB607304E2237823F03E
:10BB5C00120343F001032370FDE16378DB43637050
:10BB6C00237843F012032370F5E1A089431CA381D1
:10BB7C00F7F782FB617880B2F7F7D4FBEBE1A08991
:10BB8C00431CA381F7F778FB80B2F7F785FB607055
:10BB9C00E1E1A389013BA381237E63F07F0323763C
:10BBAC0000232362D7E1237E23F001032376D2E125
:10BBBC00227E208D42F0010121764FF6FF718842E2
:10BBCC0000F0C98142F021026362012322762362D4
:10BBDC00C1E1237883F0010313F0010F23F012026B
:10BBEC0014BF0023102313432370B4E16388628ACB
:10BBFC0063826280A388A28AA382A280E388E28AFD
:10BC0C002B80E280E382A6E1A388E2882B80A280CD
:10BC1C00E380A0E12388228A2B80228023829AE170
:10BC2C00E378A37097E1E378637194E1E37823718F
:10BC3C0091E1E378E3718EE1E378A3718BE1E37832
:10BC4C00637088E1E178E088F7F7F0FA83E1A37894
:10BC5C00E37080E1A37863717DE1A37823717AE1CD
:10BC6C00A378E37177E1A378A37174E1A37863708F
:10BC7C0071E1A178E088F7F7D9FA6CE16379E370A8
:10BC8C0069E16379A37066E16379237163E1637998
:10BC9C00E37160E16379A3715DE1637963705AE1EB
:10BCAC006179E088F7F7C2FA55E12379E37052E144
:10BCBC002379A3704FE1237963714CE12379E3710C
:10BCCC0049E12379A37146E12379637043E121793A
:10BCDC00E088F7F7ABFA3EE1E379E3703BE1E37917
:10BCEC00A37038E1E379637135E1E379237132E1D3
:10BCFC00E379A3712FE1E37963702CE1E179E088BA
:10BD0C00F7F794FA27E1A379E37024E1A379A37000
:10BD1C0021E1A37963711EE1A37923711BE1A3795E
:10BD2C00E37118E1A379637015E1A179E088F7F765
:10BD3C007DFA10E16378E3700DE16378A3700AE19A
:10BD4C006378637107E16378237104E16378E371CD
:10BD5C0001E16378A371FEE06178E088F7F766FA99
:10BD6C00F9E061786088F7F761FAF4E06178A0880F
:10BD7C00F7F75CFAEFE0E088F7F77EFAE070EAE0BC
:10BD8C00E088F7F779FAA070E5E0E088F7F774FA45
:10BD9C006071E0E0E088F7F76FFA2071DBE0E08893
:10BDAC00F7F76AFAE071D6E0E088F7F765FAA07168
:10BDBC00D1E0E088F7F760FA6070CCE0A089431C12
:10BDCC00A381F7F759FAE070C5E0A089431CA38161
:10BDDC00F7F752FAA070BEE0A089431CA381F7F7D5
:10BDEC004BFA6071B7E0A089431CA381F7F744FAC2
:10BDFC002071B0E0A089431CA381F7F73DFAE071F4
:10BE0C00A9E0A089431CA381F7F736FAA071A2E040
:10BE1C00A089431CA381F7F72FFA60709BE0A089DF
:10BE2C00B4F80680431CA381F7F726FA0146404676
:10BE3C00F7F7FCF98FE0A089431CA381F7F71CFAF4
:10BE4C002870A089431CA381F7F716FA687028881C
:10BE5C00A179431C2B80F7F7E9F9E1792888F7F7EA
:10BE6C00E5F978E0A089431CA381F7F705FA28705F
:10BE7C00A089431CA381F7F7FFF968702888431C3D
:10BE8C002B80F7F7F9F9A0712888F7F7F5F9E0712D
:10BE9C0061E0A089431CA381F7F7EEF92870A08913
:10BEAC00431CA381F7F7E8F968702888F7F7E4F9E1
:10BEBC00607050E0A089431CA381F7F7DDF928706E
:10BECC00A089431CA381F7F7D7F96178687028889B
:10BEDC00F7F7ACF93FE0E089F7F7CEF92870E08985
:10BEEC00A179431CE381F7F7A1F9E089F7F7C4F9CD
:10BEFC006870E089E179431EE381F7F797F92B88A5
:10BF0C00E38028E022786378D1072B8044BF43F488
:10BF1C0080732B80D30642BF338843F40073338085
:10BF2C00900742BF338843F4806333801F4B3288C1
:10BF3C0033F8123023800EE02046F7F757FD0AE065
:10BF4C002046FDF783FA06E02046F9F763F802E095
:10BF5C002046FBF76DF9226A002A1FDC237E990626
:10BF6C0009D5218D23F020032980616A23760139BC
:10BF7C000A44226206E001A92046F7F7E3FAE369D6
:10BF8C002880236229884FF6FE7399420AD04FF617
:10BF9C00FF73994202D02046FDF7F5FE019B012B61
:10BFAC007DF44AAFA08902B0BDE8F081180B0020E7
:10BFBC000122014B1A707047AD720020052910B593
:10BFCC0006DC0C240348521004FB01018B604A6010
:10BFDC0010BD00BF2C6600200020704770477047D2
:10BFEC007047012070477047006910B10368DB6827
:10BFFC0018477047006910B103681B6918477047F0
:10C00C00006910B103685B6918474FF0FF30704747
:10C01C00006910B103689B691847704707B5006940
:10C02C0010B94FF0FF3009E0036801220DF1070150
:10C03C009B6898470028F4D09DF8070003B05DF882
:10C04C0004FB07B500698DF8071028B103680122BD
:10C05C000DF10701DB68984703B05DF804FB0000A5
:10C06C00314B012201461A70304B93F86E00402878
:10C07C0020D13D291BD007DC242916D0262918D025
:10C08C00222908BF232115E0E0290CD003DCA729C5
:10C09C0008BF5E210EE0E72903D0E92908BF402143
:10C0AC0008E07B2106E07D2104E05D2102E07E2199
:10C0BC0000E07C211E4B1B78002B32D0D72920D0DE
:10C0CC000ADC0A2922D0202925D009292BD1194A8A
:10C0DC00137823F0400322E0D92903D00CDBDA29B2
:10C0EC0005D07047134A137823F0080317E0114A60
:10C0FC00137823F0040312E00E4A137823F00203A2
:10C10C000DE00C4A137823F0010308E0094A137878
:10C11C0023F0100303E0074A137823F02003137075
:10C12C007047F6F715BF704718680020A04D002027
:10C13C004B3100209A720020314B012201461A70BB
:10C14C00304B93F86E00402820D13D291BD007DCE2
:10C15C00242916D0262918D0222908BF232115E01E
:10C16C00E0290CD003DCA72908BF5E210EE0E729EB
:10C17C0003D0E92908BF402108E07B2106E07D219E
:10C18C0004E05D2102E07E2100E07C211E4B1B7847
:10C19C00002B32D0D72920D00ADC0A2922D0202922
:10C1AC0025D009292BD1194A137843F0400322E0FA
:10C1BC00D92903D00CDBDA2905D07047134A137840
:10C1CC0043F0080317E0114A137843F0040312E01C
:10C1DC000E4A137843F002030DE00C4A137843F037
:10C1EC00010308E0094A137843F0100303E0074AFF
:10C1FC00137843F0200313707047F6F79BBE70471B
:10C20C0018680020A04D00204B3100209A720020AD
:10C21C0013B50346006D0C4628B10DF1060201A9B9
:10C22C0007F0CFFF08E0586D08B9002021E00DF1B0
:10C23C00060201A905F056FE0028F6D0BDF8043020
:10C24C00BDF806200BB9002AEFD002F01F014900FF
:10C25C002170C2F34511D2126170A27003F01F025B
:10C26C002271C3F343125B12013A03F5EA63627164
:10C27C00A37102B010BD13B50346006D0C4628B176
:10C28C000DF1060201A907F0ACFF08E0586D08B9E2
:10C29C00002021E00DF1060201A905F033FE002873
:10C2AC00F6D0BDF80430BDF806200BB9002AEFD04B
:10C2BC0002F01F0149002170C2F34511D2126170C6
:10C2CC00A27003F01F022271C3F343125B12013AF6
:10C2DC0003F5EA636271A37102B010BD38B5856DC8
:10C2EC000446BDB94FF480700DF04CFA0146A065C0
:10C2FC0070B10570206D20B14FF4807209F04AF9CD
:10C30C0008E0606D30B14FF4807207F045F901E040
:10C31C00014BA365A06D38BDA0720020D0B5046D93
:10C32C006CB1012B08BF002A14D21146204607F02D
:10C33C0060FD78B1204608F061F958B1D0BD446D6C
:10C34C0044B1204605F017FF20B12046BDE8D0408F
:10C35C0006F0DCBC0020D0BD10B504460068436874
:10C36C00013B43603BB90368DB6A9847206810B116
:10C37C0003685B6898470023236010BD054B10B51C
:10C38C0003600446036913B11030FFF7E5FF204644
:10C39C0010BD00BFE404002010B50446FFF7EEFF0B
:10C3AC00142120460CF0F0FE204610BD10B5084CB0
:10C3BC0004F13C00FFF7E2FF04F12800FFF7DEFF79
:10C3CC0004F11400FFF7DAFF2046FFF7D7FF10BD8A
:10C3DC001430002010B103689B681847704738B5BB
:10C3EC000B6804460D4613B15A6801325A60236932
:10C3FC001BB104F11000FFF7AFFF2B68204623613F
:10C40C0038BD10B103681B6B1847704710B1036837
:10C41C009B6A1847002000217047036D13B15869BF
:10C42C0000217047436D13B193E803007047184621
:10C43C00F6E7036D13B1D86900217047436D13B152
:10C44C001869596970471846F6E770B504460846EE
:10C45C000D460DF004FB23680246294620465B6816
:10C46C00BDE87040184738B50546FFF7EEFF0446A7
:10C47C0028460CF083FD204438BD38B505460CF039
:10C48C00DCFD044628460CF079FD204438BD826B57
:10C49C0030B562B1137803F0080303F0FF00FBB171
:10C4AC00D3695069181A1BD56FF0004018E0C06BA7
:10C4BC00B0B190F831301B0707D5D0E90445D0E96D
:10C4CC000023A01A65EB030101E0002000210023EA
:10C4DC006FF000428B4208BF824201D2104630BD41
:10C4EC0030BD08B51030FFF7D2FF08BD08B51830C5
:10C4FC00FFF7CDFF08BD836B1BB11B7813F0700FDA
:10C50C0005E0C06B30B190F8313013F0500F14BF10
:10C51C0001200020704708B51830FFF7ECFF08BD6C
:10C52C0010B504461830FFF7E6FF60B1206D10B16E
:10C53C00002107F05EFC606D28B100220023BDE8ED
:10C54C00104005F018BE10BD836B23B9C06B0030D2
:10C55C0018BF012070470120704708B51830FFF74D
:10C56C00F3FF08BD10B50446806D18B10DF012F93B
:10C57C000023A36518342046FFF7E6FF20B12046C0
:10C58C00BDE8104009F0EFB910BD0000064B10B526
:10C59C0003600446FFF7E6FF044B04F11800A360A8
:10C5AC0009F0E1F9204610BD340500208403002079
:10C5BC0010B50446FFF7EAFF5C2120460CF0E4FDC1
:10C5CC00204610BD0346806B08B107F0E2BBD86B68
:10C5DC0008B105F0BBBD4FF0FF30704708B5103007
:10C5EC00FFF7F0FF08BD08B51830FFF7EBFF08BDEB
:10C5FC000346806B08B107F011BBD86B08B105F08E
:10C60C00E3BC4FF0FF30704707B501220DF1070175
:10C61C001030FFF7EDFF01280CBF9DF807004FF01D
:10C62C00FF3003B05DF804FB08B51830FFF7E0FFEE
:10C63C0008BDD0B4846B44B1012B08BF002A09D2C9
:10C64C0020461146D0BC07F0D4BBC06B10B1D0BC97
:10C65C0005F091BD0020D0BC704738B50146049858
:10C66C0014461D4610B901F118001DE001280AD12D
:10C67C000B6D01F118000BB15A6912E04B6D7BB1D7
:10C68C00D3E900230EE0022811D10B6D01F1180043
:10C69C000BB1DA6905E04B6D13B1D3E9042301E06A
:10C6AC000022002312196B41FFF7C3FF38BD002095
:10C6BC0038BD0346806B08B107F0C6BCD86B08B117
:10C6CC0006F034B9704708B51030FFF7F2FF08BD1B
:10C6DC0008B51830FFF7EDFF08BDF0B5D0F838E01D
:10C6EC009DF814409DF818509DF81C609DF8207022
:10C6FC00BEF1000F08D00897704607960695059472
:10C70C00BDE8F04007F023BFC06B38B1089707961F
:10C71C0006950594BDE8F04006F06EBAF0BD1FB565
:10C72C008A79A2F150031B0611D40C7802F26C72B8
:10C73C004B79183003944C7801330294DBB28C782B
:10C74C000194097900910421FFF7C7FF00E0002054
:10C75C0004B010BD1FB58A79A2F150031B0611D489
:10C76C000C7802F26C724B79183003944C780133CC
:10C77C000294DBB28C780194097900910221FFF7C5
:10C78C00ACFF00E0002004B010BD0346806B08B184
:10C79C0007F068BFD86B08B106F018BB704708B536
:10C7AC001830FFF7F2FF08BD08B51030FFF7EDFFAA
:10C7BC0008BD07B502AB0122103003F8011D194664
:10C7CC00FFF7E3FF03B05DF804FB000000234FF418
:10C7DC007A7203710373054B826003600B6903610A
:10C7EC0013B15A6801325A60704700BFE40400204C
:10C7FC0010B50446006940B10368DB6A984704F140
:10C80C001000BDE81040FFF7A7BD10BD38B50025DE
:10C81C000E4B044610314560183040F8183C11F8A6
:10C82C000C3C00F80C3C0A4B40F8103C51F8083C0E
:10C83C0040F8083C11F8043C00F8043C09F062F89C
:10C84C00044BA5652046A36038BD00BF340500200D
:10C85C0090050020100500202DE9F04395B000252F
:10C86C001C4B4FF47A760DF150082A4618310446C9
:10C87C0004A848F8503D8DF8045002968DF80C50E1
:10C88C001295139509F0C2F804A8DFF85090FFF741
:10C89C005BFE80B15C200CF075FC07464146FFF74F
:10C8AC00B5FF7B6825710133A6602573C4F8009031
:10C8BC0027617B6005E02071A6602073C4F80090AE
:10C8CC002061054B04A8009309F04DF8204615B0E3
:10C8DC00BDE8F0831005002084030020E404002050
:10C8EC00012B70B5044694B005D0022B40F2022304
:10C8FC0018BF002301E044F202230431684609F01A
:10C90C0015F904A8FFF720FE114E90B15C200CF035
:10C91C0039FC69460546FFF779FF00234FF47A721C
:10C92C002660237123736B68A260013325616B60F1
:10C93C0006E04FF47A7320712073A36026602061A7
:10C94C00044B04A8009309F00EF8204614B070BDF7
:10C95C00E40400208403002070B5324B8AB000241C
:10C96C00314A00934FF47A73304905A80293234659
:10C97C008DF804408DF80C400494FFF7B1FF2C4E59
:10C98C0009A92B48FFF72BFD05A8FFF7F7FC316928
:10C99C0029B10B68002205A8DB6B984703E02449FA
:10C9AC0005A8FFF713FF09A96846FFF718FD05A8AE
:10C9BC00FFF7E4FC0498FFF724FD48B3049820B17A
:10C9CC0003685B6B9847054600E01A4D29461A48E8
:10C9DC00FFF749FD049868B103689B6B984748B111
:10C9EC00164928460DF029F868B1154928460DF06E
:10C9FC0024F840B1134B22202122294600FB04309D
:10CA0C0001340DF049F86846FFF7F2FE3F2CBEDD0D
:10CA1C000748FFF7EDFE6846FFF7B0FC20460AB06A
:10CA2C0070BD00BFE40400205A720020F0600020AA
:10CA3C0068300020D32E0020003000203D2900203B
:10CA4C003C2900209E6900200146024808B5FFF7EA
:10CA5C000AFD08BD003000200146024808B5FFF76A
:10CA6C000CFD08BD0030002038B504460CF08AFEE1
:10CA7C000546A8B90E48FFF7E7FF2046FFF7ECFF85
:10CA8C000C48FFF7E1FF0C4B1A6814440F2C03D829
:10CA9C000A4D1C60154409E00948FFF7D5FF05E075
:10CAAC000848FFF7D1FF2046FFF7D6FF284638BDD0
:10CABC00802A0020942A0020B466002041720020B5
:10CACC009D2A0020B12A0020044B28B91A780AB1FB
:10CADC00187001E001221A70187870470F68002056
:10CAEC00014B1888704700BFAA6700202DE9F04F52
:10CAFC00232085B00BF014F800284FF0240014BF4D
:10CB0C00002404240BF00CF810B944F00804A4B26F
:10CB1C0026200BF005F810B944F00104A4B225202E
:10CB2C000AF0FEFF10B944F00204A4B222200AF06D
:10CB3C00F7FF10B944F01004A4B2A04B1B780BB94A
:10CB4C002402A4B29E4B1B785E0744BF44F004043D
:10CB5C00A4B21D0744BF44F00804A4B298074FF0D8
:10CB6C00290044BF44F00204A4B2D90744BF44F0E6
:10CB7C000104A4B2DA0644BF44F01004A4B29F0628
:10CB8C0044BF44F02004A4B25E0644BF44F0400409
:10CB9C00A4B20AF0C5FF10B944F02004A4B22820B6
:10CBAC000AF0BEFF10B944F04004A4B2854A4FF01D
:10CBBC00FF33854D002710680DF1040B2B6001AB82
:10CBCC005168DFF808A203C3906818601BF817605F
:10CBDC00012130460AF0B6FF002130460AF080FFF2
:10CBEC0013200AF09DFFB0FA80F812200AF098FF8B
:10CBFC0000284FEA58184FF0110014BF00230223ED
:10CC0C0048EA03080AF08CFF00284FF0050014BF17
:10CC1C000023042348EA03080AF082FF00284FF09F
:10CC2C001D0014BF0023082348EA03080AF078FF0C
:10CC3C0000284FF01E0014BF0023102348EA0308FD
:10CC4C000AF06EFF00284FF0200014BF00232023B1
:10CC5C0048EA03090AF064FF00284FF0010130464E
:10CC6C0014BF4FF000084FF040080AF039FF30466F
:10CC7C0049EA080805210AF065FF544E0AF80780B6
:10CC8C000137062FA2D1737903F0080202F0FF01DD
:10CC9C001AB123F0080301217371727902F01000AC
:10CCAC0000F0FF0320B1494B22F010025A7101230E
:10CCBC000027D5F800E03846325C002A18BF8646BB
:10CCCC0000F1010018BF01270628F5D10FB1C5F8F6
:10CCDC0000E0550644BF44F00204A4B2900644BFE1
:10CCEC0044F00104A4B2D707394F48BF44F00804FC
:10CCFC00BE4648BFA4B25507364D44BF44F00404A9
:10CD0C00A4B2900738682A6848BF44F01004A0EB1E
:10CD1C00020248BFA4B2642A07D92F4A28601578AA
:10CD2C000DB9012500E0002515702C4D2C4F2D4A16
:10CD3C0013B101232B703CE02B70002938D097F8ED
:10CD4C0000C02949BCF1000F1BD1D1F800E0BEF1A5
:10CD5C00000F03D1254B1860012325E00EF1010EC5
:10CD6C00BEF1010FC1F800E01FD90B601F49096823
:10CD7C00401AB0F5FA7F18D2117801B9012313705B
:10CD8C0013E00868012810D1DEF80000DFF85CE041
:10CD9C00DEF800E0CEEB0000B0F57A7F05D9107814
:10CDAC00B0FA80F0400910700B6001233B7000E07A
:10CDBC0039701378E3B1084B19781EE00F68002026
:10CDCC009A7200200C0B002064300020537200205B
:10CDDC009C670020B8660020176800204072002075
:10CDEC003F7200201568002004660020D8650020E2
:10CDFC003B780BB9297801B101210E200AF070FEA5
:10CE0C003B78002B3AD0327944F04003102A9BB285
:10CE1C0002D144F06004A3B22A78002A2DD0194B19
:10CE2C009C6BDA6C42F00102DA649A6B22F002021B
:10CE3C009A639A6B9207FCD472B61248036D426DDA
:10CE4C00466D1049B242056DF8D1AB42F6D1D20B0A
:10CE5C0042EA434302338B658A6D0A489342FBD105
:10CE6C0044F002038363836B064A9B07FBD5936BE9
:10CE7C0043F04003936330BFFDE71C46204605B0EA
:10CE8C00BDE8F08F00400D4008B5FFF72FFE034AB8
:10CE9C001388108020EA030398B208BDAA6700200B
:10CEAC001B4B1C4A197812781B4B30B549B10AB18F
:10CEBC001A4A0FE01A4A12780AB11A4A0AE01A4AB8
:10CECC0008E00AB1194A05E0154A12780AB1184A65
:10CEDC0000E0184A1A60184A1268002A15DB110281
:10CEEC00164801F47F41825C15481143002230F84A
:10CEFC00125054008D4205D10021124A1B6811605A
:10CF0C00185B30BD01322A2AF1D1002030BD00BFA0
:10CF1C00156800203F72002074660020001F00205E
:10CF2C0040720020AC1E0020581E0020041E002061
:10CF3C00B01D00205C1D00206430002053720020C6
:10CF4C00081D00200466002008B5022123200AF0E9
:10CF5C00F9FD022124200AF0F5FD022126200AF019
:10CF6C00F1FD022125200AF0EDFD022122200AF01C
:10CF7C00E9FD022129200AF0E5FD022128200AF012
:10CF8C00E1FD01210E200AF0DDFD01210E200AF049
:10CF9C00A7FD012110200AF0D5FD012106200AF081
:10CFAC00D1FD012118200AF0CDFD012119200AF034
:10CFBC00C9FD01211C200AF0C5FD01211F200AF02A
:10CFCC00C1FD012110200AF08BFD012106200AF081
:10CFDC0087FD012118200AF083FD012119200AF098
:10CFEC007FFD01211C200AF07BFD01211F200AF08E
:10CFFC0077FD022113200AF0A5FD022112200AF070
:10D00C00A1FD022111200AF09DFD022105200AF04C
:10D01C0099FD02211D200AF095FD02211E200AF027
:10D02C0091FD02212020BDE808400AF08BBD0000D4
:10D03C0030B50B4C01250B4B85B0204600211D70E3
:10D04C0000F010FF40F2FF721F23204602958DE87E
:10D05C000C000022044B114600F08CFF05B030BDD3
:10D06C00C272002048310020F82A0020A64A03464C
:10D07C002DE9F04F14789FB0002C40F07D8141F2E7
:10D08C001002A24D0240002A58D0A1490EA80CF063
:10D09C00DEFCA0490EA80CF0C1FC9F490EA80CF0B8
:10D0AC00BDFC0EA99A480CF0D2FC9C48FFF7CCFCB6
:10D0BC009748FFF7C9FC04A82346954A9849FFF7FF
:10D0CC000FFC089850B103689B6B984730B1954B97
:10D0DC001C60FFF741FC944B186029E0934B1B78C4
:10D0EC002BB30123924A8E4909A8FFF7F9FB0DA92E
:10D0FC009048FFF774F90069FFF783F9044609A813
:10D10C00FFF73CF99CB182480CF0A9FC804902461F
:10D11C008848FEF769FF04467D480CF0A0FCA0424D
:10D12C0002D08548FFF790FC8248FFF761FB812411
:10D13C00012304A82B70FFF721F970E000F0200404
:10D14C00A1B299B1012374497C4882242B700CF054
:10D15C007EFC6F497A480CF07AFC6E4978480CF0EA
:10D16C005DFC764976480CF059FC58E000F0400420
:10D17C00A0B230B1012308462B70FFF7A5FC0C467A
:10D18C004DE040F204441C404CB1664A1368002B3D
:10D19C0040D00121013B0446297013603FE040F26E
:10D1AC0001121A406AB15F4A1368082B03DD012192
:10D1BC00093B297003E06BB30121013B297013601B
:10D1CC002DE040F60801194061B1574B55491C68D8
:10D1DC000B68601E98421FDD0CB301330B600123FA
:10D1EC002B7019E040F202241C40C4B14E4B4D4A46
:10D1FC001C681368A4F10901994202DD0CB10933D2
:10D20C0004E0611E8B4209DA4CB101331360012337
:10D21C002B7003E01C4602E0144600E000242B783F
:10D22C00002B00F0AB80404B1A689B46002A00F0A4
:10D23C00A58090234FF0080C202210214148002695
:10D24C00DFF80CA137468DE808104FF4887300F016
:10D25C0047FE344A13689146082BD4BF0023043B85
:10D26C00CAF80030DBF80020974224DB00264FF090
:10D27C001F0E40F2FF73C8223021324802968DE80F
:10D28C000840314B00F076FE0823C8227821009329
:10D29C004FF488732B48019600F022FE4FF6FF7373
:10D2AC000296C822009378210196244B254800F061
:10D2BC0061FE2E7062E0DAF800309F4256DB334498
:10D2CC009A4252DD214A4FF0220808FB0728D9F870
:10D2DC00002093424FF0010306F1020202934FEA41
:10D2EC00021237D14FF6E0704FF4784312B210218E
:10D2FC008DE809004346134800F03CFE41460648C1
:10D30C000CF0A5FB31E000BF517200204831002029
:10D31C005A720020792A00205A6900200C2B002018
:10D32C00F0600020A0660020A86600201568002090
:10D33C001C2B00207C3000202F2B00207C6900202F
:10D34C001A680020C2720020432B00209E69002026
:10D35C00B06600204FF6FF71082312B209488DE821
:10D36C000A004346102100F005FE0136082E07F195
:10D37C0001077FF777AF79E7812000E020461FB0E7
:10D38C00BDE8F08FC2720020014B1878704700BFC7
:10D39C004B310020034B18B101221A70FFF748BE25
:10D3AC00187070474B310020004870475A720020AB
:10D3BC00F0B5044687B019480E461746184DFFF7CE
:10D3CC0043FB2046FFF740FB22460023154901A8EA
:10D3DC00FFF786FA05A92846FFF701F80069FFF761
:10D3EC0010F8044601A8FEF7C9FFA4B12869FFF79D
:10D3FC000DF80446FFF730FBBC4209D822463146F3
:10D40C002869FEF7E7FF844202D00748FFF71CFBB0
:10D41C000348FFF7EDF9204607B0F0BD942B002030
:10D42C007C300020F0600020A02B0020674B684966
:10D43C001868F0B50C4693B0664D40F2EE27664E78
:10D44C000A784AB12A78D20706D51A68D6F800E0CD
:10D45C00CEEB02020E2A0AD81A6894F800E0121ACF
:10D46C00BEF1000F00F0B080B2F5FA6FE8D901F010
:10D47C00D3FA5A4B5A4A9A645A4ADA64FE215A48E9
:10D48C0004F0FCFB40B959495948FEF7ECFF4FF446
:10D49C007A700AF00FFBF1E70024564D56495748B5
:10D4AC000CF0D5FA281914345549FEF798FF502C76
:10D4BC00F8D1544CFFF750FA5349002520604C48E2
:10D4CC00FEF7C3FF21684A48FEF7D7FFFFF73CFD84
:10D4DC004E4B29464E481D7000F0D2FBFFF706FB61
:10D4EC0010F008043DD04FF47841494800F0BAFCE4
:10D4FC0001244FF6E0724FF47843402144488DE804
:10D50C001C00444B302200F035FD374BD3F884140B
:10D51C0079B12346404A04A88DF810508DF811506B
:10D52C008DF8125006F02CFEB0B104A807F09EFC4A
:10D53C0012E0D3F8880478B18DF8411023468DF8A9
:10D54C0042108DF843100146334A04A805F080F8C8
:10D55C0010B104A805F00DF94FF47A700AF0AAFA8C
:10D56C002BE02E4E23462C4A04A81F49FFF7B8F98E
:10D57C0008A93046FEF733FF0069FEF742FF054667
:10D58C0004A8FEF7FBFEC5B130691C4FFEF73EFF49
:10D59C000546024639463069FEF71CFF854203D02A
:10D5AC001F48FFF751FA01E07C5501241B48FFF797
:10D5BC001FF914B101221B4B1A7001221A4B1A705D
:10D5CC00FFF736FD13B0F0BDBA424FE79C67002061
:10D5DC00CF720020CE720020D8730020A04D002006
:10D5EC00399A000061990000F0600020C12B0020E6
:10D5FC000030002014300020DE2B00205A72002056
:10D60C0078300020A8660020E52B00200F68002051
:10D61C00C2720020032C00201C2B00207C30002028
:10D62C00182C0020517200204B3100200022014B9D
:10D63C001A7070479A72002070B54B4800244B4DFD
:10D64C0020264B4B44608460C0F82403C0F844038C
:10D65C00036002F07FFF21466C60AC6032462C61A7
:10D66C0005F128006C61EC6185F820406C620AF0D1
:10D67C00D1F9404B284685F8854203F140022B60D6
:10D68C006C332C65EA60AB616C6585F87840C5F845
:10D69C00804285F8844285F8864285F8874203F0FB
:10D6AC0035FC3548354D364B44608460C0F89006E7
:10D6BC00036080F87546C0F87846C0F87C4680F860
:10D6CC00804680F8A44602F081FB324621466C600D
:10D6DC0005F11C00AC602C612C75AC610AF09AF958
:10D6EC00284B284685F841402B603833EC63EB60BF
:10D6FC0085F8404085F8424085F843406C64AC6442
:10D70C00EC642C6504F0EEF81F4D204B6C60284641
:10D71C002B6005F59F63AC606B6305F5A7632D6209
:10D72C00AB6305F5AF631A4EEB6305F5B7636B643A
:10D73C004023A5F84A305023A5F84C3003F08EFF57
:10D74C00144B314614482B60144D2A460BF0CFFF76
:10D75C002A46134920460BF0CAFF2A463146114887
:10D76C00BDE870400BF0C3BFE0490020A04D002085
:10D77C00B40500205C040020204300202C6700200E
:10D78C00A8030020E003002040500020C403002028
:10D79C007D9C00006803002068300020302F0020A2
:10D7AC00AD9C00007C300020034B1A780AB100229B
:10D7BC0000E001221A7070476631002010B5044653
:10D7CC000BF09EFB204610BD0F2B09DC8908D208FC
:10D7DC00C00842EA4112034942EAC02221F8132050
:10D7EC00704700BFB2670020094B82B000211A7845
:10D7FC00D2B28DF80720074A1160074A127822B975
:10D80C0019789DF807209142FAD002B0704700BFFA
:10D81C006631002078660020D272002007B5064AD7
:10D82C00127832B9054A8DE805000122044800F04F
:10D83C00A7FC03B05DF804FBD2720020B267002095
:10D84C00C272002008B5034800F050FABDE8084049
:10D85C00FFF7ECBDC272002038B5FFF795FD20B381
:10D86C00FFF712FBFFF702FC0446FFF79DFD054690
:10D87C00812C18D100200024FFF78CFD104B1C705C
:10D88C00FFF7D4FEF5F778FB2846F5F7A9FB214600
:10D89C000C4800F0E7FA0B4800F0DAFC0A4A0B4996
:10D8AC000B480BF0D1FA142006E0FFF7EDFAF5F770
:10D8BC0055FBF5F75DFC1020BDE838400AF0FAB8CE
:10D8CC00D2720020C27200206F1A0600A9B00000AC
:10D8DC009030002010B50A21084C09480BF0A0F834
:10D8EC0008480BF04BFB2046074A4FF480710CF0B4
:10D8FC007BFE2046BDE81040FEF75ABBAC72002000
:10D90C002B2C002000300020F100000005280B46D5
:10D91C0003DC01460148FEF751BB7047AC72002096
:10D92C007FB5FF231A211B220A4804930393029309
:10D93C008DE806001722162100F01CF9064A07494B
:10D94C0007480BF0D4FE0AF087F8064B186007B0B6
:10D95C005DF804FBC2720020302F0020BDB0000027
:10D96C00903000207C660020154B164910B51879B4
:10D97C00154BC8771A78154C01322478D2B21A702C
:10D98C001A78944208D800221A70114A12781AB1E7
:10D99C00887601210F4A11701A780F4B53F8222008
:10D9AC0022F01F0302F50042BFF34F8F0B490B60AF
:10D9BC0020339A42FBD8BFF34F8FBFF36F8F10BD4C
:10D9CC008066002000800E40146800201268002041
:10D9DC00527200203E7200209066002068EF00E03A
:10D9EC0010B504460BF0A8F9204610BD13B502ABD8
:10D9FC0003E90600C37C0099002B2ED072B6C37CC1
:10DA0C00DA0705D5324A43691468234083621360F0
:10DA1C00C37C9B0705D52F4A836914682340C362D6
:10DA2C001360C37C5C0705D52B4AC369146823407B
:10DA3C0003631360C37C1A0705D5284A036A14686C
:10DA4C00234043631360C37CDB0605D5244A436A39
:10DA5C00146823408363136062B683688B422AD0B8
:10DA6C00204B81609A69204BC2F30114C2F382628D
:10DA7C0053F824300132B3FBF2F211B1B2FBF1F3E3
:10DA8C0000E013467BB1B2FBF3F2914238BF013395
:10DA9C00B3F5817F02D2022B04D901E040F20113CD
:10DAAC00023B00E000235A0843EA0223120402F46A
:10DABC007F021343C360036800221A6103225A6277
:10DACC00C2681A64019A1A6601221A6102B010BD6A
:10DADC0080E100E084E100E088E100E08CE100E01E
:10DAEC0090E100E000C00F40B806002003685966C2
:10DAFC00DA6D12F4F81FFBD0586FC0B27047036890
:10DB0C00186E20F47F6222F00F0242F00F021A66A8
:10DB1C0059661A6F9207FCD41866586F80B270471A
:10DB2C00C37CE3B1DA0702D5826A0D4B1A60C37C61
:10DB3C009B0702D5C26A0B4B1A60C37C590702D5EE
:10DB4C00026B094B1A60C37C1A0702D5426B074B58
:10DB5C001A60C37CDB0602D5826B054B1A607047DA
:10DB6C0000E100E004E100E008E100E00CE100E08D
:10DB7C0010E100E070B50446FF209DF81C60237096
:10DB8C009DF81030A07123719DF81430E0710020C5
:10DB9C0063719DF81830A270E370207210466170AA
:10DBAC0001219DF8205009F0CDFF0121607809F08A
:10DBBC00C9FF0121607809F093FF0121A07809F0D9
:10DBCC008FFFFF2E0FD0FF2D0DD001213046A571F8
:10DBDC00E67109F0B7FF0221284609F0B3FF0121D5
:10DBEC00E07909F07DFF204670BD00002DE9F84377
:10DBFC00224D044689468078002117469846BDF888
:10DC0C00206009F06DFF2A212846FFF76FFFA078EE
:10DC1C00012109F065FF49462846FFF770FFA078FF
:10DC2C00012109F05DFF41462846FFF768FFA07807
:10DC3C00002109F055FF2B212846FFF757FFA0784C
:10DC4C00012109F04DFF39462846FFF758FFA0780F
:10DC5C00012109F045FF31462846FFF750FFA07817
:10DC6C00002109F03DFF2C212846FFF73FFFA0784B
:10DC7C000121BDE8F84309F033BF00BFB02F0020ED
:10DC8C0037B5174B0446174A0D4617488DE80C005C
:10DC9C0002AB13E90600FFF7A9FE0021A07809F0FA
:10DCAC001FFF0021607809F01BFF36210E48FFF79B
:10DCBC001DFF0121A07809F013FF1DB10123A02144
:10DCCC00237201E0602125720748FFF70FFF012145
:10DCDC00607809F005FF0448FFF722FF03B030BD60
:10DCEC000700008000879303B02F00202DE9F04F30
:10DCFC00044685B00179564800F018FDE178544887
:10DD0C0000F046FD6179524800F06EFD504800F07D
:10DD1C0001FC2078FF2817D0012109F013FF012105
:10DD2C00207809F0DDFE642009F0C4FE0021207883
:10DD3C0009F0D6FE642009F0BDFE2078012109F01F
:10DD4C00CFFEC82009F0B6FE424D0DF10808DFF8F1
:10DD5C0010A10A260395A946CDF808A03C483E4FD1
:10DD6C0098E80600FFF742FE0021607809F0B8FE43
:10DD7C00013E16F0FF064DD03D460021A07809F07B
:10DD8C00AFFE15F8021B3248FFF7B0FE7F7827F084
:10DD9C007F0B07F07F075FFA8BFB012F0BD901215B
:10DDAC00A078013F09F09CFE15F8011B2848FFB232
:10DDBC00FFF79CFEF1E74FB16F1C0121A07809F031
:10DDCC008FFE29783D462248FFF790FEBBF1000FED
:10DDDC0001D12F46CCE76F1C2D7801216078FF2DE7
:10DDEC0008BF4FF4FA7509F07BFE1948FFF798FE4F
:10DDFC00284609F05FFECDF808A0CDF80C903D4602
:10DE0C00134898E80600FFF7F1FD0021607809F04F
:10DE1C0067FEDEE76078012109F062FEEF233246EF
:10DE2C0031460093204640F23F13FFF7DFFE0848CF
:10DE3C00FFF776FE094B314620461E70FFF720FF98
:10DE4C000121204605B0BDE8F04FFFF719BF00BF18
:10DE5C00B02F0020070000800522006052720020C5
:10DE6C0000879303F0B51B4B85B004460F46029315
:10DE7C00F025194B1948039304AB13E90600FFF77F
:10DE8C00B5FD0021607809F02BFEEF23002220461F
:10DE9C00009340F23F131146FFF7A8FE4FF4A07613
:10DEAC0039460E48FFF72BFE013EF9D1013DF5D165
:10DEBC006078012109F014FEEF232A4629460093CD
:10DECC00204640F23F13FFF791FE0448FFF728FE6F
:10DEDC0005B0F0BD0087930307000080B02F002031
:10DEEC002DE9F0431D4685B01F4B0446BDF930703B
:10DEFC008846029391461D4B1D48039304ABBDF815
:10DF0C00346013E90600FFF771FD0021607809F019
:10DF1C00E7FD781E1FFA89F26B1E1FFA88F17D430C
:10DF2C00104400270B4480B29BB200902046FFF7B0
:10DF3C005DFEAF4205DA31460D48FFF7E0FD0137D3
:10DF4C00F7E76078012109F0CBFD0022EF23204692
:10DF5C001146009340F23F13FFF748FE0448FFF7C9
:10DF6C00DFFD05B0BDE8F083008793030700008058
:10DF7C00B02F00202DE9F04F89B09B461FFA82FA92
:10DF8C0081469DF850308846BDF84850002B0393CD
:10DF9C00BDF84C6014BF0F23072353449BB204936A
:10DFAC001BF8017B06AB002F00F0BF80704A1FFAF4
:10DFBC0088F8704802EBC7076F4A06926F4A0792BF
:10DFCC0093E80600FFF712FD002199F8010009F013
:10DFDC0087FD049A08F107034146009248469BB21C
:10DFEC005246FFF703FE07F108030593039B002B32
:10DFFC0044D03C785F48E2074FEA64044CBF2946A2
:10E00C003146FFF77CFDE3074FEA640459484CBFE7
:10E01C0029463146FFF773FDE0074FEA6404554883
:10E02C004CBF29463146FFF76AFDE1074FEA64040D
:10E03C0050484CBF29463146FFF761FDE2074FEAD5
:10E04C0064044C484CBF29463146FFF758FDE307A2
:10E05C004FEA640447484CBF29463146FFF74FFD51
:10E06C00E00744484CBF29463146FFF748FD63089A
:10E07C00404814BF29463146FFF741FD17F8014BC4
:10E08C003C48E1074FEA64044CBF29463146FFF790
:10E09C0036FDE2074FEA640436484CBF2946314648
:10E0AC00FFF72DFDE3074FEA640432484CBF2946C5
:10E0BC003146FFF724FDE0074FEA64042D484CBFBE
:10E0CC0029463146FFF71BFDE1074FEA6404294856
:10E0DC004CBF29463146FFF712FDE2074FEA6404B4
:10E0EC0024484CBF29463146FFF709FDE307214878
:10E0FC004CBF29463146FFF702FD63081D4814BF8B
:10E10C0029463146FFF7FBFC059B9F427FF46EAF1F
:10E11C0099F80100012108F1080809F0E1FC154803
:10E12C000FFA88F8FFF7FCFC3AE7134A11480692FD
:10E13C00124A079293E80600FFF758FC394699F803
:10E14C00010009F0CDFCEF233A46394600934846CE
:10E15C0040F23F13FFF74AFD012199F8010009F045
:10E16C00BFFC0448FFF7DCFC09B0BDE8F08F00BF32
:10E17C0027220060B02F0020008793030700008047
:10E18C0070B5274A9D11B1F5807F03F03F0352F81B
:10E19C0025200498059C02EB43231CDDA1F580721D
:10E1AC0003F5007691FBF2F101390D46013D027841
:10E1BC000CBF4578013034F8122001BF023034F81E
:10E1CC00155052190D4608BFC2F34F0223F8022B0B
:10E1DC009E42EBD170BD4A00B2F5807F10D1024651
:10E1EC00151A04338D421ADA157834F8155023F8C1
:10E1FC00045C12F8015B34F8155023F8025CEFE76D
:10E20C00C1F5807222F00102134400228A4206DA20
:10E21C00855C34F8155023F812500132F6E770BDC6
:10E22C009066002010B50020084C821100F03F03CE
:10E23C0054F8222002EB432303F5007223F8021B4F
:10E24C009342FBD10130F028EFD110BD9066002035
:10E25C002DE9F04F844B0024074684481C7087B08E
:10E26C0002798046824B02F11001824D1C70824B68
:10E27C00DFF808B243F821505311012102F01F02BC
:10E28C009B004FF4F03501FA02F203F1604303F501
:10E29C0061431A60B5F5004F5BF824202E464FEA17
:10E2AC00840928BF4FF400462AB906F140000BF050
:10E2BC0069FA20F01F02714B43F8092082B925211D
:10E2CC006F4803920AF0ACFB21466E480AF0B5FE8B
:10E2DC006C480AF053FE42F2107009F0EBFB039A03
:10E2EC0026F00101134600201144994202D023F874
:10E2FC00020BFAE7A101DFF8ACA14FF00109AD1B4D
:10E30C0051F80A3001F140014C441A604FF00202FE
:10E31C0083F807909A609A80C6F1000283F8069001
:10E32C00DA60C6F34F02DA83DA82574A1A614FF089
:10E33C0000029A8251F80A209A619A8B22F080028C
:10E34C004FEA02424FEA12429A839A8B92B242F0FF
:10E35C0010029A839A8B92B242F002029A8399D15C
:10E36C00DAF80020384620219A619A8B22F080023C
:10E37C001204120C9A839A8B92B242F010029A8376
:10E38C002A46424B1C70EF2440F21F130094FFF7F7
:10E39C002DFC29463846FFF745FF4946787809F0A9
:10E3AC009FFB3B4800F0B6F83A4B394804930723DF
:10E3BC00059306AB13E90600FFF718FB364B1A69F9
:10E3CC0022F001021A615A6A42F008025A620F22C4
:10E3DC001A66C3F81C901A6942EA09021A6198F885
:10E3EC0004302E4A9B0003F1804303F56C231D601F
:10E3FC001A60D8F80030DAF80020998B101D21F043
:10E40C008001090490E84140090C99831168586017
:10E41C0002F11400C3F80CE019609E60166907C87D
:10E42C001E6199612946DA615861787809F058FBC8
:10E43C002A4640F21F13384600942021FFF7D6FBE2
:10E44C002946B87809F04CFB2C211148FFF74EFBFC
:10E45C004946B87809F044FB98F80420104BDA765A
:10E46C0007B0BDE8F08F00BF146800208066002064
:10E47C003E72002069B2000000340020906600203B
:10E48C00362C00200030002064C039401268002077
:10E49C00B02F00200087930300C03940100000808B
:10E4AC0000800E40804000200D4B1A4603F12001E5
:10E4BC0010B542F8601B00211A6403F1A002094C4C
:10E4CC00C3F8802003F1E0022046C3F8C0200AF014
:10E4DC00E5FB2046044A0549BDE810400BF007B99E
:10E4EC008040002080660020302F0020E1B2000028
:10E4FC00C38B1B0402D4C1F30E0105E0C38BC1F323
:10E50C00080103F47E431943C183C38B9BB2C382BE
:10E51C00704700004368196830B50A685C6822EAE5
:10E52C000402744C0A60A26922F0E05222F030021C
:10E53C0042F0006242F01002A261047C6E4A1C445C
:10E54C00247C02EB0414A568B8242C60457C1D4483
:10E55C0095F8245002EB0515AD682C60857C1D44A4
:10E56C0095F8385002EB0515AD682C600D685C68A9
:10E57C002C430C60017C5C1803EB8101247C496901
:10E58C0002EB041464682160417C5C180A3194F835
:10E59C00244053F8211002EB041464682160817C40
:10E5AC005C1803EB810194F83840C96B02EB041240
:10E5BC0052681160827C996C1A4492F844200A606B
:10E5CC00027C196A1A44127F0A60427C596B13440C
:10E5DC00022293F830300B6003681A610F229A659F
:10E5EC00C37C002B2ED072B6C37CDD0705D5434A05
:10E5FC00436911680B4083621360C37C9C0705D58B
:10E60C003F4A836911680B40C3621360C37C59078E
:10E61C0005D53C4AC36911680B4003631360C37C86
:10E62C001A0705D5384A036A11680B404363136017
:10E63C00C37CDB0605D5354A436A11680B408363FE
:10E64C00136062B6324983688B4227D0294B8160B4
:10E65C009A69304BC2F30114C2F3826253F824302E
:10E66C000132B3FBF2F2B2FBF1F37BB1B2FBF3F28A
:10E67C008A4288BF0133B3F5817F02D2022B04D9C1
:10E68C0001E040F20113023B00E000235A0843EA88
:10E69C000223120402F47F021343C36003680022B6
:10E6AC001A6103225A62C2681A6407221A6601228E
:10E6BC001A61C37CE3B1DD0702D5826A164B1A607E
:10E6CC00C37C9C0702D5C26A144B1A60C37C5907E1
:10E6DC0002D5026B124B1A60C37C1A0702D5426B2F
:10E6EC00104B1A60C37CDB0602D5826B0E4B1A6092
:10E6FC0030BD00BF00C00F402C07002080E100E0BF
:10E70C0084E100E088E100E08CE100E090E100E0D1
:10E71C0000093D00B806002000E100E004E100E043
:10E72C0008E100E00CE100E010E100E04368427C0D
:10E73C001A4430B592F824208A4225D093F824202C
:10E74C00914205D093F8252091421DD1012100E082
:10E75C0000211C6825685C68254214D00B4CB82538
:10E76C0004EB0212926815605A1892F8245004EBCC
:10E77C00051401F10A05646853F825505B6B25609C
:10E78C0092F830201A60417430BD00BF2C07002075
:10E79C004368027C1A4430B5127C8A4221D01A7C20
:10E7AC00914204D05A7C91421BD1012100E00021FE
:10E7BC001C6825685C68254212D00A4CB82504EB0D
:10E7CC000212926815605D182A7C04EB02140A1D73
:10E7DC0003EB820264681B6A526822602A7F1A600B
:10E7EC00017430BD2C0700204368827C1A4430B57C
:10E7FC0092F838208A4226D093F83820914205D0DE
:10E80C0093F8392091421ED1012100E000211C68AF
:10E81C0025685C68254215D00B4CB82504EB021218
:10E82C00926815605D1895F8382004EB021401F11C
:10E83C000E0203EB820264689B6C5268226095F8AE
:10E84C0044201A60817430BD2C07002070B54BB386
:10E85C00046840F2012525611C46066811B10D784B
:10E86C00013101E090F83C50013C756605682E6F53
:10E87C00B60705D46D6FEDB20AB115700132013BCC
:10E88C0005686D69ED07F1D5002CE6D153B101682F
:10E89C000C6FA407FAD4496FC9B20AB111700132D6
:10E8AC00013BF3E770BD0000836C10B51A79044688
:10E8BC001C4BDA77426C12791A77826C12791A77C0
:10E8CC00026CDAB1B2F5004F04D3A2F5FF427F3AE5
:10E8DC0002640BE0436C11461868FFF709FEA36C49
:10E8EC00216C1868FFF704FE00232364A36C1A79CB
:10E8FC000C4BDA76626C1279DA7610BD03680F2154
:10E90C00996540F20131DA6119614FF47C5159611A
:10E91C000323114680F83D30C06C0368BDE81040FD
:10E92C001B68184700800E4008B50248FFF7BCFF73
:10E93C0008BD00BF602F002008B50248FFF7B4FFE8
:10E94C0008BD00BFB02F00207047002070470000AA
:10E95C000023064A436013680BB9106070475A686D
:10E96C000AB11346FBE75860704700BF04670020EC
:10E97C000020704700207047704730B5039C01257C
:10E98C001B024560002C9DF8105043F0800318BF0B
:10E99C004FF0004443EA0242002D44EA020414BF43
:10E9AC004FF4004500252C438460C16021F47F6145
:10E9BC0021F00F0101F58053036101F50053436110
:10E9CC0001F5405301F580418361C16130BD000008
:10E9DC00436A026A0BB11A6201E004490A600AB187
:10E9EC0053627047024A1360704700BF20660020D4
:10E9FC001C660020436A026A0BB11A6201E00449EA
:10EA0C000A600AB153627047024A1360704700BF34
:10EA1C002866002024660020F8B54FF480314D4B59
:10EA2C0040244FF480554FF400564FF4404743F2C6
:10EA3C00420E1A6A900704D59F625962C3F828E007
:10EA4C00F7E7900401D45E62F3E7D00401D45D6271
:10EA5C00EFE7002AEDDA12F4803001D09962E8E792
:10EA6C00520601D45C62E4E73B4A3C4CD2F880305D
:10EA7C0043F00303C2F880304FF04042384B9A63A6
:10EA8C004FF440425A630522186003F58F130A2095
:10EA9C00C3F8B4200822C3F8A422324B5A6842F0BF
:10EAAC0080625A604FF08062C3F8842009F002F84B
:10EABC00D4F8403143F00203C4F84031D4F840316B
:10EACC0013F00205FAD102F0A7FC2B46264A0121CD
:10EADC0042F823100133202BFAD14FF4807200211D
:10EAEC00224808F097FF0023214A13700122C4F832
:10EAFC0090200322C4F8A8211B4AC4F84831C4F85A
:10EB0C005421C4F84C31C4F858311A4B1A4AC4F881
:10EB1C004031D4F8843143F48053C4F88431D4F8B0
:10EB2C005831D4F85431154BC3F80022144B4FF420
:10EB3C0080321A60134BC4F84831D4F8483143F092
:10EB4C001203C4F84831D4F8483143F44023C4F8D4
:10EB5C004831F8BD00800D4000C00F4000022E402F
:10EB6C0000A00D4000800042004000205A680020A8
:10EB7C0013680020158B01003DC8000000340020F4
:10EB8C000CE100E004000003C36870B504460D46B8
:10EB9C00002B4AD0632948D908F05EFF234BA060B4
:10EBAC001A68234E5AB96561013D1C604FF0404311
:10EBBC00A261E261C6F88850C6F88C3070BDD6F8F8
:10EBCC008C1021F07F418D4218D272B600204FF08C
:10EBDC000072491BC6F88C00C6F844211A6865619E
:10EBEC00013D1C604FF04043A261E0615161D46172
:10EBFC00C6F88850C6F88C3062B670BD6D1A936931
:10EC0C007BB15A69954209D2521B5A61DA69A361E8
:10EC1C00E2616561DC61E3699C6170BDAD1A1A4605
:10EC2C00EDE76561A361E261946170BDD46500207C
:10EC3C0000022E4070B50A460646036999684906DB
:10EC4C0001D41B68FAE74021956803F13404916004
:10EC5C001168196051685960D168D96011691961DE
:10EC6C005169596191699961D1699E62D961D16A81
:10EC7C00D962116B196302F1340103C984E80300F2
:10EC8C00D16BD96319460868012801D00968FAE7E5
:10EC9C000A601946106000200C68A24205D00C686E
:10ECAC00486208460C622146F6E7002248620A6276
:10ECBC0096F8342012F0FD0F05D1094A10685862FD
:10ECCC0040B9084804E0084A1068586210B907486F
:10ECDC00036000E00362116001209D6070BD00BF05
:10ECEC001C66002020660020246600202866002078
:10ECFC002DE9F04F85B082460D4693460393CB88A1
:10ED0C00B3F5804F57D802F03BFB0646002852D093
:10ED1C0002F036FB044608B9304608E0EB88CBB16C
:10ED2C0002F02EFB30B9304602F032FB204602F0E6
:10ED3C002FFB40E095F9007001210023EA888DE853
:10ED4C000A00FB0FFF435946FFF717FE3060FF0F19
:10ED5C00046001E0012730604FF000094FF001081A
:10ED6C0029463046CDF804900223CDF800900822B5
:10ED7C00FFF703FE3B4649462046CDF804804A4641
:10ED8C00CDF80080FFF7F9FDDAF80030C4F82CB0AC
:10ED9C003146A362EB8823632B6863636B68C4F80A
:10EDAC000080A363039BDAF80000E36305B0BDE8C1
:10EDBC00F04FFFF73FBF002005B0BDE8F08F2DE905
:10EDCC00F74F8146884617469A4602F0D9FA06460E
:10EDDC00002840D07D1E0446AD0B75B102F0D0FA70
:10EDEC0038B93046356802F0D3FAA64233D02E46F5
:10EDFC00F7E72060013D0446EFE70123C4F82890B3
:10EE0C00C4F82C80236027636563A563C4F83CA019
:10EE1C003446B7F5804F99F835304146204693BFBC
:10EE2C00BA464FF4804A4FF0000B4FF0010B52469C
:10EE3C008DE82008FFF7A1FDBBF1000F04D1D044F1
:10EE4C00CAEB07072468E4E73146484603B0BDE83F
:10EE5C00F04FFFF7EFBE002003B0BDE8F08F8268E3
:10EE6C00110608B507D48268120406D5836ADB6BD9
:10EE7C001BB1984701E0002008BD012008BD00002F
:10EE8C002DE9F8432C4B4FF000081C68002C50D097
:10EE9C002046FFF7E4FF256A002844D020462E4682
:10EEAC00FFF796FDA36858063AD5A76A20462C466C
:10EEBC00002502F06DFA9EB1B36AD6F820909F42FD
:10EECC0001D04E46F7E73046FFF782FD0DB12E62BA
:10EEDC0000E03546C6F82080A64208BF4C46F0E755
:10EEEC003B6923F01F033BB19A6851061DD53B616A
:10EEFC00C7F80C80C7F81880002DC7D0AB681A046F
:10EF0C0008D5FA6B32B143F040032846AB60AB6ACC
:10EF1C00DB6B98472E6A284602F03AFA3546EBE747
:10EF2C00204602F035FA2C46B0E79A681A681B683E
:10EF3C00D7E7BDE8F88300BF206600202DE9F0413B
:10EF4C00524CD4F844516E03C4F844510FD5504B75
:10EF5C001E6866B13046FFF782FF376A28B130462B
:10EF6C00FFF736FD304602F013FA3E46F1E7280370
:10EF7C000FD5484B1E6866B13046FFF770FF376AF5
:10EF8C0028B13046FFF736FD304602F001FA3E4616
:10EF9C00F1E7A90701D5FFF773FF6A073ED5D4F84F
:10EFAC0084613A4A46F02A03C4F88431B3071DD56C
:10EFBC0016F00108384B0ED01978012916D801210A
:10EFCC0025F080751970354BC2F880304FF04043F6
:10EFDC00C2F884300AE083F800800222304B314FB3
:10EFEC009A63386800F070FDC7F80080370715D4B5
:10EFFC00294A1378022B11D170070FD503211170F8
:10F00C0042F21072C4F880204FF04042C4F88420C1
:10F01C00D4F88421910501D5214A5363EA011AD50C
:10F02C001D4B1A78012A08D102221A70D4F88431A7
:10F03C0043F48073C4F884310DE0032A0BD104220D
:10F04C001A700022D4F884011146C0F3816000F0DC
:10F05C00FFFA144B1860AB0115D5134A116891B126
:10F06C008B6913604BB10022DA615B69013BC4F818
:10F07C0088304FF04043C4F88C30C8680368BDE852
:10F08C00F0419B681847BDE8F08100BF00022E409C
:10F09C00206600202866002013680020A08601004E
:10F0AC0000A00D40AC660020D4650020844B002AE3
:10F0BC0008BF01225943036B2DE9F04F1B7D85B02E
:10F0CC00090C022B4FF0010360D10F2A01F15701FB
:10F0DC004FF0FF35DFF8ECC128BF0F224909013A88
:10F0EC0003FA02F2B2F5807FA8BF4FF48072D40805
:10F0FC0018BFA3B20024A0F840302B4627460026A8
:10F10C0017F80CE017448E44764538BF7646FF2F2F
:10F11C00DFF8B0E1F4D9B54288BF234604F101040D
:10F12C0088BF3546A242E9D1BB2D01D90020C4E0ED
:10F13C00C9B21C46A0F84420A0F8463080F84A100A
:10F14C00FF2C06D81EF804500D440EF8045014443D
:10F15C00F6E7012A01D1FF220EE0022A03D103F0C7
:10F16C000101552207E0042A99BF03F00301112283
:10F17C0003F0070101228A40DB0880F83620A0F852
:10F18C004230002380F83730012096E0052443EA12
:10F19C005305AA4204D9013C4FEA4303F7D120237B
:10F1AC009AB20392BDF80C20A0F8402090F83520BC
:10F1BC0022B984314A090221029203E0663102220B
:10F1CC00490902924FF0FF324FF0000C1546E6460B
:10F1DC000192E0463B4A4FF0000B02EBC806144686
:10F1EC00029A96F800A096F802909244F778894417
:10F1FC0032790F44CA450A4405D9BA4509D9524552
:10F20C0038BF524608E0B94503D94A4538BF4A468B
:10F21C0002E0BA4238BF3A46019F0136BA4238BFC3
:10F22C00DE460BF1010B3CBF01924546BBF1040FCE
:10F23C00D6D19844B8F11F0FCCD90CF1010C9C45D8
:10F24C00C7D1019ABB2A3FF671AFBDF80C20AEB204
:10F25C009DF808C0C9B2A0F84420A0F84660A0F8F8
:10F26C0048E080F84AC080F84B101F2D18D80EEBE0
:10F27C00C5021D44A75C02F102086744A75414F8A8
:10F28C0008700F4404F8087002F10308043214F8F3
:10F29C0008700F4404F80870A75C0F44A754E4E707
:10F2AC000123A0F8426003FA0EF280F836201C22EB
:10F2BC0002FA0EFE80F837E0184605B0BDE8F08F74
:10F2CC00AB2A01005A680020F0B51C4D40F0020634
:10F2DC00B0F84040B0F842102F461F292CD855F8F2
:10F2EC0021204FEA810ED3070AD402F0060C22F03B
:10F2FC001F03BCF1020F0FD1B3F840C064450BD90A
:10F30C00026047F80E6015E0834213D01A68D207EA
:10F31C0006D41B6823F01F03B3F840209442F3D9A2
:10F32C001A46824206D0126832F01F02F9D11A68CE
:10F33C0002601E602144D0E7F0BD00BF00400020F9
:10F34C002DE9F84F0A9F05460E4690469A4602F064
:10F35C0007F80446002800F08A8002F011F8814674
:10F36C0028B9204602F004F84846BDE8F88F4FF063
:10F37C00400B60220021204608F04CFB5A4600212D
:10F38C00484608F047FB0123032EC9F80030C9F8A2
:10F39C0008B0C4F810902563636184F835A084F834
:10F3AC00346010D10B9A39462046FFF77FFE824617
:10F3BC00002861D1484601F0EBFF204601F0D8FF50
:10F3CC005046BDE8F88FB8F1000F08D06B680BB948
:10F3DC006C6004E09A6B0AB11346FBE79C6316B1B0
:10F3EC0000210B4605E02B7D0121012B8CBF002356
:10F3FC0001236A7D287D42F0704242EA003242EAE3
:10F40C00082242EA074242EAC36343EA813194F894
:10F41C003630616043F08043EA7D43EAC253AA7DF3
:10F42C0043EA024394F8372043EA0223A36036F000
:10F43C00020317D1124B44F00201D3F858216AB9D8
:10F44C00626842F4004262602160C3F85841D3F80C
:10F45C00402142F02002C3F8402108E013682360E9
:10F46C00116004E0032E204604D1FFF72DFF204647
:10F47C00BDE8F88FBDE8F88FB8F1000FB0D0A5E764
:10F48C0000022E40F8B590F83430044613F0FD0F0E
:10F49C0068D00022614850F822309100DE0711D468
:10F4AC0023F01F039C4207D123680B500AE021F084
:10F4BC001F018C4204D00B461968CD0702D4F6E725
:10F4CC00216819600132202AE5D1236BB4F844601D
:10F4DC001B7D94F84A70022BB4F8463007D1504982
:10F4EC00FF2B25D85A5CD21B5A543344F8E71A46E2
:10F4FC00B4F848E094F84B5049491F2A18D80EEB41
:10F50C00C2033244C85C03F1020CC01BC85411F88E
:10F51C000C00401B01F80C0003F1030C043311F830
:10F52C000C00401B01F80C00C85C401BC854E4E7FD
:10F53C003C4B1D686DB3AB6A2E6A9C4201D03546BC
:10F54C00F8E72846FFF756FA236933F01F0203D079
:10F55C009D42F4D01B68F8E79D42F0D0284601F09C
:10F56C0017FFECE7036823F01F0398421FD12E4BC3
:10F57C00D3F8402122F02002C3F84021D3F84421D3
:10F58C0012F40042FAD1284BC3F85821274B1D68BE
:10F59C006DBB206930F01F0304D0056801F0F8FE44
:10F5AC002846F7E72046BDE8F84001F0E1BE1A68AE
:10F5BC0022F01F02944201D01346F8E7626812044D
:10F5CC0003D55A6842F400425A6022681A60164BFE
:10F5DC00D3F8402142F04002C3F84021D3F8442133
:10F5EC009706FBD52022104BC3F84421CEE7AB6A1B
:10F5FC002E6A9C4201D03546CAE72846FFF7E8F947
:10F60C00236933F01F0203D09D42F4D01B68F8E746
:10F61C009D42F0D0284601F0BBFEECE700400020F4
:10F62C005A6800202866002000022E402066002028
:10F63C000023064A8360436013680BB9106070475F
:10F64C005A680AB11346FBE75860704714660020ED
:10F65C00F7B505460F46164601F072FE0446002823
:10F66C0039D02422002108F0D5F92575082300256E
:10F67C00E675204665752A46A775294600932B46E4
:10F68C000195FFF75DFE0646206020B9204601F08B
:10F69C005FFE304620E001F083FE22680F4B2061B4
:10F6AC002046D36301230E4982F835300D4A13707E
:10F6BC004FF400230C4A81E80C002B460B4AFFF751
:10F6CC0017FB0B4A13680BB9146004E09A680AB173
:10F6DC001346FBE79C60204603B0F0BD51D10000FF
:10F6EC00C06000209E72002080060001C0580020DF
:10F6FC00A4660020F0B50E695EB3D76A18B1335C0E
:10F70C000133DBB200E003461FB37A78032A20D121
:10F71C00335400253A7803EB52013129C2BFC3F1AF
:10F72C0032025200D2B2A91CCCB2A24206EB0304A4
:10F73C0007D9302B0D4604D80133795CDBB2E1706C
:10F74C00F1E70022E2700130C0B2022801D8335434
:10F75C00F9E7F0BD2DE9F04F2E4F85B00646002598
:10F76C003C68DFF8B8800397DCB1A268BAB9B8F886
:10F77C00003020462168093B0093274BD1F80090BC
:10F78C003146C84750B163680DB16B6001E0039A14
:10F79C0013600023A6606360F46038E0254664685B
:10F7AC00E2E71E4B1E4DB3F80080A84409354545D1
:10F7BC002DD26B7895F800A0042B26D1BAF1090F45
:10F7CC0023D1039B4FF00009C5EB080B1C68E4B177
:10F7DC00A368C3B923680122CDF800B031461B6879
:10F7EC0020461F462B46B84760B16368B9F1000F3D
:10F7FC0002D0C9F8043001E0039A1360F368636027
:10F80C00F460A660A1466468E1E75544CFE705B013
:10F81C00BDE8F08F14660020C9580020B0670020A6
:10F82C00C0580020084B094A10B5116818780130EF
:10F83C000A46802828BF012022B1547DA042F6D070
:10F84C009268F9E7187010BDA1720020A466002020
:10F85C002DE9F0410746C06B28B1036839465B6857
:10F86C00BDE8F0411847BB6A0B268E4D1C6B237EFE
:10F87C000E2B00F21581DFE813F00F0029003E007B
:10F88C005900650074008A009300A900B300C900F8
:10F89C00D000DD00F6000B012168824B4A68D87954
:10F8AC0022F0FF6323F4E02343EA00434B60FFF7AD
:10F8BC00B9FF002300047C491A4640F4A0604B6059
:10F8CC0008602046FFF714FA0123DEE076494FF476
:10F8DC00901520684B886375426822F07F021343B1
:10F8EC00704A43602046714B81E828000023FFF7E3
:10F8FC00FFF90223C9E02B7963766B79A376AB7998
:10F90C00E3766A7A2B7A43EA0223E383EA7AAB7AC8
:10F91C0043EA02232384A97BEB7B2A7C6B700B4389
:10F92C0029701343AA7076D0032357E05E496048D0
:10F93C00604B614A81E8090000232046FFF7D8F9A3
:10F94C000423A2E02B79032B65D96B79032B62D1AD
:10F95C00EA79AB7943EA022363842B78E3B105237C
:10F96C003CE0504A608C12F8043B4F491B0443F0B6
:10F97C00407343F4D0630B6040F0FF63204643F4C4
:10F98C0080234B600023FFF7B3F906237DE03A4652
:10F99C0021460020FFF7AEFE6B78E3B107231DE094
:10F9AC00404A608C537804323F491B0443F0407347
:10F9BC0043F4D0630B6040F0FF63204643F4802394
:10F9CC004B600023FFF794F908235EE03A4621468A
:10F9DC000120FFF78FFEAB78EBB10923237646E7C6
:10F9EC00304A608C937804322F491B0443F04073E7
:10F9FC0043F4D0630B6040F0FF63204643F4802354
:10FA0C004B600023FFF774F90A233EE03A46214687
:10FA1C000220FFF76FFE267629E723494FF41023C7
:10FA2C00264A204681E80C0000231E4AFFF760F9A5
:10FA3C000C232AE01B4A2046D1789378204A43EACB
:10FA4C0001231949B3F5006F88BF4FF4006313808D
:10FA5C0013881A4A1B040A604B600023114AFFF7F3
:10FA6C0047F90D2311E00F4B20460F49DA79227725
:10FA7C001A7A62775B791B0443F410630B600023E2
:10FA8C001A464B60FFF734F90E232376BDE8F0815C
:10FA9C002046FFF75FFE0F2300222376094B1A70D6
:10FAAC00BDE8F081C0580020C06000208006000135
:10FABC00800600030000FC07C458002080060002EA
:10FACC00B06700209E720020F8B5054600282FD0A4
:10FADC00C4680027174E54B1236820461B69984709
:10FAEC0063683268A760626034601C46F3E76C6838
:10FAFC002CB1A66B2046FFF7C5FC3446F8E7286806
:10FB0C00FFF7C0FC0C4A136893B1AB420DD1AB6844
:10FB1C000CB9136000E0A360286908B101F04EFC39
:10FB2C002846BDE8F84001F013BC1C469B68EBE787
:10FB3C00F8BD00BF14660020A4660020F8B5054689
:10FB4C0000F1100400F12006002754F8040F20B136
:10FB5C000368A968DB6998472760B442F5D1F8BD02
:10FB6C00406910B103681B6A1847704710B5CC0880
:10FB7C0011F0070100EB040317BF005D08460841B4
:10FB8C00013318BFC1F10801914205D213F8014BA2
:10FB9C008C4008312043F7E707D91F2A9FBF012368
:10FBAC0003FA02F202F1FF32104010BD2DE9F04FC2
:10FBBC00012A87B004460F461D46DDF840E001D00F
:10FBCC000020FAE0BEF1180FFAD91B795A1E012A4F
:10FBDC00F6D86A79032AF3D1AA79012A02D1EA79F3
:10FBEC00012AEDD06A7A082AEAD9A97A2129E7D123
:10FBFC0095F80EC0BCF1000FE2D00620032111FBDA
:10FC0C000C018A42DCD102F10906B645D8D3002199
:10FC1C0001EB4100284490F80F80B8F1220F0AD173
:10FC2C0090F811C0017C41EA0C21B1F5487FA4F891
:10FC3C00D01304D9C4E701316145E9D3C0E70721EA
:10FC4C0011FB03618E45BBD3012B22D1A95D072982
:10FC5C00B6D12A44917A0529B2D1117B0329AFD1AF
:10FC6C0092F80EE0567BD07A46EA0E2692F80FE018
:10FC7C0010F00F02A4D000F0F0008028A0D138467C
:10FC8C008DE84040FFF75CFB0023E0602361A68415
:10FC9C0077E0AB5D072B93D1AB189A7A052A8FD1FD
:10FCAC001A7B032A8CD1997B5A7B93F80BA042EADE
:10FCBC00012BDA7B1AF00F01049281D01A7C072AEF
:10FCCC007FF47EAF5A7C052A7FF47AAF93F81390B9
:10FCDC00B9F1030F7FF474AF1A7D9E7C93F81580F5
:10FCEC009B7D42EA082816F00F0205933FF468AF9B
:10FCFC000AF0F003802B03931ED116F0F00A7FF468
:10FD0C005FAF049B0A46CDF800B0494601933846D4
:10FD1C000123FFF715FB059BE06032460193494632
:10FD2C00CDF8008053463846FFF70AFBA4F824B000
:10FD3C002061A4F8268021E0039B002B7FF440AFC8
:10FD4C0006F0F006802E7FF43BAF059B4946CDF8BC
:10FD5C000080384601930123FFF7F2FA049BE06020
:10FD6C00524601934946CDF800B03846039BFFF745
:10FD7C00E7FAA4F824802061A4F826B02369104A7D
:10FD8C00DA63E36838460F4A0F49DA630023B4F8A4
:10FD9C00D0236361A361E3612362AB7884F8A4365A
:10FDAC00AB78A16204F1280143EA024304F130026A
:10FDBC00E3622346FEF79CFF012007B0BDE8F08FFD
:10FDCC004DD7000087DC00008106002210B50446E8
:10FDDC00032100F5787001F006FB04F5A060052105
:10FDEC0001F00EFB04F5C860012101F02BFB20464D
:10FDFC00BDE81040FFF71CBC70B504460D46114819
:10FE0C00114909F0D2F8D4F87836EA6A60699A4256
:10FE1C0002BF94F8753623F0010384F87536D4F8D4
:10FE2C007C36EA6A9A4202BF94F8753623F00203D4
:10FE3C0084F8753628B1036829469B68BDE8704084
:10FE4C00184770BD003000205C2C00200146C06BB0
:10FE5C0008B1FFF7D1BF70470023064A436013680F
:10FE6C000BB9106070475A680AB11346FBE758602B
:10FE7C00704700BFD0660020F8B50B4B05460E4608
:10FE8C001C687CB123682946AA6820461F68334643
:10FE9C00B84728B1022805D1012385F8803601E046
:10FEAC006468EEE72046F8BDD06600202DE9F047E7
:10FEBC00002400F13005B0F8D083074626462146D1
:10FECC00A844A1464FF0010A80F8D243454501D31E
:10FEDC0000224FE02B78FE2B02D105F20115F5E73D
:10FEEC0003F00302022A08D0032A0AD0012A0DBF0C
:10FEFC006A7801350022023506E0B5F80120033599
:10FF0C0002E0D5F8012005354545E1D803F0FC03A6
:10FF1C00842B14D008D8082B14D0802B28D0042B79
:10FF2C00D4D11FFA82F9D1E7A02B0DD002D8902B97
:10FF3C001ED0CBE7B02B1BD0C02B14D0C6E787F854
:10FF4C00D2A3C3E791B2C1E75EB9032C09D841EA49
:10FF5C0009413846FFF790FF07EB84030134E4B204
:10FF6C005861013603E00EB93146AFE7013EF6B2F7
:10FF7C000021ABE7032C06D8231D013407EB8303C8
:10FF8C00E4B25A60F6E7BDE8F087000070B50446AD
:10FF9C0040690D4620B96A6B1D4B9A4237D105E07A
:10FFAC000368DB6898470028F5D070BDB4F8D033EF
:10FFBC002A6B9A422BD12046FFF778FF2346A28C5E
:10FFCC0004F55471E068FEF7FAFE2346A28C04F5A2
:10FFDC006471E068FEF7F3FEA06840F24C53C28BEC
:10FFEC009A4214D1038CB3F51A7F03D040F22F42FE
:04FFFC0093420CD14F
:02000004600199
:10000000074B04F12801074AA3624FF48023E362FF
:100010002346BDE87040FEF771BE70BD8106002228
:100020002109F403503100202DE9F04FB0F8D0330E
:10003000002400F13009A3B0A046A3464B44274654
:10004000A2460990159116A81192002130220F9313
:1000500007F0E6FC059404940E9408940D94039420
:1000600007940C940F9B994580F0668199F80030B5
:10007000FE2B04D199F8013003339944F2E703F0E1
:100080000302022A0BD0032A0ED0012A0DBF99F8D1
:10009000015009F10109002509F1020908E0B9F848
:1000A000015009F1030903E0D9F8015009F10509EC
:1000B0000F99894500F2408103F0FC03742B3DD079
:1000C00010D8142B24D004D8042B1ED0082B3ED0DB
:1000D000C8E7242B27D0282B45D0182BC2D1ADF848
:1000E000585042E0942B2CD007D8842B2CD0902B46
:1000F00000F01A81802BB5D16BE0B02B00F0148199
:10010000C02B50D0A02BADD131E0ABB20893A9E702
:10011000012A01D16BB202E0022A02D12BB2049370
:10012000A0E704959EE7012A01D16BB202E0022A02
:1001300002D12BB2059395E7059593E71FFA85FB4E
:1001400090E71FFA85F88DE7EBB20D938AE7172F3A
:1001500088D81F2D86D922AA7B1C02EB4706DFB266
:1001600026F8305C7EE7ADF85A50FF277AE7039B0C
:10017000A3B9089ABDF8583043EA02430C93079B91
:10018000032B9DBF099A013307994FF0000A9FBFC7
:10019000DBB202EB81020793D2F814A0039B013378
:1001A000DBB20393C0E0039B002B00F0BD80013B5A
:1001B00013F0FF03039340F0B780BAF1000F00F093
:1001C000B380DAF8003050464FF0000A9B69984738
:1001D000AAE0099B93F8D2332BB19DF854300D9AC5
:1001E0009A4240F0A18015F00103069340F08D8003
:1001F000BAF1000F00F08980DAF800305046059A15
:100200000C9900922A461B691E46049BB04715F0C4
:10021000020503D1089B26461F0474E0182F06D957
:10022000BDF85A300126BDF85850069319E0B8F1D0
:10023000010F11D9012F0FD818BF0E9B4FF00106E7
:100240000CBFBDF8585003F47F454FF6FF7318BF3D
:1002500005F58075069304E0069E4FF6FF7335465C
:100260000693089B01220A941B0412930BF1FF339F
:10027000109302FA03F3139302FA0BF35B42149305
:1002800000230B930B9B43453FD226B1069B9D4217
:100290000BD26F1C0AE06F1C22AB172F03EB450536
:1002A00028BF172735F8305C00E02F46129B5A46CE
:1002B0000A992B4311980E93FFF75EFC049B0246AC
:1002C000002BDAF8003007DA10991E2904D81399A8
:1002D00008421CBF14990A435B6950460E9998471F
:1002E0000A9B0E953D465B440A930B9B01330B938F
:1002F000C8E75A4631461198FFF73EFC049B8342FB
:1003000006DD5E4401354545F3D308FB0B440BE0A5
:10031000059B8342F5DBDAF8003040EA0701012251
:1003200050465B699847ECE74FF000030027ADF8B3
:100330005830ADF85A3095E623B0BDE8F08F70B56F
:1003400004464069CD6A0E6B18B103685B68984734
:1003500048B994F8D233A3B933462A464FF4807192
:100360002046FFF761FE04F56473A28CE0689D42AD
:1003700023460CBF294604F55471BDE87040FEF7D2
:1003800024BD012EEFD92978731E6A1C41F48071B7
:10039000E6E70146C06B08B1FFF7D1BF704770B503
:1003A000044600F55876002594F89E339D4206D207
:1003B00056F8040F08B1FFF78DFB0135F4E700256F
:1003C0001C2204F55970C4F8A453294684F89E539E
:1003D000C4F86053C4F8805384F8A15384F8A2533E
:1003E000C4F8A75307F01CFB84F8AB5384F8AC5354
:1003F00084F8AD5384F8AE5384F8AF5384F8B05307
:1004000084F8B15384F8B25384F8B35370BD00003C
:10041000F8B504460D460AB10020F8BD4D49C0F8B4
:1004200038134D49C0F81813A96921F07F4121F014
:10043000FF01B1F5106FEFD1E97E0229ECD880F809
:10044000982303F1100206981030811A19440F29DD
:1004500057D912F8101C092951D112F80F1C042980
:100460004DD112F80C1C012949D112F80B1C092995
:1004700045D112F8096C022E41D812F8071C072941
:100480003DD112F8061C052939D112F8051C01F0DE
:10049000F001802933D112F8041C03292FD112F85E
:1004A000031C01292BD112F8021C41BB94F89813AC
:1004B00012F80DEC12F80E7C31B984F8997312F829
:1004C0000D6C84F89A6309E094F899C3674518D1D4
:1004D00094F89B73B7420FD284F89AE312F8096C30
:1004E00084F89B6312F8056C06F00F0684F89C6391
:1004F00012F8016C84F89D63013184F8981310326E
:10050000A3E794F89833002B86D000211C2204F531
:100510005970C4F8A41384F89E13C4F86013C4F887
:10052000801384F8A11384F8A213C4F8A71307F06A
:1005300077FA0A4B04F5627204F55671C4F8583321
:100540004FF480132846C4F85C332346FEF7D6FBED
:100550000120F8BDAA2C0020C02C0020A0060029F4
:1005600010B5044607210C3000F036FF04F59070FA
:10057000022100F03EFF04F5F070042100F046FF78
:1005800004F53870012100F063FF2046BDE81040FB
:10059000FFF754B870B504460E4601B390F89E3389
:1005A00099421CD890F8A123012592B90C4B80F8F0
:1005B000A153B540C0F858330346C4F85C1300F5A6
:1005C00056718068FEF79AFB94F8AB3323EA050571
:1005D00003E08D4090F8AB331D4384F8AB5370BDFE
:1005E0002303080070B590F89E3304460E468B42F4
:1005F00024D390F8A1330125D3B9002980F8A15361
:1006000000F5617205FA06F514BFA323A023C0F814
:10061000583341F4802300F55671C0F85C3303462B
:100620008068FEF76BFB94F8AC3323EA050503E022
:100630008D4090F8AC331D4384F8AC5370BD00007E
:100640002DE9F04104460E4607F00CFA04F5467316
:100650009E4219D194F8B373B7B30125A84694F814
:100660009E339D4209D808FA05F33B4203D0294640
:100670002046FFF7B7FF0135F1E7304644F6206129
:10068000BDE8F041FEF786BA04F54E739E421BD1D9
:1006900094F8A263C6B1751E254495F8A433082BBF
:1006A00012D1A368002794F8A303324684F8A273FA
:1006B00004EB8604597DFEF7D1FF044BC4F86003B8
:1006C0001F70092385F8A433BDE8F0819D720020D6
:1006D00070B504460E4601B390F89E3399421CD87B
:1006E00090F8A123012592B90C4B80F8A153B54095
:1006F000C0F858330346C4F85C1300F5567180689F
:10070000FEF7FCFA94F8AD3323EA050503E08D40CB
:1007100090F8AD331D4384F8AD5370BD2301100034
:1007200070B504460E4601B390F89E3399421CD82A
:1007300090F8A123012592B90C4B80F8A153B54044
:10074000C0F858330346C4F85C1300F5567180684E
:10075000FEF7D4FA94F8AE3323EA050503E08D40A2
:1007600090F8AE331D4384F8AE5370BD23011100E1
:1007700070B504460E4601B390F89E3399421CD8DA
:1007800090F8A123012592B90C4B80F8A153B540F4
:10079000C0F858330346C4F85C1300F556718068FE
:1007A000FEF7ACFA94F8AF3323EA050503E08D4079
:1007B00090F8AF331D4384F8AF5370BD230112008E
:1007C00070B504460E4601B390F89E3399421CD88A
:1007D00090F8A123012592B90C4B80F8A153B540A4
:1007E000C0F858330346C4F85C1300F556718068AE
:1007F000FEF784FA94F8B03323EA050503E08D4050
:1008000090F8B0331D4384F8B05370BD230113003A
:1008100070B504460E4601B390F89E3399421CD839
:1008200090F8A123012592B90C4B80F8A153B54053
:10083000C0F858330346C4F85C1300F5567180685D
:10084000FEF75CFA94F8B13323EA050503E08D4026
:1008500090F8B1331D4384F8B15370BD23011400E7
:1008600070B504460E4601B390F89E3399421CD8E9
:1008700090F8A123012592B90C4B80F8A153B54003
:10088000C0F858330346C4F85C1300F5567180680D
:10089000FEF734FA94F8B23323EA050503E08D40FD
:1008A00090F8B2331D4384F8B25370BD23030400A3
:1008B00010B540F6013390F89A1390F89923044646
:1008C00043EA014300F55671C0F85C230022C0F8EA
:1008D000583303468068FEF711FA012384F8A133E8
:1008E00010BD70B505460024012695F89E339C4244
:1008F0000BD806FA04F3D5F88023134203D021461F
:100900002846FFF76FFE0134EFE72B4605F56071CF
:10091000D5F860030122BDE87040FEF756BA0146E3
:10092000C06B08B1FFF7DDBF704738B590F8B3333F
:1009300004460D462BB944F6206100F54670FEF7DB
:1009400029F9012194F8B333A940194384F8B3136A
:1009500038BD012303FA01F190F8B33323EA010112
:1009600080F8B313704700002DE9F04105461446A6
:100970000E4600297AD090F89E33994276D84F1EC1
:10098000074497F8A423092A70D8DFE802F0050588
:10099000121212121236515BE40767D5022387F850
:1009A000A433FFF7C2FF31462846BDE8F041FFF708
:1009B0008FBEE0071DD50132D2B2072A87F8A423E3
:1009C00054D12B4B197800294DD12A490978002997
:1009D00049D10121284619703146FFF7BAFF314647
:1009E00087F8A4232846FFF73BFF85F8A263BDE8FC
:1009F000F0812846FFF7ADFF33E0A10718D5314657
:100A0000FFF706FF0823A20587F8A43305D414F4E2
:100A1000806F0CBF0023022300E0012385F8A3337D
:100A200005F54E7046F2A811BDE8F041FEF7B2B8E8
:100A300014F001041AD131462846FFF749FE0C4B49
:100A40001C700EE014F0010410D100EB8108D8F8FE
:100A50006003FFF73FF8C8F8604331462846FFF7C8
:100A600037FE012300E0062387F8A433BDE8F081B8
:100A70009D7200209E72002037B50B4600225F4D0C
:100A8000044680F8A1235A6B098FAA4222D05C4DFC
:100A9000AA4202D0A32A43D13BE090F88A3380F8DF
:100AA0009E3390F88B3380F89F3390F88D3380F825
:100AB000A03390F89833012B01D9FFF7F9FE0125F7
:100AC00094F89E339D422BD829462046FFF762FDBD
:100AD0000135F5E790F89E33994225D1D0F860337F
:100AE00013BB90F89D33012590F89C2303210193BB
:100AF0002B4600958068FEF729FC4268414A234650
:100B0000C4F8600304F56071C2632A46FEF75DF91C
:100B100006E01A6B042A07D1DB6A1A68FFF724FF84
:100B200094F8A133002B67D194F8AB1349B191FA33
:100B3000A1F12046B1FA81F103B0BDE83040FFF7E2
:100B400029BD94F8AD1349B191FAA1F12046B1FA4B
:100B500081F103B0BDE83040FFF7BABD94F8AE13A1
:100B600049B191FAA1F12046B1FA81F103B0BDE893
:100B70003040FFF7D5BD94F8AF1349B191FAA1F118
:100B80002046B1FA81F103B0BDE83040FFF7F0BD77
:100B900094F8B01349B191FAA1F12046B1FA81F16C
:100BA00003B0BDE83040FFF70BBE94F8B11349B174
:100BB00091FAA1F12046B1FA81F103B0BDE83040CD
:100BC000FFF726BE94F8AC1349B191FAA1F1204683
:100BD000B1FA81F103B0BDE83040FFF703BD94F8EE
:100BE000B21349B191FAA1F12046B1FA81F103B0F3
:100BF000BDE83040FFF734BE03B030BD230308002A
:100C0000A006002913E20000704790F88432013BEF
:100C1000DBB280F8843203B943617047A0F10C0065
:100C2000FFF7F3BF0123C0F8801280F8853200235C
:100C300080F886327047A0F10C00FFF7F3BFF8B5DB
:100C40000B0C04460E461B04B3F17F4F3BD089B218
:100C5000002938D0012390F887E200F28620037043
:100C60000023DDB275451CD230F8027F0133B94252
:100C7000F7D142BBD4F87C3213B1D4F88002984744
:100C800094F88732013BDBB284F887329D421AD256
:100C900004EB45020135B2F88A12EDB2A2F88812CF
:100CA000F4E782B1D4F8783213B1D4F880029847CF
:100CB00094F88732032B9FBF5A1C03F5A27384F864
:100CC000872224F81360F8BDA0F10C00FFF7B7BF2E
:100CD000002343627047A0F11800FFF7F9BF8B783B
:100CE000834210D0CB7883420DD00B7983420AD057
:100CF0004B79834207D08B79834204D0CB791B1A7E
:100D000058425841704701207047000038B50D46E1
:100D10000F220749284608F0B0FE044630B92A469B
:100D20000449054808F047F9204638BD012038BD80
:100D3000CF2C0020DF2C002000300020A0F1180074
:100D4000FFF7E4BF012A73B504460D4646D1069A63
:100D5000182A43D91879002850D05A79032A3DD14E
:100D60009A79012A3AD1DA79012A37D15A7A092AAD
:100D700034D19A7A212A31D19A7C072A2ED1DA7C71
:100D8000052A2BD11A7D02F0F001802926D112F01C
:100D90000F0221D0597D032920D1D88A083838285C
:100DA0001CD81B7E08262846019301230096FEF7D7
:100DB000CDFA134AA0652346C26304F164013246AA
:100DC000FEF703F840F2D943EA8B9A424FF0000352
:100DD00006D140F6213205E010460FE000200DE07C
:100DE00040F62122E26504F15C01236600222346DD
:100DF0002846FDF783FF012084F8910202B070BD00
:100E00009DEB0000F8B505460E4618481F461849E8
:100E1000144608F0D0F86B6A0BB1B34221D168696F
:100E2000F8B9AA6802BB04F45F43B3F5A06F1AD106
:100E300014F0400018D06FB10F220E49384608F068
:100E40001CFE044630B90C49084808F0B4F86C623E
:100E50002046F8BD0949054808F0ADF86E6201204A
:100E6000F8BD0020F8BD1046F8BD00BF00300020DE
:100E70001F2D0020CF2C0020502D0020852D00207C
:100E8000A0F11800FFF7BEBF90F8853210B50446F8
:100E9000E3B190F88632B3B9D0F87C3283B194F8DC
:100EA00087326BB1013BD4F87C22D4F88002DBB2EC
:100EB00084F8873203F5A27334F813109047EEE7F5
:100EC000002384F88732002384F8853210BDA0F116
:100ED0000C00FFF7D9BF00000B498B4202D00B4931
:100EE0008B420ED1836893420BD1416909B18A428A
:100EF00007D1436190F88432013380F884320120B5
:100F000070470020704700BF8000010001000C0006
:100F1000A0F10C00FFF7E0BF10B5044602218030BD
:100F200000F067FA042104F5A07000F06FFA0121C7
:100F300004F5107000F08CFA2046FEF77FFB04F1F8
:100F40000C00FEF78FFF04F11800FDF707FD0023EA
:100F500084F8903210BD0346806868B193F89122FE
:100F600052B940F621311A66D965012183F89112F0
:100F700003F15C01FDF7C2BE012283F890227047A5
:100F8000002310B580F8913240F621334A6B0446B5
:100F90009A4210D10A6B72B940F62123026600F121
:100FA0005C01C3650123BDE8104080F8913203461F
:100FB0008068FDF7A3BE94F890322BB12046FFF76E
:100FC000CAFF002384F8903210BD7047F0B5560672
:100FD00019D500242B4D062606FB04F35F5BBA42AD
:100FE0000ED190F8782012F0010F264A134401D058
:100FF0001A7944E05A88150641D502F07F0202E0D2
:101000000134102CE8D100231F4D35F823609C00DB
:10101000B24203D11C4B23449A7830E00133192BA0
:10102000F3D154062AD490F8783011F0220F4FF003
:10103000000018BF42F040029B07144B48BF82F0EB
:10104000400233F81040A24208D111F0110F02D033
:1010500000F01F0213E000F120020AE001306028D6
:10106000EFD100230A4931F81300824203D103F182
:10107000A00292B203E00133602BF4D100221046AB
:10108000F0BD00BFA81C0020441C00202820002028
:10109000E820002010B5044680F86E1080F86F201C
:1010A000FFF794FFA36CA4F86C0013B1BDE81040E7
:1010B0001847FFF78AFF10BD0346806850B1064A03
:1010C00003F15C01DA654FF480321A6603F17802AD
:1010D000FDF714BE704700BF2109000290F8783078
:1010E00010B403F001048C4207D061F300035DF8F3
:1010F000044B80F87830FFF7DFBF5DF8044B704792
:1011000090F8783010B4C3F340048C4207D061F3F8
:1011100041035DF8044B80F87830FFF7CDBF5DF8F0
:10112000044B704790F8783010B4C3F380048C42BD
:1011300007D061F382035DF8044B80F87830FFF745
:10114000BBBF5DF8044B704710B5532A044680F8C6
:101150006E1084F86F2009D190F8781001F0010129
:10116000BDE8104081F00101FFF7B8BF392A09D16D
:1011700090F8781081F00201BDE81040C1F3400101
:10118000FFF7BEBF472A09D190F8781081F004011B
:10119000BDE81040C1F38001FFF7C4BFFFF716FFA1
:1011A000E36CA4F86C0013B1BDE810401847FFF7DA
:1011B0000CFF10BD2DE9F041044600F1710600F16D
:1011C000770700F1640816F8015F032D0ED9414638
:1011D0002846FFF784FD48B92A4694F87010204647
:1011E000FFF7B2FF636D0BB128469847B742EAD1CB
:1011F000636D33B904F1650604F16B0704F17008FF
:101200001CE00025012606FA05F394F87020DBB2F5
:10121000134208D094F86420134204D105F167000A
:10122000636DC0B298470135082DECD1E2E7414625
:101230002846FFF754FD58B3B74204D016F8015FB3
:10124000032DF9D9F3E7236D63B92146A06D082278
:1012500051F8643F23674B6863672346BDE8F0415C
:10126000FDF7B3BD0025012606FA05F394F87020BA
:10127000DBB2134208D194F86420134204D005F184
:101280006700236DC0B298470135082DECD1DCE72B
:101290002A4694F864102046FFF7FCFE236D002BCD
:1012A000CAD028469847C7E70146C06B08B1FFF788
:1012B00081BF70472DE9F8430D4604461F4990460B
:1012C0001F4807F078FE2B78012B29D104F1710714
:1012D000022604F16409B0450ADD17F8012F032A3C
:1012E00004D949461046FFF7FAFCE0B10136F2E7AF
:1012F0006E1C05F1070804F17009374617F8012F35
:10130000032A04D949461046FFF7E9FC88B1B845DD
:10131000F4D133680120236773686367BDE8F883FD
:101320000020BDE8F88394F870102046FFF70CFF0A
:10133000DCE769782046FFF7ADFEE8E7AF2D002037
:1013400000300020A0F11800FFF7B4BF024B18686E
:1013500008B102681A6070470C660020024B1A68D8
:1013600018600260704700BF0C660020024B1868CE
:1013700008B102681A60704700660020024B1A68C4
:1013800018600260704700BF00660020024B1868BA
:1013900008B102681A60704718660020024B1A688C
:1013A00018600260704700BF18660020054B18687F
:1013B00030B102681A600023037043708370C370F9
:1013C000704700BF10660020024B1A681860026068
:1013D000704700BF10660020242310B503FB0101F5
:1013E00004468C4204D220462434FFF7B7FFF8E7C6
:1013F00010BD602310B503FB010104468C4204D2EA
:1014000020466034FFF7BAFFF8E710BD10B500EBD7
:10141000811104468C4204D220464034FFF7BEFFBF
:10142000F8E710BD08B501210648FFF7D5FF0121F7
:101430000548FFF7DEFF04210448BDE80840FFF738
:10144000E5BF00BFDC650020A04100202042002055
:10145000352310B503FB010104468C4204D220461B
:101460003534FFF7B1FFF8E710BD0023C360036117
:10147000704770B5B0F84250044690F85230AD084D
:1014800003F0FF0243B1EBB2816B920080F852305F
:1014900003460069FDF799FC94F8533003F0FF020E
:1014A00053B1EDB22346E16B920084F853502069AA
:1014B000BDE87040FDF789BC70BD0000012AF7B59A
:1014C00004460D4640F0C6801A78092A40F0C280D2
:1014D0005A78042A40F0BE805979012902D19A79BC
:1014E000032A04D00239102940F2B4800021089860
:1014F00000221844093384F8542084F85520984277
:1015000051D91F78032F40F2A580DE19B042C0F0F8
:10151000A1805A78042A46D00B2A44D0242A0DD11F
:101520009A78511E032902D801213346E7E7F12AB0
:1015300040F09080DB78022BF6D08BE0052A2FD18B
:10154000062F40F28780DA78023A012A00F2828080
:101550009A7812F0F00713D0802F7BD194F8547052
:10156000002FE2D102F00F0284F85420DA7884F8D8
:1015700056205A791B7943EA0223A4F84030D4E775
:1015800094F85570002FD0D184F85520DA7884F87B
:1015900057205A791B7943EA0223A4F84230C4E762
:1015A000252AC2D056E0002954D094F85420E2B144
:1015B000B4F84030B4F84A10994216D30020009392
:1015C00094F85610012301902846FDF7BFFEE06015
:1015D00068B1234A2346616BC263B4F84020FDF72B
:1015E000F4FB012384F8483001E00023E36094F821
:1015F0005520BAB1B4F84230B4F84A10994211D328
:10160000002694F8571028468DE848003346FDF729
:101610009DFE206140B1134BC36384F8526084F88F
:10162000536001E0002323610023A4F84E30A4F8A6
:10163000503084F8593084F85A3084F85B3084F89C
:101640005C30A4F88031E36833B92069003018BFFA
:10165000012002E0002000E0012003B0F0BD00BF47
:1016600059F0000083F0000010B50446032100F596
:10167000F070FFF7BEFE04F540700721FFF7C6FECD
:1016800004F598600121FFF7E3FE00232046C4F82B
:101690008431C4F88831C4F88C31C4F89031C4F86E
:1016A0009431C4F89831C4F89C31C4F8A031C4F81E
:1016B000A431C4F8A831C4F8AC31C4F8B031C4F8CE
:1016C000B431C4F8B831C4F8BC31C4F8C031C4F87E
:1016D000C431C4F8C831C4F8CC31C4F8D031A4F84E
:1016E0004E30A4F85030E3602361BDE81040FDF7B0
:1016F000A5BF8A680B6BC2F30E42991AB0F84E3040
:10170000B0F85020890870B50446002088420ED0F9
:10171000656B55F8205045B1B4F84C600133B342C5
:1017200028BF0023666C46F823500130EEE7934251
:10173000A4F85020A4F84E3024BFB4F84C1052182E
:10174000013AD31AB4F84020B3EB920F06D32346E4
:10175000616BE068FDF739FB012300E0002384F8AA
:10176000483070BD0146C06B08B1FFF7C2BF70477B
:10177000CB6A826B934203D1002380F852307047CA
:10178000C26B934202D1002380F853307047014668
:10179000C06B08B1FFF7ECBF704790F84030013BD9
:1017A000DBB280F8403003B983607047012380F8D2
:1017B000423070470B0C89B2092B10B50FD101399B
:1017C000072924D8012390F8434003FA01F112B904
:1017D00024EA010100E0214380F8431010BD012BF1
:1017E0000FD13039082912D8DFE801F005071011B0
:1017F000111111110900426410BD826410BDC26450
:1018000010BD0C2B03D1B1F50E7F00D1026510BDC8
:1018100090F842302BB1012380F84130002380F84A
:1018200042307047002383617047A0F10C00FFF73E
:10183000F9BF000070B504460E460E4815460E4925
:1018400007F0B9FBA3690BB1B34210D1A06870B91E
:1018500005F45F43B3F5A06F0AD115F0800007D0FF
:101860000649044807F0A7FBA661012070BD0020CF
:1018700070BD00BF00300020DF2D0020172E00209B
:10188000A0F10C00FFF7D6BFC2B10B78022B17D125
:101890004B78042A80F8433091F90230436491F97F
:1018A0000330836407D991F90430052AC3641CBF4F
:1018B00091F905300365012280F8412010467047F8
:1018C00000207047A0F10C00FFF7DEBFA3F1011369
:1018D000012B0BD883680BB19A4207D190F84030A6
:1018E0008260013380F8403001207047002070474B
:1018F00010B50446FEF7B6FA04F10C00BDE810403E
:10190000FDF72CB82DE9F843089D0746164603EB72
:1019100001090C464C450ED03B68324621463846FC
:10192000DB6804F10108984730B12046099A314636
:101930004446A847EEE70120BDE8F8832DE9F041D1
:1019400005461F4602EB01080C4644450DD02B68A6
:10195000204606991E6AB8472146024628460134A9
:10196000B0470028F1D1BDE8F0810120BDE8F08149
:101970004FF0FF307047704737B505460C4606F00C
:101980001BF91C4B984202D800232B802EE069469D
:1019900007F062FB9DF806309DF80510503B9DF85E
:1019A00004209BB27F2B0BD80131C9B20C2907D878
:1019B0001F2A05D842EA411242EA43239BB200E0C3
:1019C00000239DF802102B8017299DF801209DF817
:1019D00000300AD83B2A08D83B2B06D8520142EAED
:1019E000C12242EA53039BB200E00023238003B0EC
:1019F00030BD00BFFFA5CE120A46D0F8841400B552
:101A00008FB051B1002368468DF800308DF8013059
:101A10008DF8023002F0BAFB0DE0D0F8880450B126
:101A20008DF831100B468DF832108DF833100146C9
:101A3000684600F013FE0FB05DF804FB0A46D0F8CC
:101A4000841400B58FB071B1002368468DF8003062
:101A50008DF801308DF8023002F098FBA8B168468D
:101A600002F0D1FA11E0D0F8880470B18DF831108D
:101A70000B468DF832108DF833100146684600F0A1
:101A8000EDFD10B1684600F0BDFE0FB05DF804FB3F
:101A90000A46D0F8841400B58FB079B100236846A7
:101AA0008DF800308DF801308DF80230012302F0FE
:101AB0006DFBA8B1684603F0DFF911E0D0F88804A7
:101AC00070B18DF8311001238DF832108DF833107C
:101AD0000146684600F0C2FD10B1684600F04FFEB6
:101AE0000FB05DF804FB10B5D0F884448EB00A4600
:101AF0006CB1002304F5896168468DF800308DF8DB
:101B000001308DF80230012302F002FC10E0D0F821
:101B1000881461B1012301F5896168468DF831406F
:101B20008DF832408DF8334000F0B8FF00E00846F1
:101B30000EB010BDD0F8843430B515468FB0ABB1BF
:101B4000002203F5896468468DF8002013468DF85D
:101B500001208DF802200A46214602F0C3FAD8B1CE
:101B60002A462146684602F028FC15E0D0F8880491
:101B700090B100F589640A4668468DF831302146F7
:101B80008DF832308DF8333000F00AFD20B12A464E
:101B90002146684600F0E2FF0FB030BDD0F8803437
:101BA00033B198794FF4007303FA00F080B27047B4
:101BB000D0F8840408B1D0F83C04704703460430E0
:101BC000D3F8842410B512B1D469013C04E0D3F8F1
:101BD00088440CB1D4F83044FFF7E0FFA4FB0001C7
:101BE00010BD38B50346051DD0F8840420B1C46982
:101BF000013C03F0D9FD08E0D3F8880420B1D0F807
:101C0000304401F0BAFE00E00446241A2846FFF7EB
:101C1000C5FFA4FB000138BD38B500F59265FF2370
:101C2000044680F8C41480F8B834284605F0B8F8A3
:101C3000C4F88C54284604F08FFC30B9D4F88C14C6
:101C40002046BDE8384003F019BF002038BD70B50C
:101C500088B0064601A805AD06F29C4480E80E0057
:101C600007C885E80B00204695E80E0004F01EF931
:101C7000C6F88C442CB196F8B304B0FA80F0400951
:101C800000E0204608B070BD7FB50C4605461E48F2
:101C900005F000FCFE2C85F8CD440ED14FF000017C
:101CA000281DFFF7B9FF044685F8CC0440BB2E2061
:101CB000032105F04DFF204623E0362C4FF00000B5
:101CC0001FD8124B2E1D8DF805000293C5F8C034A5
:101CD00004AB03908DF8044085F8BD04C5F8C40436
:101CE000304685F8BC4413E90E00FFF7B0FF20B181
:101CF000D5F89014304603F0C1FE85F8CC0400E01E
:101D0000012004B070BD00BF6DF2000040787D017D
:101D100030B590F8B83485B00446FF2B04D190F864
:101D2000C414FFF779FF19E0D0F8BC14D0F8C02430
:101D30008DF8043004AB90F8B95402918DF8055039
:101D4000039213E90E00FFF782FF38B1D4F88C1428
:101D5000204605B0BDE8304003F090BE05B030BD70
:101D60002DE9F041D0F890448CB006461F460CB9DE
:101D7000002024E0236820469B699847B0F5405F27
:101D80008046F5D94FF4007007F002FD05460028A3
:101D9000EED0B8F1806F02463B46214601A802D939
:101DA00001F0AEF901E003F0DBFA0446284607F043
:101DB000F7FC002CDCD0301DFFF7AAFF01200CB08F
:101DC000BDE8F0817FB5D0F8906405460EB90020DB
:101DD00027E090F8CC2490F8CD34BAB1FE2B05D092
:101DE0003368694630469B6B98471AE03368304643
:101DF0005B6C9847421CF3D090B995F8CD34FE2B1C
:101E0000E5D103212E2005F0A3FEE0E7FE2B03D150
:101E1000064B9B689B03DAD5281DFFF779FF00E08E
:101E2000012085F8CC0404B070BD00BF00800042E2
:101E30001548164A164BC0F89424164A036000232E
:101E4000C0F8A024144AC0F88434C0F8A82407229B
:101E5000C0F88834C0F8AC24012280F89C3480F8A3
:101E6000B524292280F89D3480F8BA3480F8C8342B
:101E700080F8CC34FF2380F8B7240849084A80F85A
:101E8000CD3407F03ABC00BFF0600020000600200F
:101E9000D00500206006002000093D006BF2000024
:101EA000302F0020F0B500F1240385B005460F4621
:101EB00001AC164693E8070084E807007A01214642
:101EC000286A01F0ECFC012805D132462146286A37
:101ED00001F096FC00E0002005B0F0BD10B504460E
:101EE00000F02AFD002384F8313084F8333010BD2F
:101EF00038B50D46144600F124010022006A01F0B5
:101F00007FFC20B143892B8003890120238038BDC9
:101F100038B50D46144600F124010022006A01F094
:101F20006FFC20B1C3892B8083890120238038BDB9
:101F300038B50D4690F83110044651B9382205F0F5
:101F40006FFD40230120256284F8313084F833008E
:101F500038BD002038BD0000F0B40C784D1C202C9A
:101F600001D12946F9E71A4F116091600D460E46DE
:101F700015F8014BDCB12F2C13D01F2C24D9A4F160
:101F80002201C9B21D2903D827FA01F1C9071BD4C0
:101F900004F0BF013C2917D05C2C0DD114E02F2C8C
:101FA00005D10E4611F8014B202CF8D1F9E71E603F
:101FB0001146F0BC01F04EBB2E2C01D12946D5E7CD
:101FC000202CFBD09560F9E70020F0BC704700BFE3
:101FD000010100312DE9F84F90F8333004460E46E8
:101FE0001546DF0777D5580603D494F83130190722
:101FF0000CD5D4E90001D4E9042310EB050841F124
:1020000000094B4508BF424500D2151AA94604F104
:10201000180AB9F1000F43D0206AD4E90023D0F8A0
:10202000381401EA0208C8F3080BB8F1000F1ED1FA
:10203000134307D194F831305A064CBFD0F83434EA
:10204000E36905E094F833305B0603D5A3690133F7
:10205000A3610CE05246A16901F0EDFB00283ADBD8
:1020600005D194F8313013F0500F19D133E0276ABD
:102070004FEA5822A16997F845E40239D7F82C04B1
:1020800001FA0EF1014401EB0208BBF1000F4FD140
:10209000B9F5007F4CD3D7F81C12884504D147E02E
:1020A000C9EB0500BDE8F88FB9F5806F2AD301238D
:1020B0004FEA592B03FA0EF39A1A934528BF934619
:1020C000884512D80BEB080399420ED207F504702D
:1020D00005F08BF948B994F832304FF0FF3043F0F7
:1020E000020384F83230BDE8F88FD7F81402324684
:1020F000414603681F695B46B8470028EBD04FEAAA
:102100004B270AE0D7F81402324641460368DB68E1
:1021100098470028DFD04FF400773E44C7EB090909
:10212000D4E90023D21943F10003C4E9002370E786
:102130000022414607F5047005F07DF90028CAD059
:10214000CBF5007700EB0B0130464F4528BF4F46DB
:102150003A4605F0CBFBE0E7F7B501220DF10701A8
:1021600004468569D0E90067FFF734FF0128A561BF
:102170000CBF9DF807004FF0FF30C4E9006703B0C3
:10218000F0BD2DE9F74F1F4690F831B08369044642
:1021900016460193BBF1000F52D0D0E90089B94532
:1021A00008BF904550D056EA070302D1002383614F
:1021B00043E01BF0080F05D0D0E90401B94208BF85
:1021C00090423DD3236A16F1FF3093F845A447F1BE
:1021D000FF3100930AF1090A5FFA8AFA524607F0C2
:1021E00091FA94F833200546530603D5E3691D445C
:1021F000A56122E018F1FF30524649F1FF3107F0A6
:1022000081FA854202D358EA09030AD11BF0400F34
:1022100016BF009BE369D3F83434A36104F11808B6
:1022200009E02D1AFAE74246A169206A013D01F052
:1022300002FB002804DD002DF5D1C4E9006703E0AE
:10224000019B0020A36100E0012003B0BDE8F08FF6
:102250002DE9F04F9A4690F831308DB004460E4685
:10226000154673BB91F8313013F0500F29D00AF0A6
:102270000303012B00F08281022B40F07A810323BB
:102280000AF0080949EA03090DB32B694FF00F085A
:10229000002230460E33B3FBF8F808F102080023A1
:1022A0005FFA88F8FFF76DFF4FF0000B5F462022C2
:1022B00004A93046FFF78EFE002800F0BC802028DD
:1022C00008D0002084F8310084F8330062E14FF038
:1022D0000308E9E79DF81020110611D427B93368E7
:1022E000203B0193B369009347453CBF0137FFB2E0
:1022F00012B14FF0000BDAE7002D40F09C80E0E7D0
:10230000BBF1000F27D1474538BF0027852ACED122
:102310003822594620464FF0010B05F081FB9DF80D
:1023200011309DF8142084F8303002F03703D206C3
:1023300058BF43F0080384F83130336A2362B3692D
:1023400063623368203BA36296F83330C3F3801393
:1023500084F82C30ABE7C02A2BD19DF8113084F8DB
:102360003390980744BF49F0400384F83330DDE9E7
:102370000623C4E90423099BE361DDE90A23C4E9D8
:1023800002231DB91AF4006F9BD126E02B682A693D
:102390006B604FF00003AB819DF813309A42A8D1D7
:1023A000BDF81420AB8AD11AD1F1000B4BEB010B15
:1023B0007DE7C12A9DD12A4604A9204601F0CCF828
:1023C00008B9834673E7AA89002A7FF470AF696869
:1023D000AA6891427FF46BAFD4E71AF4884F03D117
:1023E00094F833309A0705D594F8313013F0110F73
:1023F0007FF467AF1AF4806F10D094F833309B07E6
:102400007FF55FAF002200232046FFF7BAFE0028C9
:102410003FF457AF204600F07FFC08E01AF4804FED
:1024200000F0AE802046D4E90423FFF7AAFE00287E
:102430003FF447AFA4E01AF4007F3FF442AF19F035
:10244000020F3FF43EAF002D3FF43BAF47451CD297
:10245000202204A93046FFF7BDFD50B93046D6F81A
:1024600018A000F088FA00283FF42BAFC6F818A097
:10247000ECE720287FF425AF27B93368203B019390
:10248000B36900930137FFB2E0E73822002120460C
:1024900096F8337005F0C4FA336AC7F3801708F171
:1024A000FF3A2362082384F82C705FFA8AFA84F8D2
:1024B00031300027009B6362019BA3622B68AF81D0
:1024C0006B605FFA87FBC3454FD201225946204615
:1024D000FFF7E8FC064600283FF4F3AE90F9002031
:1024E000002AFFF6EEAE2022002105F099FABBF19A
:1024F000000F1ED185233370284B84F830A086F856
:1025000001A01B687BB10DF10B020DF10E0103A8B8
:102510009847BDF80C307381BDF80E3033819DF8BB
:102520000B3033751FE045F221437381F3817382D1
:1025300019E0BBF1010F0CD169F07F03C02286F8CE
:1025400001B0327084F833302B69F370AB8AB380FA
:1025500009E0C12306F11E0B3370AA8992B969689C
:10256000AA6891420ED10137ABE7204600F0E4F9AA
:1025700010E0002B7FF4A5AE012381E602237FE665
:10258000012007E0284605F067F826F8020F5E45AF
:10259000E3D1E8E70DB0BDE8F08F00BFC4660020CE
:1025A000F0B51F4697B0002305460C4601928DF802
:1025B00051308DF852308DF85330ADF8143090F81A
:1025C00031300BB1002047E091F8313013F0500F5B
:1025D000F8D013782F2B12D1019B1A782F2A02D111
:1025E00001330193F8E7216A1AB92846FFF7A0FCE6
:1025F00032E008A8FFF79CFC0028E3D008AC01AB50
:1026000002AA01992846FFF7A7FC0028DAD0019B0F
:102610001B78DBB1002302AA21462846FFF718FEEB
:102620000028CFD008AA2B4605F1300E14461868B2
:10263000083353F8041C1646734503C63246F6D1D8
:10264000186830602846FFF749FCD8E73B4602AAE5
:1026500021462846FFF7FCFD17B0F0BD19B101F582
:102660008961FFF79DBF0846704730B4134690F864
:10267000312072B991F8315015F0500F09D0D1E9DD
:102680000045002504F01F042C4302D130BCFFF7A5
:10269000DFBD002030BC704710B500230478CA03AA
:1026A000012B42EA5101C25C12FA81F189B204D1D4
:1026B000852C14BF0122032200E0012213441F2BAA
:1026C000EDD9084610BD10B5044604F08EFE58B191
:1026D00004F5047004F089FE30B1D4F840040368B6
:1026E000BDE81040DB691847002010BDF8B504466E
:1026F000006AA16901B10131012200F0DCFF01286B
:10270000054601D8002638E001230146206A1A4612
:1027100001F024F806460028F4D0A26994F833307A
:1027200022B943F0400384F8333025E0590613D52D
:102730000132954220D023F04003E16984F8333020
:10274000A369994208D24F1C206A3A4601F0C9F8A1
:102750000028D7D03946F3E74FF0FF322946206AE8
:1027600001F0BFF80028CDD0A16929B12A46206A1E
:1027700001F0B7F80028C5D0A5613046F8BD70B5A6
:1027800090F8333004469A0701D4002070BDC56923
:102790000DB9002528E05B0614D5066AD0E90201D0
:1027A00096F8452410F1FF3002F1090241F1FF31A2
:1027B000D2B206F0A7FF0023421C2946304600F0A3
:1027C000CDFF03E02946006A01F0A8F80028E0D117
:1027D000DBE701222046FFF765FB01350028D4D056
:1027E000037803F07F030370E9B294F830308B4232
:1027F000EFD20023206A84F8313084F83330FFF7B9
:1028000062FF70BD10B590F8313088B00446D9062B
:1028100001D400201DE000220023FFF7B2FC20229B
:1028200069462046FFF7D6FB38B12028F1D19DF844
:1028300000301A06EDD4002BF1D10823204684F88D
:10284000313094F8333043F0020384F83330FFF72B
:1028500096FF08B010BD00002DE9F34100260546A3
:10286000DFF8D0803746F1B295F830308B424AD34A
:1028700000222846FFF716FB044600284FD00378B5
:10288000C02B1DD0C12B37D0852B48D195F83130C6
:1028900003F037038380D8F8003033B30DF103021F
:1028A0000DF1060101A898479DF80330BDF80620F8
:1028B0006375BDF80430A281E3812282638214E053
:1028C00095F8333013F0400F437814BF43F0020300
:1028D00023F002034370D5E90423C0E90223EB6926
:1028E0004361D5E90223C0E906232A6A92F810322F
:1028F00043F0010382F8103239462046FFF7CCFE40
:1029000001360746AFE7012205F12401286A00F0ED
:1029100077FF20B14780286AFFF7D5FE30B995F8D8
:102920003230002043F0010385F8323002B0BDE8B8
:10293000F08100BFC466002010B590F83130044625
:102940000BB9012010BD90F833301A0607D503F0FB
:102950007F0380F83330BDE81040FFF77DBF006A89
:10296000FFF7B1FE0028ECD194F8323043F00103B8
:1029700084F8323010BD2DE9F04190F83130044632
:10298000580603D5206A01F091F800E0A068236A98
:10299000D3F83C341844B0F1806F58D22046FFF78A
:1029A000A5FE002853D0256A95F81032D90705D521
:1029B00005F5047004F019FD002848D04FF0FF33EE
:1029C000002605F508754FF4007245F8043C3146C1
:1029D00005F8106C284605F023F8226AA3694FF029
:1029E000010892F84514023BD2F82C748B401F4426
:1029F000236A93F8452408FA02F2B24209D9D3F8BF
:102A000040042A46B91903681B6A9847F8B1013691
:102A1000EEE794F83120520614D494F8332062F093
:102A20007F02D4E9020184F83320D3F83C24002348
:102A300080185941C4E90201D4E9040112184B413C
:102A4000C4E904232046BDE8F041FFF775BF00202C
:102A5000BDE8F08110B591F83130044613F0500F05
:102A60001AD040F60223FFF7F3FBA8B1102320464B
:102A700084F83130FFF77FFF70B1A3692046002250
:102A8000E3610023FFF77DFBC123204684F8333048
:102A9000BDE81040FFF750BF002010BDF0B51F4645
:102AA00097B0002305460C460192ADF814308DF81E
:102AB00051308DF852308DF8533090F83130002B72
:102AC00049D191F8313013F0500F44D013782F2BA7
:102AD0000DD1019B1A782F2A02D101330193F8E717
:102AE000216A08A8FFF724FA002834D008AC01AB0B
:102AF00002AA01992846FFF72FFA60B3019B1B78C1
:102B00001BB3002302AA21462846FFF7A1FB98B178
:102B100008AA2B4605F1300E14461868083353F8FE
:102B2000041C1646734503C63246F6D11868306059
:102B30002846FFF7D3F9DAE76FB102AA2146284603
:102B4000FFF788FF0028E3D105E002AA21462846C6
:102B5000FFF780FF00E0002017B0F0BDF0B50023C4
:102B60009DB004468DF831308DF832308DF8333019
:102B70008DF869308DF86A308DF86B3090F831300F
:102B800013F0180F01D100203AE0006A0B6A984256
:102B9000F9D140F601236846FFF702FD0028F2D084
:102BA0000EAA234604F1300716461868083353F876
:102BB000041C1546BB4203C52A46F6D1186809AA6B
:102BC00004F12403286007CA83E807009DF8303029
:102BD000204684F8303094F8333063F07F0384F873
:102BE0003330FFF7A9FE0028CDD0002330461593DF
:102BF00002238DF86B3008238DF86930FFF7BFFD95
:102C00001DB0F0BD2DE9F84F1C4690F83130064656
:102C100088461B079DF828B09DF82CA09DF83050E1
:102C20009DF8349039D5A2F2BC7297B27F2F34D878
:102C3000631E0B2B31D80BF1FF331E2B2DD8BAF1AD
:102C4000170F2AD83B2D28D8B9F13B0F25D8FFF70D
:102C500073FE10B34FEA690319F0010F4BEA4414F5
:102C600043EA451508BF4FF0000944EA47244FF0F6
:102C7000000745EACA2518BF4FF06409A4B2BB4655
:102C8000ADB208F0010AF9B296F830308B4234D375
:102C900000223046FFF706F910B90020BDE8F88F92
:102CA0000378852B04D0F8D3C03B012B1FD9F4E760
:102CB00096F83130326A03F03703838092F810328D
:102CC00043F0010382F81032BAF1000F01D00582FF
:102CD000448218F0020F1EBF80F8149005814481D1
:102CE00018F0040F1EBF80F815908581C4815946E5
:102CF0000137FFF7D1FC8346C5E7012206F1240125
:102D0000306A00F07DFD0028C7D0A0F802B0306A1C
:102D1000FFF7D9FCBDE8F88F73B590F8333004465F
:102D20009A0701D4002054E0C569002D40D003F07B
:102D30004003866903F0FF01F3B1236AD0E9020181
:102D400093F8452410F1FF3002F1090241F1FF31FF
:102D5000D2B206F0D7FC421C2EB1013D731CAD1B54
:102D600001932A4401E00195E6611AB30023019919
